:1000000062C7000091C700008FC700008DC70000C5
:100010008BC7000089C7000087C7000085C70000A4
:1000200083C7000081C700007FC700007DC70000B4
:100030007BC700000C94ED7B77C7000075C70000FC
:1000400073C7000071C700006FC700006DC70000D4
:100050006BC7000069C7000067C700000C947A8670
:1000600063C700000C94648A0C949A8A5DC70000F0
:100070005BC7000059C7000057C7000055C7000004
:1000800053C7000051C700004FC700004DC7000014
:100090004BC7000049C7000047C700000C94546DCF
:1000A00043C7000041C700003FC700003DC7000034
:1000B0003BC7000039C7000037C7000035C7000044
:1000C00033C7000031C700002FC700000C940F8B0E
:1000D0000C94458B29C700000C94BA8B0C94F08BC0
:1000E00023C70000284A084A314A314A314A314A76
:1000F000314A314A314A314A314A314A5F487148BE
:1001000078487E4885488B4890489948A048B74829
:10011000BA48314ACC48CF48D248D548EF48F14890
:10012000F848FF48124919492049314A314A314AB1
:10013000314A314A314A314A314A314A314A5B49BE
:10014000314A314A314A314A314A314A5F4AC787D6
:10015000CA87B987BD87C3870188CE87D287D887EA
:10016000DC87E087E687EA87EE870188F487F887EF
:10017000FC87084AD73B3BCE016E84BCBFFDC12F34
:100180003D6C74319ABD56833DDA3D00C77F11BE88
:10019000D9E4BB4C3E916BAAAABE000000803F0789
:1001A000634236B79BD8A71A39685618AEBAAB5512
:1001B0008C1D3CB7CC5763BD6DEDFD753EF61772D7
:1001C00031BF000000803F08000000BE92244912A9
:1001D0003EABAAAA2ABECDCCCC4C3E00000080BECD
:1001E000ABAAAAAA3E00000000BF000000803F00AA
:1001F00000000000084178D3BB4387D1133D190E9E
:100200003CC3BD4282AD2B3E68EC8276BED98FE105
:10021000A93E4C80EFFFBE01C4FF7F3F00000000FD
:1002200000003E4D6F74696F6E20627920756C74AA
:100230007261736F6E632073656E736F723A0A003A
:1002400023696E7075742044535463616C696272E3
:100250006174653A004E6F20445320546865726D96
:100260006F6D657465722100234E6F2073656E7328
:100270006F7220666F7220504D21004E6F207365A3
:100280006E736F722100504D313A322E353A313053
:10029000004D6561737572696E672E2E004F3220B6
:1002A000436F6E6300434F3220436F6E63005365AC
:1002B0006E736F72206572726F722100234E6F2011
:1002C00073656E736F722100434F3220436F6E630C
:1002D000004D6561737572696E67007048207661C4
:1002E0006C756500547572626964697479004E6F4B
:1002F0002073656E736F72210049522054656D70D2
:1003000065726174757265004D6561737572696EB1
:10031000672E2E004C6967687420496E74656E7391
:1003200069747900416E676C65732F00676574535B
:10033000656C665465737442697428293A200069B3
:1003400073496E74657272757074456E61626C6526
:10035000642831293A2000676574496E74657272A9
:100360007570744D617070696E672831293A20008C
:10037000676574496E74657272757074536F7572C7
:1003800063652831293A2000676574496E74657287
:1003900072757074536F7572636528293A2000670F
:1003A00065745261746528293A20332E3134313511
:1003B000393F00616363656C2E69734C6F77506FD2
:1003C00077657228293A2000616363656C2E697332
:1003D00041736C65657028293A2000616363656C20
:1003E0002E6973546170536F757263654F6E5A282E
:1003F000293A2000616363656C2E69735461705300
:100400006F757263654F6E5928293A2000616363E6
:10041000656C2E6973546170536F757263654F6EAE
:100420005828293A2000616363656C2E6973416323
:10043000746976697479536F757263654F6E5A2863
:10044000293A2000616363656C2E697341637469A6
:1004500076697479536F757263654F6E5928293ABE
:10046000200069734163746976697479536F75729A
:1004700063654F6E5828293A2000697354617044AF
:100480006574656374696F6E4F6E5A28293B2066E8
:10049000616C73653F2000697354617044657465D5
:1004A0006374696F6E4F6E5A28293B2074727565AC
:1004B0003F20006973546170446574656374696FAB
:1004C0006E4F6E5928293B2066616C73653F200092
:1004D0006973546170446574656374696F6E4F6EBF
:1004E0005928293B20747275653F20006973546157
:1004F00070446574656374696F6E4F6E5828293B4C
:100500002066616C73653F200069735461704465B7
:1005100074656374696F6E4F6E5828293B2074723E
:1005200075653F20006765745375707072657373ED
:1005300042697428293B2066616C73653F2000671F
:100540006574537570707265737342697428293BC2
:1005500020747275653F2000697341637469766920
:100560007479416328293A20006973496E61637484
:1005700069766974795A456E61626C656428293AB6
:1005800020006973496E61637469766974795945AD
:100590006E61626C656428293A20006973496E6156
:1005A0006374697669747958456E61626C65642814
:1005B000293A2000697341637469766974795A45F0
:1005C0006E61626C656428293A2000697341637426
:1005D000697669747959456E61626C656428293A57
:1005E00020006973416374697669747958456E6156
:1005F000626C656428293A200067657446726565F7
:1006000046616C6C4475726174696F6E28293A207A
:10061000006765744672656546616C6C5468726506
:1006200073686F6C6428293A200067657454696D9B
:1006300065496E616374697669747928293A200086
:10064000676574496E616374697669747954687218
:100650006573686F6C642829200067657441637452
:1006600069766974795468726573686F6C64282957
:100670002000676574446F75626C655461705769DA
:100680006E646F7728292000676574446F75626C0B
:10069000655461704C6174656E637928293A200055
:1006A0006765745461704475726174696F6E28294E
:1006B0003A2000676574417869734F6666736574A4
:1006C0002826782C2026792C20267A293A200067A3
:1006D00065745461705468726573686F6C6428291E
:1006E0003A200058595A2047733A200058595A2046
:1006F000434F554E54533A20007365742067616927
:100700006E735B5D3A006761696E735F6F726967F4
:100710005B5D3A00466C616D65204952004F66662C
:10072000206169722D636F6E642100497427732004
:10073000746F6F20636F6F6C210054656D7020695A
:10074000732066696E6521004973206169722D63AB
:100750006F6E64206F6E3F00497427732071756956
:10076000746520686F742100497427732076657260
:100770007920686F74210054656D702048756D692B
:100780006469747900234E6F2073656E736F7220F5
:10079000666F722074656D7020262068756D6964BF
:1007A00069747921004E6F2053656E736F7221005A
:1007B00054656D702048756D6964697479004F6681
:1007C00066206169722D636F6E642100497427731E
:1007D00020746F6F20636F6F6C210054656D702003
:1007E00069732066696E6521004973206169722D05
:1007F000636F6E64206F6E3F0049742773207175BC
:1008000069746520686F74210049742773207665C8
:10081000727920686F7421200023616E6F7468659F
:100820007220495220696E7075743D00236B6579A2
:10083000323D00236B6579323D00496E76616C690B
:1008400064206B65792100237265706C6965733D66
:1008500000233A53686F772F48696465204C4344FE
:10086000002A3A546869732048656C700044433A22
:10087000436C656172204C43440044423A526573B4
:100880006574204C6F676765720044373A4D6F742A
:10089000696F6E0044363A44532054656D700044CD
:1008A000353A555620496E74656E73697479004403
:1008B000343A4F3220636F6E632E0044333A434F15
:1008C0003220636F6E632E0044323A504D28313A25
:1008D000322E353A3130290044323A504D28313ADF
:1008E000322E353A3130292A0044313A5475726239
:1008F00069646974790044303A566F6C7461676555
:1009000000393A6F7220334420616363656C2E00B6
:10091000393A496E636C2E20616E672E00383A704A
:10092000482076616C756500373A49522054656DF0
:100930007000373A49522054656D702A00363A4D9E
:1009400061676E65746963206669656C6400353A39
:10095000476173204C6576656C00343A49522046F5
:100960006C616D6500333A4C6967687420496E7438
:100970002E00323A616E64204865696768740032FF
:100980003A54656D702050726573737572650031ED
:100990003A54656D702048756D69646974790030EA
:1009A0003A536F756E64204C6576656C00303A532F
:1009B0006F756E64204C6576656C2A0020202020BF
:1009C0002020202020202020202020002020202047
:1009D0002020202020202020202020002020202037
:1009E0002020202020202020202020200020202027
:1009F0002020202020202020202020202000202017
:100A00002020202020202020202020202020002006
:100A100020202020202020202020202020202000F6
:100A20004C6F6767657220446972656374696F6EA5
:100A300000232D2D2D2D2D2D2D2D2D2D2D2D2D2D1D
:100A40002D2D2D2D2D2D2D2D2D2D2D2D2D2D2D2DD6
:100A50002D2D2D2D2D2D00235265736F6C7574690E
:100A60006F6E3A20202000234D696E2056616C7510
:100A7000653A2020202000234D61782056616C7556
:100A8000653A202020200023556E69717565204944
:100A9000443A202020200023447269766572205653
:100AA00065723A202020002353656E736F723A20DE
:100AB00020202020202000232D2D2D2D204D61676A
:100AC0006E657469632053656E736F72202D2D2DD2
:100AD0002D2D2D2D2D2D2D2D2D2D2D2D2D2D2D2D46
:100AE0002D006E6F20484D4335383833206D6167D7
:100AF0006E657469632073656E736F72202E2E2E7F
:100B000020436865636B20776972696E67210020F6
:100B1000766F6C746167653D002354757262696419
:100B2000697479205570706572204C696D69743AEA
:100B3000200020766F6C746167653D0023434F325F
:100B4000207A65726F20766F6C74202800234F32F4
:100B50002063616C6962726174696F6E3A20002370
:100B6000547572626964697479204C6F776572207C
:100B70004C696D69742056313A20002350617261CE
:100B80006D65746572730043616C6962726174694A
:100B90006F6E2050726573737572653D00536561A9
:100BA000206C6576656C20502863616C63293D007C
:100BB000234572726F723A70726573737572652035
:100BC000424D503038352C20636865636B2077695F
:100BD00072696E67210049522054656D70207365FB
:100BE0006E736F7220666F756E6400504D322E35D5
:100BF0002073656E736F72206C696B656C7920660B
:100C00006F756E6400536F756E64204C6576656C0D
:100C10002073656E736F7220666F756E6400536526
:100C20006E736F7220736C6F7420616E64207479C0
:100C300070653A0057656C636F6D6520746F204571
:100C40006455484B00005EBCE2613FDD83C29C7E80
:100C500020A3FD1F41009D23BE46DB65F88C11AF2C
:100C600032CA57E97400000A0B02090C0D0E08077E
:100C7000030401000000000000000000000000006C
:100C80000000000000000000000000000000000064
:100C90000012111000000000000000000000000021
:100CA00000000000000000000000000102102020F1
:100CB00008081020401020408002010201080402B0
:100CC0000101020408102040808040201008040226
:100CD000018004020180402010080402010804027F
:100CE0000101020408102040800102040810204085
:100CF0008005050505070508080808020202020A22
:100D00000A080804040404010101010101010103AE
:100D100003030303030303040707070C0C0C0C0C69
:100D20000C0C0C0202020206060606060606060B5C
:100D30000B0B0B0B0B0B0B000020002300260029D4
:100D4000002C002F00320000010000030106010901
:100D50000100002200250028002B002E0031003465
:100D60000002010000050108010B01000021002420
:100D70000027002A002D003000330001010000048C
:100D80000107010A014E414E494E495459494E4608
:100D9000CDCCCC3D0AD7233C17B7D13877CC2B32FA
:100DA0009595E6241FB14F0A000020410000C8427B
:100DB00000401C4620BCBE4CCA1B0E5AAEC59D74DA
:100DC00000407A10F35A00A0724E18090010A5D402
:100DD000E80000E87648170000E40B54020000CA5F
:100DE0009A3B000000E1F5050000809698000000A5
:100DF00040420F000000A086010000001027000004
:100E00000000E803000000006400000000000A0089
:100E1000000000000100000000002C76D888DC678C
:100E20004F0823DFC1DFAE59E1B1B796E5E3E453E4
:100E3000C63AE651997696E8E6C28426EB898C9B01
:100E400062ED407C6FFCEFBC9C9F40F2BAA56FA5A1
:100E5000F490055A2AF75C936B6CF9676DC11BFC23
:100E6000E0E40D47FEF520E6B500D0ED902E03003E
:100E7000943577050080841E080000204E0A00008B
:100E800000C80C333333330F986E12831141EF8D4A
:100E90002114893BE65516CFFEE6DB18D1844B388A
:100EA0001BF77C1D901DA4BBE424203284725E22BB
:100EB0008100C9F124ECA1E53D2703356B6CCC8A98
:100EC000778B228CD93511241FBECFEFD1E2DEBF44
:100ED000CDBF00E00CBF1BE0A0E0B2E0EAE0F1E42F
:100EE00001E00BBF02C007900D92A23AB107D9F7FB
:100EF00021E1A2EABBE001C01D92A33AB207E1F7EB
:100F00001EE0C4ECDEE000E006C022970109FE010D
:100F10000BBF0E94F798CA3BD10780E00807A9F7EA
:100F20000E9425940C9474A06BC8CF92DF92EF922C
:100F3000FF920F931F93E82FF92F05C0015011095D
:100F40002109310961F1908196239417B9F305C005
:100F5000015011092109310911F19081962394134F
:100F6000F7CFC12CD12CE12CF12C0AC08FEFC81A7D
:100F7000D80AE80AF80A0C151D052E053F0579F078
:100F800080818623841791F36C2D7D2D8E2D9F2DCE
:100F90001F910F91FF90EF90DF90CF90089560E048
:100FA00070E080E090E01F910F91FF90EF90DF9054
:100FB000CF90089529EB3AE0FC0131832083089516
:100FC000089529EB3AE0FC01318320830C9433949B
:100FD0002F923F924F925F926F927F928F929F9249
:100FE000AF92BF92CF92DF92EF92FF920F931F9337
:100FF000CF93DF93CDB7DEB72E970FB6F894DEBF51
:101000000FBECDBF8C017E876D87DC014D915C9159
:10101000119712962D913C911397421753072CF478
:10102000942F852FA901292F382FD801149660E01D
:1010300070E0CB01E2E0F0E0ED84FE84EE15FF0508
:1010400044F5CD90DD90C216D3065CF44901AA2484
:1010500097FCA094BA2C680D791D8A1D9B1D9601E2
:1010600016C04C155D055CF44A01AA2497FCA094B7
:10107000BA2C680D791D8A1D9B1DA60108C0EE249F
:10108000D7FCE094FE2C6C0D7D1D8E1D9F1D3196AE
:10109000D3CF0E94CC956B017C016D857E8562501B
:1010A0007109882777FD8095982F0E94CC959B0128
:1010B000AC01C701B6010E9400956B017C012D8532
:1010C0003E85243131050CF4BFC04801412C512C20
:1010D0003201A12CB12CD4016D917D914D01882755
:1010E00077FD8095982F0E94CC95A70196010E94CC
:1010F00035949B01AC010E9460979B01AC01C30138
:10110000B2010E9436942B013C01BFEFAB1ABB0A1F
:10111000ED85FE85AE16BF06F1F6BF01615071097F
:10112000882777FD8095982F0E94CC959B01AC0174
:10113000C301B2010E9400950E9413984B015C010B
:1011400020E030E040E85FE30E94A19618160CF022
:101150007BC018870F83212C312C1B821C821D829F
:101160001E821A821982AF81B8858D919D91B887B0
:10117000AF839C01442737FD4095542F29873A8738
:101180004B875C87CA01B9010E94CC95A7019601E3
:101190000E9435942B013C0120E030E0A9010E941F
:1011A000A196181624F0C301B201905802C0C301E1
:1011B000B201A50194010E94FC9487FF13C08B81AA
:1011C0009C81AD81BE8129853A854B855C85820FE6
:1011D000931FA41FB51F8B839C83AD83BE833FEFFA
:1011E000231A330A49815A814F5F5F4F5A834983DB
:1011F0008D859E854817590709F0B5CF20E030E06E
:1012000040EC5FE3C501B4010E9460974B015C01B3
:1012100095E0291631040CF49CCF6B817C818D8183
:101220009E810E94CC956B017C01B101882777FDDE
:101230008095982F0E94CC959B01AC01C701B60107
:101240000E9400956B017C01C701B6012E960FB676
:10125000F894DEBF0FBECDBFDF91CF911F910F91EC
:10126000FF90EF90DF90CF90BF90AF909F908F90C6
:101270007F906F905F904F903F902F900895CF9305
:10128000DF93EC01FB01248135810E947093CE0134
:10129000DF91CF91089526E00C94D189DC01ED9186
:1012A000FC910190F081E02D1994EF92FF920F9341
:1012B0001F93CF93DF931F92CDB7DEB77C01FC0164
:1012C00000811181C80169830E94739C698168173C
:1012D00019F0C8010E947B9CC7010F90DF91CF914C
:1012E0001F910F91FF90EF900895EF92FF920F934F
:1012F0001F93CF93DF931F921F92CDB7DEB705EEFA
:101300001BE0855E9B407C01C701800F911FF801A7
:1013100061918F019A838983CE010196C6DFFCE03B
:101320000D351F0789F785EE9BE00F900F90DF9139
:10133000CF911F910F91FF90EF9008950F931F93FE
:10134000CF93DF931F921F92CDB7DEB70AE21EE064
:10135000F80160818EED93E09A838983CE01019636
:10136000A4DFF80161818FED93E09A838983CE0138
:1013700001969BDFC8010F900F90DF91CF911F91D5
:101380000F9108950F931F93CF93DF9300D000D058
:10139000CDB7DEB78C018091FB0C8823A1F064E00F
:1013A00077E0CE0101960E948990B801CE010196A6
:1013B0000E948292BC0186EC9FE00E94EF8CCE01DD
:1013C00001960E941E9026960FB6F894DEBF0FBEBF
:1013D000CDBFDF91CF911F910F910895BF92CF9212
:1013E000DF92EF92FF920F931F93CF93DF93CDB7CE
:1013F000DEB762970FB6F894DEBF0FBECDBF6C01AB
:101400007B018A018091F504882309F480C08091D2
:10141000F404882309F47BC077FF09C0E094F094BA
:1014200040E06E2D8CE19EE00E9447664CC040E09B
:1014300060E08CE19EE00E9447660E94C48628EE30
:1014400033E040E050E00E94C598BA01A9012AE0CB
:10145000CE0101960E947F91BE016F5F7F4FCE014A
:1014600007960E9408916EEA78E0CE0107960E94E6
:101470009392BC01CE010D960E940891CE01079671
:101480000E941E90CE0101960E941E90BE01635FD5
:101490007F4F8CE19EE00E94C68CB98840E06B2DA6
:1014A0008CE19EE00E944766E114F10411F4EB2CFC
:1014B00006C040E06E2D8CE19EE00E944766CE01A2
:1014C0000D960E941E90B6018CE19EE00E94C68C93
:1014D0006FE07AE08CE19EE00E94A38CF6016481CB
:1014E0006E0D40E08CE19EE00E9447660E94C4863B
:1014F0006093180E7093190E80931A0E90931B0E22
:10150000B801882777FD8095982F0E94F386629610
:101510000FB6F894DEBF0FBECDBFDF91CF911F9104
:101520000F91FF90EF90DF90CF90BF9008954F9272
:101530005F926F927F92AF92BF92CF92DF92EF92C3
:10154000FF920F931F93CF93DF93CDB7DEB76297D0
:101550000FB6F894DEBF0FBECDBF6C017B015A0100
:101560008091F504882309F498C08091F4048823BD
:1015700009F493C00E94C4860091180E1091190EB0
:1015800020911A0E30911B0E4090E8045090E9040F
:101590006090EA047090EB04040D151D261D371DA4
:1015A000061717072807390708F077C0F7FE0AC0A3
:1015B00087010095109540E0602F8CE19EE00E942D
:1015C000476647C040E060E08CE19EE00E944766CD
:1015D0000E94C48628EE33E040E050E00E94C598A7
:1015E000BA01A9012AE0CE0101960E947F91BE01B5
:1015F0006F5F7F4FCE0107960E9408916EEA78E0F8
:10160000CE0107960E949392BC01CE010D960E94D6
:101610000891CE0107960E941E90CE0101960E946D
:101620001E90BE01635F7F4F8CE19EE00E94C68CDE
:1016300009891A89E114F10441F00E0D1F1D40E0E3
:10164000602F8CE19EE00E944766CE010D960E94BD
:101650001E90B6018CE19EE00E94C68C6EEF79E090
:101660008CE19EE00E94A38CF6016481600F40E053
:101670008CE19EE00E9447660E94C4866093180E2B
:101680007093190E80931A0E90931B0EB501882744
:1016900077FD8095982F0E94F38662960FB6F89496
:1016A000DEBF0FBECDBFDF91CF911F910F91FF9095
:1016B000EF90DF90CF90BF90AF907F906F905F9052
:1016C0004F9008958F929F92AF92BF92CF92DF92E8
:1016D000EF92FF920F931F93CF93DF937C016B01E7
:1016E000EA018091F504882309F474C08091F40420
:1016F000882309F46FC077FF1CC0C094D09441E0E8
:101700006C2D8CE19EE00E944766B7018CE19EE063
:101710000E94C68C6DEE79E08CE19EE00E94A38C65
:10172000F70164816C0D41E08CE19EE00E94476608
:101730003EC00E94C4860091E8041091E904209103
:10174000EA043091EB048090140E9090150EA09056
:10175000160EB090170E080D191D2A1D3B1D0617F9
:10176000170728073907B0F541E06C2D8CE19EE0A2
:101770000E944766B7018CE19EE00E94C68C6CED2A
:1017800079E08CE19EE00E94A38CF70164816C0DEE
:1017900041E08CE19EE00E9447660E94C48660930F
:1017A000140E7093150E8093160E9093170EBE01B3
:1017B000882777FD8095982FDF91CF911F910F910A
:1017C000FF90EF90DF90CF90BF90AF909F908F9061
:1017D0000C94F386DF91CF911F910F91FF90EF90C2
:1017E000DF90CF90BF90AF909F908F9008958091A1
:1017F000F504882379F08091F404882359F06FED83
:101800008CE19EE00E94D58C6BE975E08CE19EE056
:101810000C94D48C0895CF93DF93EC018091F50460
:101820008823A1F08091F404882381F06FED8CE18E
:101830009EE00E94D58C8C819D81892B39F0BE0160
:101840008CE19EE0DF91CF910C94C68CDF91CF911B
:1018500008958091F504882301F18091F404882390
:10186000E1F08CE19EE00E943B6640E060E08CE1AC
:101870009EE00E9447666CEC79E08CE19EE00E945D
:10188000A38C41E060E08CE19EE00E9447666CEB37
:1018900079E08CE19EE00C94A38C0895CF93DF93C4
:1018A000CDB7DEB72C970FB6F894DEBF0FBECDBF15
:1018B00080915B0C90915C0C892B01F56AE075E0DE
:1018C000CE0107960E9489906EE07EE0CE010796D9
:1018D0000E948292BC01CE0101960E94089148ECC0
:1018E00050E06FEF7FEFCE01019678DDCE010196DB
:1018F0000E941E90CE0107960E941E9080915B0C64
:1019000090915C0C019701F56EE075E0CE010796B1
:101910000E9489906EE07EE0CE0107960E9482923E
:10192000BC01CE0101960E94089148EC50E06FEF97
:101930007FEFCE01019652DDCE0101960E941E90EE
:10194000CE0107960E941E9064E175E0CE010796D5
:101950000E94899068E07EE0CE0107960E94829204
:10196000BC01CE0101960E94089140ED57E06FEF57
:101970007FEFCE010196A6DECE0101960E941E9059
:10198000CE0107960E941E908091280E9091290EFC
:10199000019719F46DEA79E002C06FE979E0CE01B0
:1019A00001960E94279248EC50E06FEF7FEFCE0146
:1019B0000196BDDDCE0101960E941E906FE879E090
:1019C000CE0101960E94279240ED57E06FEF7FEF26
:1019D000CE01019677DECE0101960E941E906FE740
:1019E00079E0CE0101960E94279248EC50E06FEF1B
:1019F0007FEFCE0101969BDDCE0101960E941E90E5
:101A000062E779E0CE0101960E94279240ED57E00F
:101A10006FEF7FEFCE01019655DECE0101960E9459
:101A20001E9065E679E0CE0101960E94279248EC6F
:101A300050E06FEF7FEFCE01019679DDCE01019688
:101A40000E941E906AE579E0CE0101960E942792DD
:101A500040ED57E06FEF7FEFCE01019633DECE0110
:101A600001960E941E906EE479E0CE0101960E94DC
:101A7000279248EC50E06FEF7FEFCE01019657DDE3
:101A8000CE0101960E941E906DE379E0CE01019691
:101A90000E94279240ED57E06FEF7FEFCE01019655
:101AA00011DECE0101960E941E908091280E909129
:101AB000290E039719F462E379E002C068E279E045
:101AC000CE0101960E94279248EC50E06FEF7FEF25
:101AD000CE0101962CDDCE0101960E941E906DE193
:101AE00079E0CE0101960E94279240ED57E06FEF1A
:101AF0007FEFCE010196E6DDCE0101960E941E9099
:101B000060E179E0CE0101960E94279248EC50E016
:101B10006FEF7FEFCE0101960ADDCE0101960E94A4
:101B20001E9061E079E0CE0101960E94279240ED7F
:101B300057E06FEF7FEFCE010196C4DDCE01019635
:101B40000E941E9066EF78E0CE0101960E942792D7
:101B500048EC50E06FEF7FEFCE010196E8DCCE015C
:101B600001960E941E9069EE78E0CE0101960E94D7
:101B7000279240ED57E06FEF7FEFCE010196A2DD97
:101B8000CE0101960E941E908091280E9091290E00
:101B9000029719F468ED78E002C068EC78E0CE01B5
:101BA00001960E94279248EC50E06FEF7FEFCE0144
:101BB0000196BDDCCE0101960E941E906BEB78E091
:101BC000CE0101960E94279240ED57E06FEF7FEF24
:101BD000CE01019677DDCE0101960E941E906FEA3C
:101BE00078E0CE0101960E94279248EC50E06FEF1A
:101BF0007FEFCE0101969BDCCE0101960E941E90E4
:101C00006FE978E0CE0101960E94279240ED57E0FF
:101C10006FEF7FEFCE01019655DDCE0101960E9458
:101C20001E9064E978E0CE0101960E94279248EC6C
:101C300050E06FEF7FEFCE01019679DCCE01019687
:101C40000E941E906AE878E0CE0101960E942792D9
:101C500040ED57E06FEF7FEFCE01019633DDCE010F
:101C600001960E941E906AE778E0CE0101960E94DC
:101C7000279248EC50E06FEF7FEFCE01019657DCE2
:101C8000CE0101960E941E906DE678E0CE0101968D
:101C90000E94279240ED57E06FEF7FEFCE01019653
:101CA00011DDCE0101960E941E9061E678E0CE0122
:101CB00001960E94279248EC50E06FEF7FEFCE0133
:101CC000019635DCCE0101960E941E9061E578E018
:101CD000CE0101960E94279240ED57E06FEF7FEF13
:101CE000CE010196EFDCCE0101960E941E902C964B
:101CF0000FB6F894DEBF0FBECDBFDF91CF91089530
:101D00004F925F926F927F928F929F92AF92BF920B
:101D1000CF92DF92EF92FF92CF93DF93CDB7DEB7F2
:101D20002C970FB6F894DEBF0FBECDBF92DD8EE2CA
:101D30009DE00E94D6622B013C018EE29DE00E9454
:101D400067624B015C0160913802709139028091A9
:101D50003A0290913B020E94CC95AB01BC018EE20D
:101D60009DE00E9473646B017C01C301B2010E947B
:101D7000CC9520E030E048EC52E40E940095AB01A5
:101D8000BC0122E0CE0101960E94AB91BE016F5FC3
:101D90007F4F80E09DE00E941091CE0101960E944D
:101DA0001E9061E279E080E09DE00E94609260E038
:101DB0007DE086E09DE00E94F3906DE179E0CE0148
:101DC00001960E94899060E07DE0CE0101960E941C
:101DD0008292BC0180E09DE00E94F390CE010196CA
:101DE0000E941E9064E976E08CE09DE00E942691BE
:101DF00021E0B501A401CE0101960E94AB91BE0184
:101E00006F5F7F4F8CE09DE00E945A92CE01019659
:101E10000E941E9069E175E08CE09DE00E94609256
:101E200021E0B701A601CE0107960E94AB91BE0149
:101E3000695F7F4FCE0101960E9408916CE677E0C2
:101E4000CE0101960E949392BC018CE09DE00E941D
:101E50005A92CE0101960E941E90CE0107960E94D2
:101E60001E9060E07DE0CE0101960E94089160E343
:101E700075E0CE0101960E9493926CE07DE00E9495
:101E80008292BC018CE09DE00E94F390CE0101960D
:101E90000E941E9066E07DE0CE0101960E940891AE
:101EA0004AE050E060E070E0CE01019697DACE01A2
:101EB00001960E941E9021E0B501A401CE01019679
:101EC0000E94AB91BE016F5F7F4F82E19DE00E9457
:101ED0001091CE0101960E941E9062E17DE0CE013C
:101EE00001960E9408914AE050E06FEF7FEFCE012B
:101EF0000196E8DBCE0101960E941E906FE175E02D
:101F0000CE0101960E948990CE01019684DCCE011B
:101F100001960E941E9021E0B701A601CE0107960E
:101F20000E94AB91BE01695F7F4FCE0101960E9476
:101F300008916CE677E0CE0101960E949392BC0175
:101F400082E19DE00E94F390CE0101960E941E90D6
:101F5000CE0107960E941E9062E17DE0CE010196BF
:101F60000E9408914AE050E068EF7FEFCE010196B1
:101F7000A9DBCE0101960E941E908091FD0C882362
:101F800031F068E572E080E090E00E94F3862C96E4
:101F90000FB6F894DEBF0FBECDBFDF91CF91FF909B
:101FA000EF90DF90CF90BF90AF909F908F907F90F9
:101FB0006F905F904F900895CF93DF93EC018C81E9
:101FC0009D81892B61F0BE0186EC9FE00E94EF8C21
:101FD000BE0180E091E1DF91CF910C94EF8CDF9115
:101FE000CF9108951F93CF93DF93CDB7DEB7A89716
:101FF0000FB6F894DEBF0FBECDBF182F85E49DE06D
:102000000E943C6A81110EC062EE7AE0CE01019618
:102010000E942792CE010196CFDFCE0101960E9449
:102020001E90A8C0BE016F5F7F4F85E49DE00E94B7
:102030001E69112309F498C08091FB0C882309F4D0
:1020400093C067EB7AE086EC9FE00E94DF8C67EA42
:102050007AE086EC9FE00E94A38CBE016F5F7F4F09
:1020600086EC9FE00E94FF8C67E97AE086EC9FE0B7
:102070000E94A38C4D855E856F8578892AE030E0CB
:1020800086EC9FE00E94DB8D67E87AE086EC9FE0BB
:102090000E94A38C49895A896B897C892AE030E0A7
:1020A00086EC9FE00E94DB8D67E77AE086EC9FE09C
:1020B0000E94A38C20E030E040E251E4698D7A8DEB
:1020C0008B8D9C8D0E946097AB01BC0122E030E0BB
:1020D00086EC9FE00E94F78E62E375E086EC9FE05D
:1020E0000E94FF8C67E67AE086EC9FE00E94A38C5A
:1020F00020E030E040E251E46D8D7E8D8F8D98A11F
:102100000E946097AB01BC0122E030E086EC9FE0CA
:102110000E94F78E62E375E086EC9FE00E94FF8CE0
:1021200067E57AE086EC9FE00E94A38C20E030E037
:1021300040E251E469A17AA18BA19CA10E94609721
:10214000AB01BC0122E030E086EC9FE00E94F78EFC
:1021500062E375E086EC9FE00E94FF8C61E37AE029
:1021600086EC9FE00E94DF8C64EF71E080E090E0FD
:102170000E94F386A8960FB6F894DEBF0FBECDBFBF
:10218000DF91CF911F9108954F925F926F927F924E
:102190008F929F92AF92BF92CF92DF92EF92FF9277
:1021A0000F931F93CF93DF93CDB7DEB7CA54D109F6
:1021B0000FB6F894DEBF0FBECDBF8C0164E97BE0A3
:1021C000CE01CD960E94899064E97BE0CE01C7964E
:1021D0000E948990BE016F5F7F4F85E49DE00E9461
:1021E000CF6A4D885E886F88788CC98CDA8CEB8CCE
:1021F000FC8C8D8D9E8DAF8DB8A12B968CAF9DAF35
:10220000AEAFBFAF2B97C8010197039708F0E2C1AB
:10221000A7019601C301B20190580E94A9942BED29
:102220003FE049EC5FE30E94369420913402309104
:10223000350240913602509137020E9436944B018C
:102240005C0120E030E0A9010E94FC9487FD09C0F8
:102250008092E90C9092EA0CA092EB0CB092EC0CFC
:1022600010C02BED3FE049EC50E4C501B4010E94E1
:1022700036946093E90C7093EA0C8093EB0C909386
:10228000EC0C8090E90C9090EA0CA090EB0CB090D4
:10229000EC0C2BED3FE049EC50E4C501B4010E9489
:1022A000A196181684F42BED3FE049EC50E4C501EB
:1022B000B4010E9435946093E90C7093EA0C80930A
:1022C000EB0C9093EC0C20E030E044E353E460919D
:1022D000E90C7091EA0C8091EB0C9091EC0C0E944F
:1022E00060972BED3FE049E450E40E940095609335
:1022F000E50C7093E60C8093E70C9093E80C0E9439
:1023000099954AE0CE018B960E94549166E375E060
:10231000CE0185960E948990BE01655D7F4FCE01FA
:1023200085960E94829260E475E00E949392BC01BF
:1023300082E19DE00E94F390CE0185960E941E905E
:10234000CE018B960E941E908090E50C9090E60C3A
:10235000A090E70CB090E80C20E030E044EB52E4B1
:10236000C501B4010E94FC94181694F020E030E0FE
:1023700040E05FE3C501B4010E9436940E94999544
:102380004AE0CE018B960E94549167E475E023C029
:1023900020E030E044E353E4C501B4010E94FC9422
:1023A0001816A4F1A501940160E070E884E393E4B9
:1023B0000E9435946093E50C7093E60C8093E70CD3
:1023C0009093E80C0E9499954AE0CE018B960E946A
:1023D00054916AE475E0CE0185960E948990BE0111
:1023E000655D7F4FCE0185960E948292BC01CE0131
:1023F000CD960E94F390CE0185960E941E90CE014C
:102400008B960E941E906CE879E063C020E030E07B
:1024100047E853E4C501B4010E94FC94181604F186
:1024200020E030E044E353E4C501B4010E94359458
:1024300020E030E040E05FE30E9436946093E50CDA
:102440007093E60C8093E70C9093E80C0E949995AA
:102450004AE0CE018B960E9454916AE475E01FC059
:10246000A501940160E070E084EB93E40E94359450
:1024700020E030E040E05FE30E9436946093E50C9A
:102480007093E60C8093E70C9093E80C0E9499956A
:102490004AE0CE018B960E94549167E475E0CE012C
:1024A00085960E948990BE01655D7F4FCE0185961D
:1024B0000E948292BC01CE01CD960E94F390CE0183
:1024C00085960E941E90CE018B960E941E906DE410
:1024D00075E0CE01C7960E942691BE01635C7F4FD6
:1024E000CE0185960E9408914AE050E060E070E0DD
:1024F000CE0185960E94EE09CE0185960E941E901F
:102500000E94C4862091E8043091E9044091EA04D5
:102510005091EB048090180E9090190EA0901A0E16
:10252000B0901B0E280D391D4A1D5B1D261737075D
:102530004807590708F441C20E94C4860E94CA9500
:102540004B015C016091E8047091E9048091EA0418
:102550009091EB040E94CC9520E030E040E85EE3EF
:102560000E94609727966CAF7DAF8EAF9FAF279785
:102570006091180E7091190E80911A0E90911B0E99
:102580000E94CC959B01AC0127966CAD7DAD8EADC4
:102590009FAD27970E9436949B01AC01C501B40101
:1025A0000E94FC9487FD09C260E375E0CE01859628
:1025B0000E948990BE01695C7F4FCE0185960E9482
:1025C0008292BC01CE01CD960E945A92CE01859690
:1025D0000E941E90C8010297029708F0C8C120E02F
:1025E00030E040E251E4C301B2010E9460974B0128
:1025F0005C0120E030E040E251E4C701B6010E94F6
:1026000060976B017C0120E030E040E251E42B96C2
:102610006CAD7DAD8EAD9FAD2B970E9460972B0169
:102620003C010E94C48620915D0C30915E0C40916B
:102630005F0C5091600C621B730B840B950B0E9416
:10264000CA9520E030E04AE754E40E940095AB01CF
:10265000BC0123E0CE018B960E94AB9163E675E04E
:10266000CE0185960E948990BE01655D7F4FCE01A7
:1026700085960E9482926EEA78E00E949392BC0155
:1026800080E09DE00E94F390CE0185960E941E900E
:10269000CE018B960E941E9060E07DE0CE01859673
:1026A0000E94089162E17DE0CE0185960E948292AF
:1026B000BE01635C7F4F0E948292BC01CE01CD9629
:1026C0000E94F390CE0185960E941E906FE475E003
:1026D0008CE09DE00E94269121E0B501A401CE018D
:1026E00085960E94AB91BE016B5D7F4F8CE09DE0B3
:1026F0000E945A92CE0185960E941E9021E0B3015D
:10270000A201CE0185960E94AB9121E0B701A601FE
:10271000CE01C1960E94AB9160E375E0CE018B962D
:102720000E948990BE016F5C7F4FCE018B960E9404
:10273000829260E375E00E949392BE016B5D7F4FD1
:102740000E9482926AE575E00E949392BC018CE03F
:102750009DE00E945A92CE018B960E941E90CE015F
:10276000C1960E941E90CE0185960E941E90A501E2
:102770009401C501B4010E9460974B015C01A7015F
:102780009601C701B6010E9460979B01AC01C5018B
:10279000B4010E9436946B017C01A3019201C30134
:1027A000B2010E9460979B01AC01C701B6010E9473
:1027B00036940E9413986093E10C7093E20C80931E
:1027C000E30C9093E40C6EE575E08CE09DE00E94D4
:1027D00060924091E10C5091E20C6091E30C709199
:1027E000E40C21E0CE018B960E94AB91BE01655DA9
:1027F0007F4FCE0185960E94089163E375E0CE017C
:1028000085960E949392BC0182E19DE00E94F39024
:10281000CE0185960E941E90CE018B960E941E903E
:1028200062E17DE08CE09DE00E945A92C090E10C54
:10283000D090E20CE090E30CF090E40C20E030E06B
:102840004AE754E4C701B6010E94A19687FD29C05A
:1028500020E030E04AE754E4C701B6010E94009549
:10286000AB01BC0123E0CE018B960E94D991BE0141
:10287000655D7F4FCE0185960E94089164E375E007
:10288000CE0185960E949392BC0182E19DE00E9458
:10289000F390CE0185960E941E90CE018B960E94E9
:1028A0001E9020E030E64AE656E46091E10C70911B
:1028B000E20C8091E30C9091E40C0E94FC94BE0128
:1028C000635C7F4F87FF4FC0CE0185960E940891C1
:1028D00062E675E0CE0185960E9493926CE07DE001
:1028E0000E948292BC018CE09DE00E94F390CE0198
:1028F00085960E941E900330110599F46CE07DE0EE
:10290000CE0185960E940891CE01859655DBCE01B9
:1029100085960E941E9064E97BE08CE09DE00E9419
:10292000269165E675E0CE018B960E94899062E162
:102930007DE0CE018B960E948292BC01CE018596ED
:102940000E9408914AE050E06FEF7FEFCE0185963C
:102950000E94620BCE0185960E941E90CE018B963E
:102960000E941E9004C08CE09DE00E94F3906AE0FB
:1029700070E080E090E00E94F386CE01C7960E944E
:102980001E90CE01CD960E941E90C65BDF4F0FB603
:10299000F894DEBF0FBECDBFDF91CF911F910F9195
:1029A000FF90EF90DF90CF90BF90AF909F908F906F
:1029B0007F906F905F904F90089564E97BE0CE0127
:1029C00085960E948990CE0185960E940B0CCE01BF
:1029D00085960E941E90BE01695C7F4F8CE19EE04F
:1029E0000E94C68CE1CD8F929F92AF92BF92CF9200
:1029F000DF92EF92FF920F931F93CF93DF9300D05C
:102A000000D0CDB7DEB78C01C0900A02D0900B0287
:102A1000E0900C02F0900D0220E030E040E450E441
:102A2000C701B6010E94A19618166CF420E030E0B0
:102A30004AE754E4C701B6010E9460970E94999545
:102A40006B017C0106C080E3C82E85E7D82EE12CFF
:102A5000F12C0E94290C40E060E08CE19EE00E9495
:102A600047666EE675E08CE19EE00E94D48C41E002
:102A700060E08CE19EE00E9447666FE775E08CE1C4
:102A80009EE00E94D48C64E670E080E090E00E94BA
:102A9000F3860E94C48660935D0C70935E0C8093F5
:102AA0005F0C9093600C0E94C48680905D0C9090A7
:102AB0005E0CA0905F0CB090600CDC01CB0188191B
:102AC0009909AA09BB098C159D05AE05BF055CF4E3
:102AD000C8015ADB0E94C48664E170E080E090E0A7
:102AE0000E94F386E0CF0130110509F041C06CE08F
:102AF0007DE086E09DE00E94F3900E94290C66E054
:102B00007DE0CE0101960E9408914AE050E060E02D
:102B100070E0CE0101960E94EE09CE0101960E945E
:102B20001E9060E27AE0CE0101960E9427924AE070
:102B300050E06FEF7FEFCE0101960E94620BCE0155
:102B400001960E941E9067E875E0CE0101960E94F2
:102B500089906CE07DE0CE0101960E948292BC01DA
:102B60008CE09DE00E94F390CE0101960E941E90A1
:102B700026960FB6F894DEBF0FBECDBFDF91CF9182
:102B80001F910F91FF90EF90DF90CF90BF90AF908B
:102B90009F908F900895CF92DF92EF92FF92CF9304
:102BA000DF9300D000D0CDB7DEB70E94290C6EE1D4
:102BB00070E080E090E00E94F3868EE29DE00E944B
:102BC00067626B017C0164E670E080E090E00E9447
:102BD000F38664E976E08CE09DE00E94269121E096
:102BE000B701A601CE0101960E94AB91BE016F5FB5
:102BF0007F4F8CE09DE00E945A92CE0101960E9488
:102C00001E906CE07DE0CE0101960E9408914AE0A2
:102C100050E060E070E0CE0101960E94EE09CE0126
:102C200001960E941E900E94F70B6AE975E08CE005
:102C30009DE00E946092C092F10CD092F20CE09262
:102C4000F30CF092F40C20E030E040EF51E4C701C7
:102C5000B6010E94A19687FD03C069E078E054C0E8
:102C600020E030E040ED51E4C701B6010E94A1969A
:102C700087FD1FC069EF77E0CE0101960E94279281
:102C80004AE050E06FEF7FEFCE0101960E94620BA9
:102C9000CE0101960E941E908091F804882331F0A5
:102CA0006CED75E080E090E00E94F38669EE77E0DD
:102CB0002BC020E030E040EB51E4C701B6010E9498
:102CC000A19687FD03C06BED77E01EC06CEC77E04A
:102CD000CE0101960E9427924AE050E06FEF7FEF0D
:102CE000CE0101960E94620BCE0101960E941E90B9
:102CF0008091F804882331F06CED75E080E090E07D
:102D00000E94F3866EEB77E0CE0101960E94279237
:102D10004AE050E06FEF7FEFCE0101960E94620B18
:102D2000CE0101960E941E906CE271E080E090E07E
:102D30000E94F3868091F804882331F068EE73E0F6
:102D400080E090E00E94F38626960FB6F894DEBFEE
:102D50000FBECDBFDF91CF91FF90EF90DF90CF906E
:102D60000895CF92DF92EF92FF92CF93DF93CDB78A
:102D7000DEB72C970FB6F894DEBF0FBECDBF60EB69
:102D800077E0CE0101960E9427924AE050E06FEF73
:102D90007FEFCE0101960E94620BCE0101960E9448
:102DA0001E906091C6047091C70486E79DE00E9462
:102DB000A364E12CF12C64E670E080E090E00E94D6
:102DC000F3866091C6047091C70486E79DE00E9477
:102DD000A3642FEFE21AF20A23E0E216F1045CF397
:102DE0002AE0E216F1041CF4892B29F703C0892B91
:102DF00009F0D4C06091780D7091790D882777FD26
:102E00008095982F0E94CC956B017C016093F10C0A
:102E10007093F20C8093F30C9093F40C6091760D08
:102E20007091770D882777FD8095982F0E94CC951B
:102E30006093ED0C7093EE0C8093EF0C9093F00C7C
:102E400021E0B701A601CE0107960E94AB9164E98B
:102E500076E0CE0101960E948990BE01695F7F4FA6
:102E6000CE0101960E948292BC018CE09DE00E94FE
:102E7000F390CE0101960E941E90CE0107960E940B
:102E80001E904091ED0C5091EE0C6091EF0C709102
:102E9000F00C21E0CE0107960E94AB916DE975E040
:102EA000CE0101960E948990BE01695F7F4FCE01DD
:102EB00001960E948292BC018CE09DE00E945A9291
:102EC000CE0101960E941E90CE0107960E941E9090
:102ED0006EE676E08CE09DE00E94609264E97BE023
:102EE000CE0101960E94899044E150E060E070E0DC
:102EF000CE0101960E94EE09CE0101960E941E901D
:102F00006091F10C7091F20C8091F30C9091F40CA3
:102F10000E9499954AE0CE0101960E945491BE010B
:102F20006F5F7F4F86E09DE00E941091CE01019679
:102F30000E941E9040E066E08CE19EE00E944766A1
:102F400066E07DE08CE19EE00E94C68C6FED8CE136
:102F50009EE00E94D58C6FE175E08CE19EE00E94BE
:102F6000D48C6091ED0C7091EE0C8091EF0C9091EF
:102F7000F00C0E9499954AE050E08CE19EE00E949E
:102F8000BE8D6EE676E08CE19EE00E94D48C64E615
:102F900070E080E090E00E94F38618C065EA77E078
:102FA000CE0101960E9427924AE050E060E070E076
:102FB000CE0101960E94EE09CE0101960E941E905C
:102FC00065E877E08CE09DE00E9407922C960FB6B2
:102FD000F894DEBF0FBECDBFDF91CF91FF90EF9091
:102FE000DF90CF900895CF92DF92EF92FF92CF9330
:102FF000DF93CDB7DEB72C970FB6F894DEBF0FBEC8
:10300000CDBF67E777E0CE0101960E9427924CE2A0
:1030100051E06FEF7FEFCE0101960E94620BCE016F
:1030200001960E941E906091C6047091C70486E7C5
:103030009DE00E94A364E12CF12C64E670E080E046
:1030400090E00E94F3866091C6047091C70486E701
:103050009DE00E94A3642FEFE21AF20A23E0E21639
:10306000F1045CF32AE0E216F1041CF4892B29F741
:1030700003C0892B09F057C16091780D7091790DCB
:10308000882777FD8095982F0E94CC956B017C0155
:103090006093F10C7093F20C8093F30C9093F40C0A
:1030A0006091760D7091770D882777FD8095982F28
:1030B0000E94CC956093ED0C7093EE0C8093EF0C16
:1030C0009093F00C21E0B701A601CE0107960E9473
:1030D000AB9164E976E0CE0101960E948990BE0131
:1030E000695F7F4FCE0101960E948292BC018CE005
:1030F0009DE00E94F390CE0101960E941E90CE01A9
:1031000007960E941E904091ED0C5091EE0C60913C
:10311000EF0C7091F00C21E0CE0107960E94AB916C
:103120006DE975E0CE0101960E948990BE01695F4C
:103130007F4FCE0101960E948292BC018CE09DE0FF
:103140000E945A92CE0101960E941E90CE010796CF
:103150000E941E906EE676E08CE09DE00E946092F8
:1031600064E97BE0CE0101960E94899044E150E041
:1031700060E070E0CE0101960E94EE09CE0101965A
:103180000E941E906091F10C7091F20C8091F30CF2
:103190009091F40C0E9499954AE0CE0101960E940C
:1031A0005491BE016F5F7F4F86E09DE00E941091B9
:1031B000CE0101960E941E9040E066E08CE19EE008
:1031C0000E94476666E07DE08CE19EE00E94C68C2E
:1031D0006FED8CE19EE00E94D58C6FE175E08CE193
:1031E0009EE00E94D48C6091ED0C7091EE0C809169
:1031F000EF0C9091F00C0E9499954AE050E08CE120
:103200009EE00E94BE8D6EE676E08CE19EE00E941C
:10321000D48C64E670E080E090E00E94F38688E160
:103220009DE00E940F94C090F10CD090F20CE090C1
:10323000F30CF090F40C20E030E040EF51E4C701D3
:10324000B6010E94A19687FD03C068E677E054C0EE
:1032500020E030E040ED51E4C701B6010E94A196A4
:1032600087FD1FC068E577E0CE0101960E94279296
:103270004AE050E06FEF7FEFCE0101960E94620BB3
:10328000CE0101960E941E908091F804882331F0AF
:103290006CED75E080E090E00E94F38668E477E0F2
:1032A0002BC020E030E040EB51E4C701B6010E94A2
:1032B000A19687FD03C06AE377E01EC06BE277E06A
:1032C000CE0101960E9427924AE050E06FEF7FEF17
:1032D000CE0101960E94620BCE0101960E941E90C3
:1032E0008091F804882331F06CED75E080E090E087
:1032F0000E94F3866DE177E0CE0101960E9427924D
:103300004AE050E06FEF7FEFCE0101960E94620B22
:10331000CE0101960E941E9062E370E080E090E092
:103320000E94F38601C037DC2C960FB6F894DEBFFE
:103330000FBECDBFDF91CF91FF90EF90DF90CF9088
:103340000895CF92DF92EF92FF921F93CF93DF9376
:10335000CDB7DEB7AA970FB6F894DEBF0FBECDBFCC
:10336000182F882351F08091FB0C882331F064E9F9
:103370007BE086EC9FE00E94FF8C8AE79DE00E9444
:103380001F6FBE016F5F7F4F8AE79DE00E94BF6E97
:10339000CE010D967C01112391F18091FB0C8823C5
:1033A00071F166E077E0C7010E942792C7010E9491
:1033B000C209C7010E941E90FE0131966F01F601FD
:1033C00041915191619171916F0126E030E086EC5D
:1033D0009FE00E94F78E60E375E086EC9FE00E941C
:1033E000D48CCE14DF0459F764E97BE0C7010E9456
:1033F0008990C7010E94C209C7010E941E9023E95B
:1034000038E144E85FE369817A818B819C810E9485
:1034100060976D877E878F87988B22E430E645E83A
:103420005FE36D817E818F8198850E946097698BB3
:103430007A8B8B8B9C8B25E83BEE41E95FE36985BA
:103440007A858B859C850E9460976D8B7E8B8F8B98
:10345000988FB7018AE79DE00E949F6E112309F4BF
:103460009EC08091FB0C882309F499C0B7018AE7BC
:103470009DE00E94BF6E6E01F9E1CF0ED11C69EF95
:1034800076E0C6010E942792C6010E94C209C601C9
:103490000E941E90F70141915191619171917F01BC
:1034A00022E030E086EC9FE00E94F78E60E375E05A
:1034B00086EC9FE00E94D48CEC14FD0459F764E97B
:1034C0007BE0C7010E948990C7010E94C209C70121
:1034D0000E941E906E01F5E2CF0ED11C9601AE0146
:1034E000495D5F4FBE01675D7F4F8AE79DE00E94A7
:1034F00002706CEE76E086EC9FE00E94A38C69A5DA
:103500007AA54AE050E086EC9FE00E94BE8D60E321
:1035100075E086EC9FE00E94D48C6FA178A54AE00C
:1035200050E086EC9FE00E94BE8D60E375E086EC83
:103530009FE00E94D48C6DA17EA14AE050E086EC11
:103540009FE00E94BE8D64E97BE086EC9FE00E94D4
:10355000FF8CB7018AE79DE00E94407063EE76E041
:1035600086EC9FE00E94A38CF701419151916191FB
:1035700071917F012AE030E086EC9FE00E94F78E97
:1035800060E375E086EC9FE00E94D48CEC14FD04AF
:1035900059F764E97BE086EC9FE00E94FF8C61E0D4
:1035A00070E08AE79DE00E94336F1123A9F08091BB
:1035B000FB0C882389F06FEC76E086EC9FE00E949C
:1035C000A38C8AE79DE00E948A704AE050E0BC012B
:1035D00086EC9FE00E94C58D24E030E043E050E09F
:1035E00062E070E08AE79DE00E94406F112309F4D9
:1035F00041C08091FB0C8823E9F163EB76E086EC17
:103600009FE00E94A38C9E012B5D3F4FAE01495D60
:103610005F4FBE01675D7F4F8AE79DE00E949C700F
:1036200069A57AA54AE050E086EC9FE00E94BE8D35
:1036300060E375E086EC9FE00E94D48C6FA178A5D2
:103640004AE050E086EC9FE00E94BE8D60E375E0AA
:1036500086EC9FE00E94D48C6DA17EA14AE050E0F0
:1036600086EC9FE00E94BE8D64E97BE086EC9FE0E3
:103670000E94FF8C65E070E08AE79DE00E945D6F2C
:103680001123A9F08091FB0C882389F060EA76E091
:1036900086EC9FE00E94A38C8AE79DE00E94DF7089
:1036A0004AE050E0BC0186EC9FE00E94C58D66E0D8
:1036B00070E08AE79DE00E946A6F1123A9F0809173
:1036C000FB0C882389F068E876E086EC9FE00E9496
:1036D000A38C8AE79DE00E94F1704AE050E0BC01B3
:1036E00086EC9FE00E94C58D67E070E08AE79DE070
:1036F0000E946D6F1123A9F08091FB0C882389F043
:1037000062E776E086EC9FE00E94A38C8AE79DE06A
:103710000E9403714AE050E0BC0186EC9FE00E94E9
:10372000C58D68E070E08AE79DE00E947A6F112302
:10373000A9F08091FB0C882389F06AE576E086EC9D
:103740009FE00E94A38C8AE79DE00E9415714AE0E9
:1037500050E0BC0186EC9FE00E94C58D69E070E0FE
:103760008AE79DE00E94876F1123A9F08091FB0CEE
:10377000882389F060E476E086EC9FE00E94A38CC9
:103780008AE79DE00E9427714AE050E0BC0186EC88
:103790009FE00E94C58D6AE070E08AE79DE00E948C
:1037A000946F1123A9F08091FB0C882389F06AE2C1
:1037B00076E086EC9FE00E94A38C8AE79DE00E9461
:1037C00039714AE050E0BC0186EC9FE00E94C58D53
:1037D0006BE070E08AE79DE00E94A16F1123A9F0E1
:1037E0008091FB0C882389F061E176E086EC9FE014
:1037F0000E94A38C8AE79DE00E944B714AE050E052
:10380000BC0186EC9FE00E94C58D6CE070E08AE709
:103810009DE00E94AE6F112309F494C08091FB0CCF
:10382000882309F48FC069EF75E086EC9FE00E9461
:10383000A38C8AE79DE00E945D714AE050E0BC01E4
:1038400086EC9FE00E94C58D62EE75E086EC9FE0FD
:103850000E94A38C8AE79DE00E948272682F70E02C
:103860004AE050E086EC9FE00E94C58D6BEC75E06D
:1038700086EC9FE00E94A38C8AE79DE00E948672FE
:10388000682F70E04AE050E086EC9FE00E94C58D12
:1038900064EB75E086EC9FE00E94A38C8AE79DE0D4
:1038A0000E948A72682F70E04AE050E086EC9FE048
:1038B0000E94C58D6BE975E086EC9FE00E94A38CA9
:1038C0008AE79DE00E948E72682F70E04AE050E027
:1038D00086EC9FE00E94C58D62E875E086EC9FE073
:1038E0000E94A38C8AE79DE00E949272682F70E08C
:1038F0004AE050E086EC9FE00E94C58D69E675E0E5
:1039000086EC9FE00E94A38C8AE79DE00E9496725D
:10391000682F70E04AE050E086EC9FE00E94C58D81
:1039200068E575E086EC9FE00E94A38C8AE79DE045
:103930000E949A72682F70E04AE050E086EC9FE0A7
:103940000E94C58D61E08AE79DE00E94377261E0C8
:103950008AE79DE00E943C7261E08AE79DE00E9458
:1039600041721123B1F08091FB0C882391F06FE339
:1039700075E086EC9FE00E94A38C8AE79DE00E94A0
:103980009E72682F70E04AE050E086EC9FE00E9453
:10399000C58D60E08AE79DE00E9441721123B1F07D
:1039A0008091FB0C882391F065E275E086EC9FE046
:1039B0000E94A38C8AE79DE00E949E72682F70E0AF
:1039C0004AE050E086EC9FE00E94C58D61E08AE706
:1039D0009DE00E9446721123B1F08091FB0C882378
:1039E00091F069E075E086EC9FE00E94A38C8AE785
:1039F0009DE00E94A272682F70E04AE050E086ECE1
:103A00009FE00E94C58D60E08AE79DE00E944672BB
:103A10001123B1F08091FB0C882391F06CEE74E0DF
:103A200086EC9FE00E94A38C8AE79DE00E94A27230
:103A3000682F70E04AE050E086EC9FE00E94C58D60
:103A400061E08AE79DE00E944B721123B1F0809102
:103A5000FB0C882391F060ED74E086EC9FE00E94FF
:103A6000A38C8AE79DE00E94A672682F70E04AE06E
:103A700050E086EC9FE00E94C58D60E08AE79DE003
:103A80000E944B721123B1F08091FB0C882391F0BE
:103A900063EB74E086EC9FE00E94A38C8AE79DE0D4
:103AA0000E94A672682F70E04AE050E086EC9FE02A
:103AB0000E94C58D61E08AE79DE00E94507211234B
:103AC000B1F08091FB0C882391F067E974E086ECFB
:103AD0009FE00E94A38C8AE79DE00E94AA72682F53
:103AE00070E04AE050E086EC9FE00E94C58D60E007
:103AF0008AE79DE00E9450721123B1F08091FB0C87
:103B0000882391F06AE774E086EC9FE00E94A38C22
:103B10008AE79DE00E94AA72682F70E04AE050E0B8
:103B200086EC9FE00E94C58D61E08AE79DE00E94DF
:103B3000197261E08AE79DE00E941E7261E08AE7E7
:103B40009DE00E94237260E08AE79DE00E94287257
:103B500060E08AE79DE00E942D7260E08AE79DE0C8
:103B60000E943272112309F495C08091FB0C8823C6
:103B700009F490C062E674E086EC9FE00E94A38C9A
:103B80008AE79DE00E94AE72682F70E04AE050E044
:103B900086EC9FE00E94C58D64E474E086EC9FE0B3
:103BA0000E94A38C8AE79DE00E94B272682F70E0A9
:103BB0004AE050E086EC9FE00E94C58D66E274E02A
:103BC00086EC9FE00E94A38C8AE79DE00E94B6727B
:103BD000682F70E04AE050E086EC9FE00E94C58DBF
:103BE0006DE074E086EC9FE00E94A38C8AE79DE084
:103BF0000E94BA72682F70E04AE050E086EC9FE0C5
:103C00000E94C58D64EF73E086EC9FE00E94A38C58
:103C10008AE79DE00E94BE72682F70E04AE050E0A3
:103C200086EC9FE00E94C58D6BED73E086EC9FE013
:103C30000E94A38C8AE79DE00E94C272682F70E008
:103C40004AE050E086EC9FE00E94C58D68EC73E08E
:103C500086EC9FE00E94A38C8AE79DE00E94C672DA
:103C6000682F70E04AE050E086EC9FE00E94C58D2E
:103C700063EB73E086EC9FE00E94A38C8AE79DE0F3
:103C80000E94CA72682F70E04AE050E086EC9FE024
:103C90000E94C58D60E08AE79DE00E94557240ED6C
:103CA0005FE069E470E48AE79DE00E949871112367
:103CB00009F44EC08091FB0C882309F449C06FE9D8
:103CC00073E086EC9FE00E94A38C8AE79DE00E944F
:103CD0006F71AB01BC0122E030E086EC9FE00E94F6
:103CE000F88E68E873E086EC9FE00E94A38C8AE778
:103CF0009DE00E94D3714AE050E0682F86EC9FE07F
:103D00000E94F78D60E773E086EC9FE00E94A38C31
:103D100061E08AE79DE00E94CE72682F70E04AE081
:103D200050E086EC9FE00E94C58D67E573E086EC6D
:103D30009FE00E94A38C61E08AE79DE00E94D2721E
:103D4000682F70E04AE050E086EC9FE00E94C58D4D
:103D500041E061E08AE79DE00E945A721123B9F0C8
:103D60008091FB0C882399F06FE373E086EC9FE071
:103D70000E94A38C61E08AE79DE00E94D672682FC2
:103D800070E04AE050E086EC9FE00E94C58D41E083
:103D900061E08AE79DE00E945F7260E08AE79DE053
:103DA0000E9414721123D1F08091FB0C8823B1F092
:103DB0006CE273E086EC9FE00E94A38C8AE79DE0B2
:103DC0000E947E72682F70E04AE050E086EC9FE02F
:103DD0000E94C58D8AE79DE00E94DA72AA960FB60E
:103DE000F894DEBF0FBECDBFDF91CF911F91FF9042
:103DF000EF90DF90CF9008952F923F924F925F9275
:103E00006F927F928F929F92AF92BF92CF92DF92EA
:103E1000EF92FF920F931F93CF93DF93CDB7DEB74F
:103E2000C554D1090FB6F894DEBF0FBECDBF2B012C
:103E30003C012DA33EA34FA358A70E94C4862296FF
:103E40006CAF7DAF8EAF9FAF229720E9421621E085
:103E500052066104710434F020E9422E5524539433
:103E6000612C712C8DA19EA1AFA1B8A58031974284
:103E7000A105B1052CF030E127E290E080E004C01C
:103E80003DA12EA19FA188A54091FD0C411104C028
:103E90003DA32EA39FA388A722966CAD7DAD8EADCA
:103EA0009FAD229728EE33E040E050E00E94C59895
:103EB00026962CAF3DAF4EAF5FAF2697F1E0FDAB3E
:103EC00019A61AA61BA61CA68E01035F1F4F222748
:103ED0003327A901241935094609570929AB3AABFB
:103EE0004BAB5CAB29A53AA54BA55CA58DA19EA1CA
:103EF000AFA1B8A5281739074A075B070CF035C3EF
:103F000069A57AA58BA59CA50E94CC9520E030E000
:103F10004AE754E40E940095AB01BC0123E0C801CC
:103F20000E94AB91B80186E09DE00E941091C8010B
:103F30000E941E908DA19EA1AFA1B8A50A97A105D0
:103F4000B10594F42AE026964CAD5DAD6EAD7FAD23
:103F50002697C8010E947F91B80186E09DE00E94EB
:103F60001091C8010E941E90BE016F5F7F4F8AE7CB
:103F70009DE00E94407063EA75E08CE09DE00E9445
:103F80002691DE0111961D01C12CD12C7601F10183
:103F900081909190A190B1901F01A5019401C5015C
:103FA000B4010E9460979B01AC01C701B6010E9459
:103FB00036946B017C0123E0B501A401CE01439648
:103FC0000E94D991BE016D5E7F4FC8010E94089189
:103FD00060E375E0C8010E949392BC018CE09DE013
:103FE0000E945A92C8010E941E90CE0143960E94E0
:103FF0001E902016310659F6C701B6010E9413988B
:104000006B017C01FDE24F16F1E05F066104710473
:1040100044F00E94290C40E060E08CE19EE00E94A8
:10402000476623E0B701A601C8010E94AB9162E692
:1040300075E0CE0143960E94899066E07DE0CE0156
:1040400043960E94829260EB75E00E949392B801C1
:104050000E94829265EB75E00E949392BC018CE015
:104060009DE00E945A92CE0143960E941E90C80184
:104070000E941E902DEC3CEC4CE45FE3C701B601BE
:104080000E94A19629813A814B815C812DA73EA790
:104090004FA758AB18160CF0ACC12AE939E949E929
:1040A0005FE3C701B6010E94FC9487FFA2C13DA94E
:1040B000332309F49EC189849A84AB84BC8420E0B4
:1040C00030E0A901C501B4010E94FC94CD80DE80DE
:1040D000EF80F884882309F12DA53EA54FA558A9A6
:1040E000CA01B9010E9460976EAB7FAB88AF99AFF0
:1040F000A7019601C701B6010E9460979B01AC0120
:104100006EA97FA988AD99AD0E9436940E9413983C
:10411000A50194010E94A99404C06BED7FE089EC95
:104120009FE320EE3EE245E652E40E9460976EABCC
:104130007FAB88AF99AF20E030E0A901C701B6019D
:104140000E94FC94882309F12DA53EA54FA558A9EE
:10415000CA01B9010E9460976AAF7BAF8CAF9DAF77
:10416000A5019401C501B4010E9460979B01AC01B7
:104170006AAD7BAD8CAD9DAD0E9436940E941398C4
:10418000A70196010E94A99404C06BED7FE089EC21
:104190009FE320EE3EE245E652E40E9460976AAF5C
:1041A0007BAF8CAF9DAF20E030E0A9016DA57EA56F
:1041B0008FA598A90E94FC948823F9F0A501940189
:1041C000C501B4010E9460974B015C01A7019601F3
:1041D000C701B6010E9460979B01AC01C501B40103
:1041E0000E9436940E9413982DA53EA54FA558A96C
:1041F0000E94A9946B017C0108C09BEDC92E9FE031
:10420000D92E99ECE92E9FE3F92E63E675E0C801FB
:104210000E94899066E07DE0C8010E94829268EB6E
:1042200075E00E949392BC018CE09DE00E94F390A7
:10423000C8010E941E9063E675E0C8010E94899043
:1042400066E07DE0C8010E94829262ED75E00E9406
:104250009392BC0186E09DE00E94F390C8010E9409
:104260001E9021E04EA95FA968AD79ADC8010E94FA
:10427000AB9121E04AAD5BAD6CAD7DADCE01439617
:104280000E94AB9120EE3EE245E652E4C701B60142
:104290000E946097AB01BC0121E0CE014F960E94C5
:1042A000AB91BE01615E7F4FCE0149960E9408919D
:1042B00060E375E0CE0149960E949392BE016D5E67
:1042C0007F4F0E94829260E375E00E949392B80152
:1042D0000E948292BC0180E09DE00E94F390CE019A
:1042E00049960E941E90CE014F960E941E90CE01CC
:1042F00043960E941E90C8010E941E904DE24416F3
:1043000041E054066104710474F469A57AA58BA593
:104310009CA525E030E040E050E00E94C598672B66
:10432000682B692BC1F566E07DE0C8010E94089109
:1043300045E050E06FEF7FEFC8010E94970AC80187
:104340000E941E906BED75E0C8010E94899045E0C7
:1043500050E061EF7FEFC8010E94EE09C8010E94A2
:104360001E9064E97BE0C8010E948990C8010E9408
:104370000B0CC8010E941E9060E07DE0C8010E9405
:10438000089145E050E060E070E0C8010E94620BD7
:10439000C8010E941E9060E07DE08CE09DE00E94DC
:1043A0005A925FE1451651046104710434F489A501
:1043B0009AA5ABA5BCA5B7FD11C06CE07DE0C80116
:1043C0000E940891C8010E94DC0FC8010E941E9043
:1043D00064E97BE08CE09DE00E942691B201C3017C
:1043E00077FE04C069A97AA98BA99CA90E94F386CB
:1043F000A9C023E04DA55EA56FA578A9C8010E94BC
:10440000AB9163E675E0CE0143960E94899066E029
:104410007DE0CE0143960E9482926DED75E00E9490
:104420009392B8010E94829266EB75E00E9493928B
:10443000BC0186E09DE00E94F390CE0143960E946D
:104440001E90C8010E941E9049855A856B857C8507
:1044500023E0C8010E94D9914D815E816F817885EA
:1044600023E0CE0149960E94D991BE01675E7F4F3D
:10447000CE0143960E94089162EE75E0CE0143960C
:104480000E949392B8010E94829266EB75E00E94AE
:104490009392BC0180E09DE00E94F390CE01439690
:1044A0000E941E90CE0149960E941E90C8010E9453
:1044B0001E909DE2491691E059066104710474F45E
:1044C00069A57AA58BA59CA525E030E040E050E0E9
:1044D0000E94C598672B682B692BF1F466E07DE09C
:1044E000C8010E9408914AE050E06FEF7FEFC801D9
:1044F0000E94970AC8010E941E9060E07DE0C801FA
:104500000E9408914AE050E060E070E0C8010E941B
:10451000620BC8010E941E906CE07DE0C8010E9401
:104520000891C8010E94DC0FC8010E941E9064E936
:104530007BE08CE09DE00E942691C301B2010E94C5
:10454000F3861DAA0E94C4869B01AC0122968CAD05
:104550009DADAEADBFAD2297281B390B4A0B5B0B4F
:1045600029A73AA74BA75CA7BDCC66E07DE0CE01AA
:104570000D960E9408914AE050E06FEF7FEFCE0168
:104580000D960E94EE09CE010D960E941E909DA9E7
:104590009923B1F16BED75E0CE010D960E948990E3
:1045A00045E050E061EF7FEFCE010D960E94EE09ED
:1045B000CE010D960E941E908091FD0C882391F0F3
:1045C00064E273E0CE010D960E94279245E050E030
:1045D00060E070E0CE010D960E94EE09CE010D96CE
:1045E0000E941E9064E97BE0CE010D960E948990A6
:1045F000CE010D960E940B0CCE010D960E941E90CE
:1046000060E07DE0CE010D960E9408914AE050E006
:104610006FEF7FEFCE010D960E94620BCE010D96DB
:104620000E941E90CB5BDF4F0FB6F894DEBF0FBE2B
:10463000CDBFDF91CF911F910F91FF90EF90DF9051
:10464000CF90BF90AF909F908F907F906F905F9032
:104650004F903F902F900895CF92DF92EF92FF926C
:104660000F931F93CF93DF93CDB7DEB72C970FB681
:10467000F894DEBF0FBECDBF8091FD0C811102C04A
:104680000E94290C83E690E10E94338A64E670E080
:1046900080E090E00E94F38668E073E086E09DE0B1
:1046A0000E94079266E07DE0CE0101960E9408918B
:1046B00044E150E060E070E0CE0101960E94EE0916
:1046C000CE0101960E941E9069EF72E086E09DE0A7
:1046D0000E94079266E07DE0CE0101960E9408915B
:1046E00044E150E06FEF7FEFCE0101960E94620B34
:1046F000CE0101960E941E9060E070E08DEF9DE07B
:104700000E9444746B017C0104E010E0A701960153
:10471000C701B6010E945498882309F43DC0015096
:10472000110909F011C16EEE72E086E09DE00E9471
:10473000079266E07DE0CE0101960E9408914AE072
:1047400050E060E070E0CE0101960E94EE09CE01DB
:1047500001960E941E9065EE75E0CE0101960E94C2
:10476000899066E07DE0CE0101960E948292BC01B4
:104770008CE09DE00E94F390CE0101960E941E9075
:104780008091280E9091290E039709F0CCC01092C9
:10479000290E1092280EC7C021E0B701A601CE0154
:1047A00007960E94AB9167EF75E0CE0101960E94DB
:1047B0008990BE01695F7F4FCE0101960E9482926F
:1047C000BC018CE09DE00E94F390CE0101960E9416
:1047D0001E90CE0107960E941E906CE07DE0CE01F7
:1047E00001960E94089142E350E06FEF7FEFCE0107
:1047F00001960E94620BCE0101960E941E900E94BB
:10480000F70B6AE975E08CE09DE00E94609260E041
:1048100070E08DEF9DE00E9442746B017C0104E02A
:1048200010E0A7019601C701B6010E9454988823A1
:1048300059F00150110909F096C064E97BE082E16A
:104840009DE00E94269150C021E0B701A601CE0153
:1048500007960E94AB9164E976E0CE0101960E9432
:104860008990BE01695F7F4FCE0101960E948292BE
:10487000BC0182E19DE00E94F390CE0101960E946E
:104880001E90CE0107960E941E9060E375E0CE0157
:1048900001960E94899062E17DE0CE0101960E941E
:1048A0008292BC0186E09DE00E94F390CE010196C9
:1048B0000E941E9066E07DE0CE0101960E94089164
:1048C0004AE050E060E070E0CE0101960E94970A55
:1048D000CE0101960E941E900E94F70B6AE975E0D6
:1048E00082E19DE00E94609262E17DE0CE0101964E
:1048F0000E94089160E375E0CE0101960E949392B8
:104900006CE07DE00E948292BC018CE09DE00E9400
:10491000F390CE0101960E941E9083E090E0909368
:10492000290E8093280E64E670E080E090E00E94FB
:10493000F3868091FD0C882329F160E273E080E02A
:1049400090E00E94F3861EC064E670E080E090E094
:104950000E94F38660E070E08DEF9DE00E94447459
:104960006B017C01D3CE68EC70E080E090E00E94A7
:10497000F38660E070E08DEF9DE00E9442746B0171
:104980007C014FCF2C960FB6F894DEBF0FBECDBF83
:10499000DF91CF911F910F91FF90EF90DF90CF901B
:1049A00008951F93CF93DF93182FC1E9DCE0812F87
:1049B0000E948987899399936CE370E080E090E08E
:1049C0000E94F3868CE0C13ED80789F768E270E068
:1049D00081E99CE00E94E80720E030E040EA50E4F2
:1049E0000E94609720E030E040E85AE30E94609720
:1049F000DF91CF911F9108954F925F926F927F92B6
:104A00008F929F92AF92BF92CF92DF92EF92FF92DE
:104A10000F931F93CF93DF93CDB7DEB764970FB695
:104A2000F894DEBF0FBECDBF7C018B0164EE72E057
:104A300086E09DE00E9407920E94290C66E07DE0DE
:104A4000CE0101960E9408914AE050E06FEF7FEF9F
:104A5000CE0101960E94EE09CE0101960E941E90A1
:104A6000C7019FDF698B7A8B8B8B9C8B40901A02DE
:104A700050901B0260901C0270901D02A3019201D5
:104A8000609116027091170280911802909119029C
:104A90000E9435944B015C0120E030E0A9010E94A6
:104AA000FC94882309F451C0C0902202D0902302C4
:104AB000E0902402F090250220E030E0A901C70137
:104AC000B6010E94FC9418160CF03FC080911E02A3
:104AD00090911F02A0912002B09121028D879E87A4
:104AE000AF87B88B9C01AD01C701B6010E94FC9451
:104AF000882359F1A70196016D857E858F85988958
:104B00000E9400950E94ED966D877E878F87988B17
:104B1000A301920169897A898B899C890E943594C5
:104B2000A50194010E9400952D853E854F855889E9
:104B30000E9460970E946D959B01AC01C701B60170
:104B40000E9460976B017C0103C0C12CD12C7601BF
:104B500066E07DE0CE0101960E9408914AE050E0B7
:104B600060E070E0CE0101960E94EE09CE01019650
:104B70000E941E9020E030E64AEE56E4C701B601DE
:104B80000E94A19618163CF460E076E08CE09DE06F
:104B90000E94269144C001151105B9F421E0B70126
:104BA000A601CE0107960E94AB916FE076E0CE01A0
:104BB00001960E948990BE01695F7F4FCE010196E8
:104BC0000E94829263E176E01BC00230110539F544
:104BD00022E049895A896B897C89CE0107960E9417
:104BE000AB916FE076E0CE0101960E948990BE0104
:104BF000695F7F4FCE0101960E94829267E176E065
:104C00000E949392BC018CE09DE00E94F390CE0143
:104C100001960E941E90CE0107960E941E906CE0A5
:104C20007DE0CE0101960E9408914AE050E06FEFCE
:104C30007FEFCE0101960E94620BCE0101960E9489
:104C40001E9064E670E080E090E00E94F386809120
:104C5000FD0C882331F060E273E080E090E00E9478
:104C6000F38664960FB6F894DEBF0FBECDBFDF911A
:104C7000CF911F910F91FF90EF90DF90CF90BF9059
:104C8000AF909F908F907F906F905F904F9008951E
:104C90004F925F926F927F928F929F92AF92BF924C
:104CA000CF92DF92EF92FF92CF93C82F8091BA0BF1
:104CB00081110DC00E94C4866093AE0B7093AF0B40
:104CC0008093B00B9093B10B81E08093BA0B8091ED
:104CD000B20B81110DC00E94C4866093AA0B709321
:104CE000AB0B8093AC0B9093AD0B81E08093B20B38
:104CF0001092900C10928F0CE0908F0CF090900C12
:104D000088E2E816F1040CF08AC08C2F0E94898793
:104D1000F701EE0FFF1FEF56F34F9183808368E298
:104D200070E081E99CE00E94E80720E030E040EA82
:104D300050E40E94609720E030E040E85AE30E948F
:104D400060976B017C016093A60B7093A70B809317
:104D5000A80B9093A90B40902A0250902B026090D0
:104D60002C0270902D02A301920160912602709195
:104D7000270280912802909129020E9435949B017C
:104D8000AC0160E070E080EC90E40E9435944B014F
:104D90005C0120E030E0A9010E94FC9420E030E0BA
:104DA00040E650E4811105C0C701B6010E9460973A
:104DB0001EC0C701B6010E946097A30192010E9424
:104DC000369420E030E040E850E40E943594A5019C
:104DD00094010E94009520E030E040EC50E40E94F5
:104DE000609720E030E040E850E40E943694609301
:104DF000A20B7093A30B8093A40B9093A50B64E17B
:104E000070E080E090E00E94F38680918F0C90919A
:104E1000900C01969093900C80938F0C6DCF6091C5
:104E2000A20B7091A30B8091A40B9091A50BCF9135
:104E3000FF90EF90DF90CF90BF90AF909F908F90BA
:104E40007F906F905F904F900895CF92DF92EF9296
:104E5000FF92CF93DF93CDB7DEB72C970FB6F894C0
:104E6000DEBF0FBECDBF6BED72E086E09DE00E941D
:104E7000079266E07DE0CE0101960E9408914AE02B
:104E800050E060E070E0CE0101960E94EE09CE0194
:104E900001960E941E908091810290918202F8DE1C
:104EA0006B017C0120E030E0A9010E94A19687FD02
:104EB00022C022E0B701A601CE0107960E94AB9165
:104EC00069E176E0CE0101960E948990BE01695F9A
:104ED0007F4FCE0101960E948292BC018CE09DE042
:104EE0000E94F390CE0101960E941E90CE0107967B
:104EF0000E941E9006C06DE176E08CE09DE00E946D
:104F000026916CE07DE0CE0101960E9408914AE076
:104F100050E06FEF7FEFCE0101960E94620BCE0151
:104F200001960E941E902C960FB6F894DEBF0FBE1D
:104F3000CDBFDF91CF91FF90EF90DF90CF9008959C
:104F40002F923F924F925F926F927F928F929F9299
:104F5000AF92BF92CF92DF92EF92FF920F931F9387
:104F6000CF93DF9300D01F92CDB7DEB76B017C01EA
:104F70005A8349835901FA01208131814281538149
:104F80000E94FC94181614F0F50183C010E0015043
:104F9000104C000F111F000F111FE981FA81E00F63
:104FA000F11F2081318142815381C701B6010E94E6
:104FB000A19687FF6BC011E0612E712C4301880C14
:104FC000991C880C991CE981FA81E80DF91D208053
:104FD000318042805380A2019101C701B6010E9435
:104FE000A196181614F41F5FE7CFA2019101C70123
:104FF000B6010E94FC948501080D191D811102C0A3
:10500000F80147C0C3018150904C880F991F880F49
:10501000991FA981BA81A80FB91F2D913D914D917A
:105020005C9129833A834B835C83F501E80FF91F78
:1050300080809180A280B380C701B6010E94359420
:105040006B017C01A5019401F8016081718182816D
:1050500093810E9435949B01AC01C701B6010E9467
:1050600060976B017C0129813A814B815C81C2018F
:10507000B1010E9435949B01AC01C701B6010E94A9
:105080000095A50194010E94369407C0F501E00F38
:10509000F11F60817181828193810F900F900F9039
:1050A0000F90DF91CF911F910F91FF90EF90DF90C4
:1050B000CF90BF90AF909F908F907F906F905F90B8
:1050C0004F903F902F900895CF92DF92EF92FF92F2
:1050D0001F93CF93DF93182FCAE0D0E0C12CD12CBF
:1050E0007601812F0E948987BC01882777FD8095F2
:1050F000982F0E94CC959B01AC01C701B6010E947C
:1051000036946B017C0162E370E080E090E00E94E5
:10511000F386219731F720E030E040E251E4C70107
:10512000B6010E94009520E030E040EA50E40E9481
:10513000609720E030E040E85AE30E946097DF91FA
:10514000CF911F91FF90EF90DF90CF900895FC01D9
:1051500020E030E0772767FD7095AB0142505109A0
:10516000DF01A81BB90BA417B50724F4A1912A0FDE
:10517000311DF6CFA9014E5B5F4F860F971FFC01D3
:105180003297208130E0322F222731968081280FFC
:10519000311D81E04217530709F080E00895FF9226
:1051A0000F931F93CF93DF93F82E0AE010E0C0E037
:1051B000D0E08F2D0E948987C80FD91F65E070E06D
:1051C00080E090E00E94F3860150110991F7CE0132
:1051D0006AE070E00E947C98CB01DF91CF911F9133
:1051E0000F91FF9008950F931F93CF93DF93CDB747
:1051F000DEB72E970FB6F894DEBF0FBECDBF8D87FA
:105200009E870E94290C8D859E85C9DF8C0162E3F3
:1052100070E080E090E00E94F386B801882777FD77
:105220008095982F0E94CC9520E030E040EA50E431
:105230000E94609720E030EC4FE754E40E94009514
:10524000AB01BC0123E0CE0107960E94AB9167E75A
:1052500077E0CE0101960E948990BE01695F7F4F81
:10526000CE0101960E94829260E476E00E949392C1
:10527000BC018CE09DE00E94F390CE0101960E945B
:105280001E90CE0107960E941E9063E476E086E0B1
:105290009DE00E94269166E07DE0CE0101960E948D
:1052A00008914AE050E068E070E0CE0101960E946B
:1052B000EE09CE0101960E941E906CE07DE0CE01C9
:1052C00001960E9408914AE050E06FEF7FEFCE0117
:1052D00001960E94620BCE0101960E941E9066E02C
:1052E0007DE08CE09DE00E945A928091FD0C882325
:1052F00031F060E273E080E090E00E94F3862E9649
:105300000FB6F894DEBF0FBECDBFDF91CF911F91D6
:105310000F910895CF93DF93CDB7DEB72C970FB6DB
:10532000F894DEBF0FBECDBF3ADF9093F60C8093AA
:10533000F50C62E370E080E090E00E94F3866091FB
:10534000F50C7091F60C4AE0CE0101960E94549142
:10535000BE016F5F7F4F8CE09DE00E941091CE01F7
:1053600001960E941E908091740D9091750D892B6D
:1053700009F45FC060E77DE0CE0107960E940891C6
:10538000BE01695F7F4FCE0101960E94089144E102
:1053900050E060E070E0CE0101960E94EE09CE017F
:1053A00001960E941E906BE476E0CE0101960E9469
:1053B00089906CE07DE0CE0101960E948292BC0152
:1053C00086E09DE00E94F390CE0101960E941E901F
:1053D00066E07DE0CE0101960E94089144E150E034
:1053E0006FEF7FEFCE0101960E94620BCE01019616
:1053F0000E941E90BE01695F7F4FCE0101960E9400
:10540000089160E375E0CE0101960E94939266E0F8
:105410007DE00E948292BC018CE09DE00E94F390AE
:10542000CE0101960E941E90CE0107960E941E900A
:1054300054C066E576E086E09DE00E94269166E035
:105440007DE0CE0101960E94089144E150E060E0C9
:1054500070E0CE0101960E94EE09CE0101960E94F5
:105460001E906AE576E0CE0101960E9489906CE07C
:105470007DE0CE0101960E948292BC0186E09DE013
:105480000E94F390CE0101960E941E9066E07DE09E
:10549000CE0101960E94089144E150E06FEF7FEF4A
:1054A000CE0101960E94620BCE0101960E941E90D1
:1054B0006BE476E0CE0101960E9489906CE07DE07D
:1054C000CE0101960E948292BC018CE09DE00E9478
:1054D000F390CE0101960E941E908091FD0C8823CE
:1054E00031F060E273E080E090E00E94F3862C9659
:1054F0000FB6F894DEBF0FBECDBFDF91CF910895F8
:105500000F931F93CF93DF93CDB7DEB72C970FB6D2
:10551000F894DEBF0FBECDBF8C0181E00E9486876C
:1055200064E670E080E090E00E94F3860E94290C1F
:10553000C80135DE60E074E0681B790B4AE0CE01FB
:1055400007960E9454916AE576E0CE0101960E948A
:105550008990BE01695F7F4FCE0101960E948292C1
:10556000BC018CE09DE00E94F390CE0101960E9468
:105570001E90CE0107960E941E9040E066E08CE1EE
:105580009EE00E94476664E177E0CE0101960E94AA
:10559000279242E350E068E070E0CE0101960E945D
:1055A000EE09CE0101960E941E906CE07DE0CE01D6
:1055B00001960E94089142E350E06FEF7FEFCE0129
:1055C00001960E94620BCE0101960E941E9061E638
:1055D00076E0CE0101960E9489906CE07DE0CE01DC
:1055E00001960E948292BC018CE09DE00E94F390A3
:1055F000CE0101960E941E908091FD0C882331F00F
:1056000060E273E080E090E00E94F3862C960FB693
:10561000F894DEBF0FBECDBFDF91CF911F910F91E8
:1056200008950F9390E0BBDDBC01882777FD80953E
:10563000982F0E94CC952DE038E643E55BE30E946D
:10564000609706E021E532E049E652E079DC20E0AF
:1056500030E048EC52E40E94609720E030E048EAF5
:1056600051E40E94609720914D0230914E0240918A
:105670004F02509150020E9400950F910895CF92D1
:10568000DF92EF92FF92CF93DF93CDB7DEB72C97E7
:105690000FB6F894DEBF0FBECDBFC3DF6B017C0138
:1056A0006DE972E086E09DE00E94079266E07DE091
:1056B000CE0101960E94089142E350E060E070E064
:1056C000CE0101960E94EE09CE0101960E941E9025
:1056D00022E0B701A601CE0107960E94AB916DE2D0
:1056E00076E0CE0101960E948990BE01695F7F4FEE
:1056F000CE0101960E9482926BE676E00E94939220
:10570000BC018CE09DE00E94F390CE0101960E94C6
:105710001E90CE0107960E941E906CE07DE0CE01A7
:1057200001960E94089142E350E06FEF7FEFCE01B7
:1057300001960E94620BCE0101960E941E908091FC
:10574000FD0C882331F060E273E080E090E00E947D
:10575000F3862C960FB6F894DEBF0FBECDBFDF9157
:10576000CF91FF90EF90DF90CF900895CF92DF928E
:10577000EF92FF920F9390E012DDBC01882777FD36
:105780008095982F0E94CC952DE038E643E55BE3A9
:105790000E94609706E021E532E049E652E0D0DB66
:1057A00020E030E048EC52E40E9460976B017C01FD
:1057B00020E030E0A9010E94FC94181634F0C12CBE
:1057C000D12C48EAE42E41E4F42EC0924D02D0924E
:1057D0004E02E0924F02F09250020F91FF90EF9034
:1057E000DF90CF9008952F923F924F925F927F92D9
:1057F0008F929F92AF92BF92CF92DF92EF92FF92E1
:105800000F931F93CF93DF9300D01F92CDB7DEB7D6
:105810006C0188EA94E09C838B83E6E9F4E0FA83E8
:10582000E9830FE11CE0EE24E394F12C6DE3262ED6
:10583000312C7EE3472E512CE0E1AE2EB12CF1E16C
:105840008F2E912CA7E17A2E80919404909195044B
:105850008E159F050CF4ECC0F1E0CF16D10431F4A5
:10586000F80180819181E981FA8109C0F2E0CF16C7
:10587000D10439F4E981FA8180819181F801918321
:105880008083E981FA8180819181009749F4EB81DD
:10589000FC81808191819093B9048093B80428C0E1
:1058A0008130910549F4EB81FC8180819181909355
:1058B000C7048093C6041CC08230910549F4EB8173
:1058C000FC81808191819093C5048093C40410C0B1
:1058D000039771F4EB81FC81808191819093BB04EB
:1058E0008093BA0464E97BE080E79DE00E94269102
:1058F000E981FA8181919191FA83E983843091055C
:1059000049F4EB81FC812081318130938202209324
:10591000810230C08530910549F4EB81FC81208102
:1059200031813093C3042093C20424C08630910592
:1059300049F4EB81FC81208131813093BF042093B5
:10594000BE0424C08730910549F4EB81FC8120819D
:1059500031813093BD042093BC0446C08A30910548
:1059600049F4EB81FC81208131813093C104209383
:10597000C0043AC08531910549F4EB81FC81208156
:1059800031813093C9042093C8042EC0863191051B
:1059900049F4EB81FC81208131813093E304209331
:1059A000E20422C087319105F9F4EB81FC8120816A
:1059B0003181A901475051094230510540F4B0925C
:1059C000E704A092E6049092E5048092E404255056
:1059D00031092230310540F43092E7042092E60488
:1059E0005092E5044092E4049C012B5031092A3086
:1059F000310598F4EB81FC81208131813093BB0427
:105A00002093BA04789EB001799E700D11246D57D1
:105A10007D4F80E79DE00E942691FFEFEF1AFF0A7D
:105A20008B819C8102969C838B830E5F1F4F0CCFD2
:105A30000F900F900F900F90DF91CF911F910F91CA
:105A4000FF90EF90DF90CF90BF90AF909F908F909E
:105A50007F905F904F903F902F90089581E08093CA
:105A6000F4048091F504882321F08CE19EE00C94ED
:105A7000F66508958CE19EE00E94F2651092F404B0
:105A800008958091F50481110AC081E08093F504A6
:105A90008093F4048CE19EE00E9479660CC08091B2
:105AA000F404882341F0E6DF8CE19EE00E947366F7
:105AB0001092F5040895D2CF4F925F926F927F9229
:105AC000AF92BF92CF92DF92EF92FF920F931F930C
:105AD000CF93DF93CDB7DEB7EA970FB6F894DEBF6A
:105AE0000FBECDBF182F64E97BE0CE01C5960E94A2
:105AF0008990612FCE0145960E944168BE016B5E80
:105B00007F4FCE0101960E946474CE0101960E94DF
:105B1000C375CE0101960E9457776CE0CE010196C5
:105B20000E94B376CE0101960E946D74082F10E09A
:105B30000330110509F46FC160E776E0CE01C59628
:105B40000E94269164E97BE08CE09DE00E94269112
:105B5000BE016B5C7F4FCE0183960E9408914AE0A4
:105B600050E060E070E0CE0183960E94EE09CE0125
:105B700083960E941E9041E060E08CE19EE00E94CE
:105B8000476664E976E0CE01C5960E942691B5E6A7
:105B9000AB2EBCE0BB2ECC24C394D12CE12CF12C39
:105BA000E016F1060CF0EDC06E2DCE0101960E94BC
:105BB000E477F50121913191419151915F010E946A
:105BC00036942B013C0120E030E04CEF52EC0E9477
:105BD000FC9487FF25C04AE0B601CE0189960E9459
:105BE00054916AED77E0CE0183960E948990BE01C0
:105BF000675D7F4FCE0183960E9482926AE776E0CE
:105C00000E949392BC018CE09DE00E945A92CE01CA
:105C100083960E941E90CE0189960E941E9049C0D4
:105C200022E0B301A201CE0183960E94AB914AE02B
:105C3000B601CE018F960E9454916AED77E0CE01B5
:105C400089960E948990BE01615D7F4FCE01899641
:105C50000E94829267E878E00E949392BE016D5D97
:105C60007F4F0E948292BC0180E09DE00E94F390F1
:105C7000CE0189960E941E90CE018F960E941E90A2
:105C8000CE0183960E941E9060E07DE0CE01839657
:105C90000E94089160E375E0CE0183960E94939282
:105CA000BC018CE09DE00E945A92CE0183960E9436
:105CB0001E900130110559F4E114F10409F05AC0A5
:105CC0006CE07DE0CE01C5960E94F39053C0023097
:105CD000110511F522E0B301A201CE0189960E94BF
:105CE000AB91BE01675D7F4FCE0183960E94089104
:105CF00060E375E0CE0183960E949392BC01CE01D1
:105D0000C5960E945A92CE0183960E941E90CE01A3
:105D100089960E941E902EC060E07DE0CE018396A1
:105D20000E94089144E150E06FEF7FEFCE0183962F
:105D30000E94620BCE0183960E941E906BE975E073
:105D4000CE0183960E948990CE0183960E940B0C0F
:105D5000CE0183960E941E908091F504882351F015
:105D60008091F404882331F060ED77E080E090E0EA
:105D70000E94F386FFEFEF1AFF0A8FEFC81AD80AC6
:105D80000FCFCE01C5960E94B3938CE09DE00E9498
:105D9000B39301151105C9F465E572E08CE09DE04F
:105DA0000E94079266E876E0CE0183960E94899071
:105DB0004AE050E06FEF7FEFCE0183960E94620BC6
:105DC000CE0183960E941E90E2C0043011050CF0B3
:105DD000F7C0BE016B5C7F4FCE0183960E94089195
:105DE0004AE050E06FEF7FEFCE0183960E94620B96
:105DF000CE0183960E941E906BE975E0CE018396DA
:105E00000E948990CE0183960E940B0CCE0183964E
:105E10000E941E90D5C061E976E0CE01C5960E9431
:105E20002691BE016B5C7F4FCE0183960E94089144
:105E30004AE050E060E070E0CE0183960E94EE09F7
:105E4000CE0183960E941E9064E97BE08CE09DE089
:105E50000E9426916CE07DE0CE01C5960E94F390F1
:105E600000E010E0602FCE0101960E94E4776B0104
:105E70007C0122E0AB01BC01CE010115110569F4E2
:105E800083960E94AB91BE016D5D7F4F8CE19EE0D9
:105E90000E94C68CCE0183961BC089960E94AB914E
:105EA000BE01675D7F4FCE0183960E94089160E33B
:105EB00075E0CE0183960E949392BC01CE01C596F7
:105EC0000E945A92CE0183960E941E90CE0189961E
:105ED0000E941E9022E0B701A601CE0189960E9481
:105EE000AB91BE01675D7F4FCE0183960E94089102
:105EF00060E375E0CE0183960E949392BC018CE032
:105F00009DE00E945A92CE0183960E941E90CE017F
:105F100089960E941E900F5F1F4F0330110509F0F4
:105F2000A1CFCE01C5960E94B393BE016B5C7F4F9B
:105F3000CE0183960E9408914AE050E06FEF7FEF18
:105F4000CE0183960E94620BCE0183960E941E9022
:105F50000E94F70B8CE09DE00E94B39367E976E026
:105F6000CE0183960E9489906CE07DE0CE018396FD
:105F70000E94829261EA76E00E949392BC018CE0DA
:105F80009DE00E94F390CE0183960E941E90CE0168
:105F9000C5960E941E90EA960FB6F894DEBF0FBE1B
:105FA000CDBFDF91CF911F910F91FF90EF90DF90C8
:105FB000CF90BF90AF907F906F905F904F9008957B
:105FC00061EA76E08CE09DE00E946092E0CF8F92E3
:105FD0009F92AF92BF92CF92DF92EF92FF920F9378
:105FE0001F93CF93DF93CDB7DEB7A2970FB6F89488
:105FF000DEBF0FBECDBF5C016A017B01122F809115
:10600000FB0C8823D9F060E472E086EC9FE00E94EC
:10601000A38C4AE050E0B50186EC9FE00E94BE8D63
:1060200060E375E086EC9FE00E94D48C22E030E0D3
:10603000B701A60186EC9FE00E94F88E612FCE0189
:1060400045960E944168BE016B5E7F4FCE0101966E
:106050000E946474CE0101960E94C375CE01019620
:106060000E9457776CE0CE0101960E94B376CE0174
:1060700001960E946D74082F10E00B30110514F08A
:106080000AE010E08BE5A816B10408F44FC045E61D
:10609000842E4CE0942EC12CD12C7601A12CB12C55
:1060A000A016B106BCF46A2DCE0101960E94E477D9
:1060B0009B01AC01F40161937193819391934F0122
:1060C000C701B6010E9436946B017C01FFEFAF1A45
:1060D000BF0AE6CFB801882777FD8095982F0E94E8
:1060E000CC959B01AC01C701B6010E9400956B01E4
:1060F0007C0135E6832E3CE0932EA12CB12CA0161A
:10610000B1060CF052C0F4012081318142815381EB
:10611000C701B6010E943594F40161937193819394
:1061200091934F01FFEFAF1ABF0AE9CFA114B10459
:1061300039F425E6822E2CE0922EA12CB12C1DC024
:106140000A151B050CF0850101501109602FCE01C5
:1061500001960E94E4779B01AC01000F111F000F14
:10616000111F0B59134FC701B6010E943594F80156
:10617000608371838283938318C0A016B106ACF448
:106180006A2DCE0101960E94E4779B01AC01C70104
:10619000B6010E943594F4016193719381939193B8
:1061A0004F01FFEFAF1ABF0AE8CFA2960FB6F894DF
:1061B000DEBF0FBECDBFDF91CF911F910F91FF903A
:1061C000EF90DF90CF90BF90AF909F908F90089509
:1061D000CF93DF93C6EED4E060E088810E943B88D5
:1061E00082E090E00E94198761E088810E943B88EC
:1061F0008AE090E00E94198760E088810E943B88D5
:1062000020E432E44FE050E061E08091E4040E9439
:1062100098880E94CA9520E030E048EC52E40E9441
:1062200000952091040E3091050E4091060E50917C
:10623000070E0E94609720E030E44CE156E40E9493
:10624000009520E030E040E05FE30E946097DF913E
:10625000CF910895CF92DF92EF92FF92B9DF6B0159
:106260007C0120E030E040E050E40E94A196181646
:106270001CF4AEDF6B017C0120E030E040E050E434
:10628000C701B6010E94A19618161CF4A1DF6B018C
:106290007C0120E030E040E050E4C701B6010E94FC
:1062A000A19618161CF494DF6B017C0120E030E00D
:1062B00040E050E4C701B6010E94A19618162CF4E4
:1062C000FF90EF90DF90CF9083CFC701B601FF9092
:1062D000EF90DF90CF9008954F925F926F927F92F0
:1062E0008F929F92AF92BF92CF92DF92EF92FF92E6
:1062F000CF93DF9300D01F92CDB7DEB7ABDF9B010A
:10630000AC0169833A834B835C830E94D0862B0166
:106310003C016EE170E080E090E00E94F3869ADF3D
:106320006B017C010E94D0864B015C0184189508AA
:10633000A608B70829813A814B815C8181ED8816D6
:1063400087E09806A104B1040CF43DC0C701B60172
:106350000E9435946B017C0120E030E0A9010E948D
:10636000A19618165CF426EA3BE944EC5BE3C7010E
:10637000B6010E94FC9487FF0BC025C026EA3BE9CA
:1063800044EC5BEBC701B6010E94A1961816DCF045
:10639000C501B40128EE33E040E050E00E94C5980A
:1063A000CA01B9010E94CC954B015C0120E030E0AC
:1063B0004AE754E4C701B6010E946097A501940121
:1063C0000E94009503C060E070E0CB010F900F9039
:1063D0000F900F90DF91CF91FF90EF90DF90CF90D3
:1063E000BF90AF909F908F907F906F905F904F90F5
:1063F000089523E333E948E853E40E94009520E040
:1064000030E040E85FE30E9436940E94139826E64D
:1064100036EA45EA53E40E9460976093040E709355
:10642000050E8093060E9093070E08954F925F928B
:106430006F927F928F929F92AF92BF92CF92DF9294
:10644000EF92FF92CF93DF93CDB7DEB76C970FB685
:10645000F894DEBF0FBECDBF6B017C010E94C486E5
:106460006D8B7E8B8F8B988F61E08091E6040E940C
:10647000028860E08091E4040E9402888EE29DE040
:106480000E9467626093000E7093010E8093020E6B
:106490009093030EAEDFDEDE6D877E878F87988B4D
:1064A0000E94D086698B7A8B8B8B9C8B6AE070E024
:1064B00080E090E00E94F38662E272E08CE09DE072
:1064C0000E94079220E030E04AE754E4C701B60199
:1064D0000E946097698F7A8F8B8F9C8F412C512CF3
:1064E0003201C12CD12C7601C701B6010E94CC9596
:1064F000298D3A8D4B8D5C8D0E94FC9487FF87C15E
:106500000E94C4862D893E894F89588D621B730B6A
:10651000840B950B0E94CA9520E030E04AE754E4D2
:106520000E940095AB01BC0123E0CE0101960E94C0
:10653000AB91BE016F5F7F4F86E09DE00E9410919E
:10654000CE0101960E941E9085DE6B017C010E94A7
:10655000D0864B015C0189899A89AB89BC89881AEC
:10656000990AAA0ABB0A91ED891697E09906A10437
:10657000B1040CF441C020E030E0A901C701B6012C
:106580000E94A19618165CF426EA3BE944EC5BE312
:10659000C701B6010E94FC9487FF0BC02DC026EAFC
:1065A0003BE944EC5BEBC701B6010E94A1961816CB
:1065B0001CF1C501B40128EE33E040E050E00E9438
:1065C000C598CA01B9010E94CC954B015C012D858B
:1065D0003E854F855889C701B6010E94359420E059
:1065E00030E04AE754E40E946097A50194010E94BC
:1065F00000954B015C0103C0812C912C540166E095
:106600007DE0CE0101960E9408916DEB76E0CE010F
:1066100001960E949392BC0186E09DE00E94F39057
:10662000CE0101960E941E9023E0B701A601CE0183
:1066300007960E94AB91BE01695F7F4FCE01019624
:106640000E94089164EB76E0CE0101960E9493923D
:10665000BC0180E09DE00E94F390CE0101960E9473
:106660001E90CE0107960E941E9022E0B501A40163
:10667000CE0101960E94AB9163E675E0CE010796CC
:106680000E94899066E07DE0CE0107960E9482928A
:1066900067EB76E00E94939260E07DE00E94829238
:1066A00067EC76E00E949392BE016F5F7F4F0E947D
:1066B00082926BEB76E00E949392BC018CE09DE0AD
:1066C0000E945A92CE0107960E941E90CE0101961A
:1066D0000E941E9020E030E0A901C501B4010E9493
:1066E000A19687FD06C060E375E080E09DE00E9412
:1066F000609222E0B501A401CE0107960E94AB9101
:10670000BE01695F7F4FCE0101960E9408916BEB3D
:1067100076E0CE0101960E949392BC0180E09DE05C
:106720000E945A92CE0101960E941E90CE010796B9
:106730000E941E906CE07DE0CE0101960E940891BF
:10674000CE0101960E94DC0FCE0101960E941E90A0
:10675000C301B20125E030E040E050E00E94C5985E
:10676000672B682B692B21F56FEB76E0CE01019644
:106770000E94899045E050E060E070E0CE01019613
:106780000E94EE09CE0101960E941E9060E07DE01D
:10679000CE0101960E94089145E050E06FEF7FEF37
:1067A000CE0101960E94620BCE0101960E941E90BE
:1067B00064E97BE08CE09DE00E94269165E070E05A
:1067C00080E090E00E94F3860E94C4866B017C0109
:1067D0002D893E894F89588DC21AD30AE40AF50AD9
:1067E00039DD6D877E878F87988B0E94D086698B75
:1067F0007A8B8B8B9C8B6AE070E080E090E00E944B
:10680000F3863FEF431A530A630A730A6DCE60E0C2
:106810008091E6040E9402886C960FB6F894DEBF61
:106820000FBECDBFDF91CF91FF90EF90DF90CF9063
:10683000BF90AF909F908F907F906F905F904F90A0
:1068400008950F931F93CF93DF93CDB7DEB72C97A7
:106850000FB6F894DEBF0FBECDBF06EE14E061E0C8
:10686000F80180810E94028860E08091E4040E9427
:1068700002888EE29DE00E9467626093000E709332
:10688000010E8093020E9093030EB3DDE3DCAB01A7
:10689000BC0123E0CE0107960E94AB91BE01695F67
:1068A0007F4FCE0101960E9408916CE677E0CE0101
:1068B00001960E949392BC0186E09DE00E94F390B5
:1068C000CE0101960E941E90CE0107960E941E9056
:1068D00068EB76E0CE0101960E94899066E07DE04B
:1068E000CE0101960E948292BC018CE09DE00E9444
:1068F000F390CE0101960E941E90EEDCAB01BC012C
:1069000022E0CE0107960E94AB91BE01695F7F4FE6
:10691000CE0101960E9408916BEB76E0CE010196C4
:106920000E949392BC0180E09DE00E94F390CE0112
:1069300001960E941E90CE0107960E941E9066EC62
:1069400076E0CE0101960E94899060E07DE0CE0164
:1069500001960E948292BC018CE09DE00E945A92B6
:10696000CE0101960E941E9060E375E0CE01019673
:106970000E94899060E07DE0CE0101960E948292A3
:10698000BC0186E09DE00E945A92CE0101960E94D1
:106990001E906FEB76E0CE0101960E9489904AE04E
:1069A00050E060E070E0CE0101960E94EE09CE0159
:1069B00001960E941E9066E07DE0CE0101960E9445
:1069C000089145E050E06FEF7FEFCE0101960E9405
:1069D000620BCE0101960E941E906AEC76E08CE07C
:1069E0009DE00E94609260E0F80180810E94028830
:1069F0002C960FB6F894DEBF0FBECDBFDF91CF91BE
:106A00001F910F9108958F929F92AF92BF92CF9254
:106A1000DF92EF92FF920F9320E044E064E18CE17B
:106A20009EE00E946C656DED76E08EE09EE00E9437
:106A3000899063EE76E088E09EE00E94899020E1F4
:106A400041E168E18DEF9DE00E944D7354E0E52E39
:106A500004E02AEC34E04EEC54E062ED74E08EE8A1
:106A60009DE00E941E788AE79DE00E94826E64E9A4
:106A70007BE080E79DE00E9489908091BE04909128
:106A8000BF0490936F0D80936E0D8090450290909F
:106A90004602A0904702B0904802209141023091F6
:106AA00042024091430250914402C501B4010E9448
:106AB00035946B017C0160936A0D70936B0D80932C
:106AC0006C0D90936D0D6091490270914A02809116
:106AD0004B0290914C0260935E0D70935F0D80931A
:106AE000600D9093610D8092620D9092630DA09263
:106AF000640DB092650D20913D0230913E024091AF
:106B00003F02509140020E9435949B01AC01C701A5
:106B1000B6010E9400956093660D7093670D809397
:106B2000680D9093690D4FEF5FEFBA0185E49DE02A
:106B30000E946B698EE29DE00E94486164E97BE0FF
:106B400084E29DE00E94899064E97BE08EE19DE013
:106B50000E94899064E97BE088E19DE00E94899031
:106B600064E97BE082E19DE00E94899064E97BE03A
:106B70008CE09DE00E94899064E97BE086E09DE0E6
:106B80000E94899064E97BE080E09DE00E9489900A
:106B9000609132027091330284EE9BE00F91FF907E
:106BA000EF90DF90CF90BF90AF909F908F900C941C
:106BB000997C80E09DE00E941E9086E09DE00E940E
:106BC0001E908CE09DE00E941E9082E19DE00E945C
:106BD0001E9088E19DE00E941E908EE19DE00E9443
:106BE0001E9084E29DE00E941E9089EB9AE09093B3
:106BF000460D8093450D80E79DE00E941E9088E041
:106C00009EE00E941E908EE09EE00C941E906F927B
:106C10007F928F929F92AF92BF92CF92DF92EF922C
:106C2000FF920F931F93CF93DF93CDB7DEB7E89713
:106C30000FB6F894DEBF0FBECDBF4B015C0183E6FB
:106C400090E10E94338A64E670E080E090E00E9468
:106C5000F38640E855E260E070E083E690E10E9450
:106C60004B0964E670E080E090E00E94F38661E901
:106C700072E086E09DE00E94079266E07DE0CE0132
:106C800001960E94089142E350E06FEF7FEFCE0142
:106C900001960E94EE09CE0101960E941E9066E8C0
:106CA00072E086E09DE00E94079266E07DE0CE0102
:106CB00001960E94089142E350E06FEF7FEFCE0112
:106CC00001960E94620BCE0101960E941E90809157
:106CD000280E9091290E8D7F712CC12CD12CE12C86
:106CE000F12C00E010E0019709F459C0F2E46F2E96
:106CF0000E94C486681979098A099B09683B7B4010
:106D00008105910508F04BC083E690E10E94C4889C
:106D1000892BF1F14CED55E060E070E083E690E105
:106D20000E94368F68AE41E050E0BE01685C7F4F44
:106D300083E690E10E941D90882351F14FE150E0DD
:106D4000BE016F5F7F4F83E690E10E943C8F898197
:106D50008D34F1F46FE1CE0101960E94A7288823BB
:106D6000B9F00C8110E0102F00278D81080F111D44
:106D7000EE80F12CFE2CEE248F81E80EF11CC884ED
:106D8000D12CDC2CCC248985C80ED11C772473949B
:106D900062E370E080E090E00E94F386A9CF0E9459
:106DA000C486681979098A099B09683B7B4081057B
:106DB000910510F47110C3C00E94290C66E07DE0BB
:106DC000CE0180960E94089142E350E066E070E0B8
:106DD000CE0180960E94EE09CE0180960E941E9000
:106DE000772009F4D1C082E090E09093290E80933F
:106DF000280E4AE0B601CE0180960E9454914AE0E6
:106E0000B701CE0186960E9454914AE0B801CE01A6
:106E1000C2960E945491BE016E5C7F4FCE018C964B
:106E20000E9408916FEE79E0CE018C960E949392B9
:106E3000BE016A5D7F4F0E9482926FEE79E00E94F0
:106E40009392BE01605E7F4F0E948292BC018CE0F3
:106E50009DE00E94F390CE018C960E941E90CE0180
:106E6000C2960E941E90CE0186960E941E90CE0170
:106E700080960E941E906CE07DE0CE0180960E947C
:106E800008914AE050E06FEF7FEFCE0180960E94BC
:106E9000620BCE0180960E941E906BEE76E08CE134
:106EA0009EE00E94D48C61EF76E08CE09DE00E9431
:106EB00026914AE0B601CE0180960E9454914AE0A4
:106EC000B701CE0186960E9454914AE0B801CE01E6
:106ED000C2960E945491BE016E5C7F4FCE018C968B
:106EE0000E94089160E375E0CE018C960E94939217
:106EF000BE016A5D7F4F0E94829260E375E00E944E
:106F00009392BE01605E7F4F0E9482926BEE76E0AC
:106F10000E949392BC018CE09DE00E945A92CE01A7
:106F20008C960E941E90CE01C2960E941E90CE01A9
:106F300086960E941E90CE0180960E941E9062E36B
:106F400070E080E090E00E94F38683E690E10E948A
:106F5000338A62E370E080E090E00E94F386E89676
:106F60000FB6F894DEBF0FBECDBFDF91CF911F915A
:106F70000F91FF90EF90DF90CF90BF90AF909F90D8
:106F80008F907F906F9008956BE772E08CE09DE0AA
:106F90000E9407926CE07DE0CE0180960E940891ED
:106FA0004AE050E060E070E0CE0180960E94620B03
:106FB000CE0180960E941E9068E672E08CE09DE013
:106FC0000E9407928091280E9091290E029709F055
:106FD000B6CF1092290E1092280EB1CF7F928F92C9
:106FE0009F92AF92BF92CF92DF92EF92FF920F9358
:106FF0001F93CF93DF9300D000D0CDB7DEB74C0105
:1070000083E690E10E94338A40E052EC61E070E058
:1070100083E690E10E944B094CED55E060E070E0A2
:1070200083E690E10E94368F64E670E080E090E0B5
:107030000E94F386A12CB12C712CA814B9040CF079
:1070400051C065E070E080E090E00E94F38600E0CF
:1070500010E0C12CD12C760171100FC083E690E1B5
:107060000E94C488892B31F485E1C816D104E1045B
:10707000F1041CF40330110554F08FEFA81AB80A7C
:1070800064E670E080E090E00E94F386D6CF83E66D
:1070900090E10E94C488892B69F083E690E10E9408
:1070A000DD88E1E0F0E0EC0FFD1FE00FF11F8083D1
:1070B0000F5F1F4F65E070E080E090E00E94F38674
:1070C000023011054CF089818B3B31F477247394A5
:1070D0008A818A3A09F0712C8FEFC81AD80AE80A17
:1070E000F80ABACF872D26960FB6F894DEBF0FBEEA
:1070F000CDBFDF91CF911F910F91FF90EF90DF9067
:10710000CF90BF90AF909F908F907F9008958F9277
:107110009F92AF92BF92CF92DF92EF92FF920F9326
:107120001F93CF93DF93CDB7DEB72C970FB6F894AC
:10713000DEBF0FBECDBF61E08091F6040E940288E1
:1071400061E08091F6040E943B888CE19EE00E9401
:107150007A658CE19EE00E94BF664CEE54E060E0F0
:107160008CE19EE00E9480660E94290C0E942E2DD8
:107170008EED93E090938E0C80938D0C0E94739C07
:1071800080932A0E8FED93E00E94739C80932B0EC8
:1071900080912A0E90912B0E1816190654F4109215
:1071A000F804019731F410922B0E10922A0E0E94CF
:1071B0009E0964E37CE0CE0101960E9427924AE09A
:1071C00050E06FEF7FEFCE0101960E94EE09CE01F5
:1071D00001960E941E9040E052EC61E070E086EC67
:1071E0009FE00E944B098091F804882331F068EEFB
:1071F00073E080E090E00E94F38686EC9FE00E94BE
:10720000DD88182F823709F441C110928E0C10923C
:107210008D0C95EEC92E9BE0D92EE12CF12CC701E7
:107220000E94739CD6018D936D01BFEFEB1AFB0A90
:10723000E8E7EE16F10499F78091E50B9091E60BE3
:10724000A091E70BB091E80B85369105A105B1053A
:107250000CF41CC18093380290933902A0933A0237
:10726000B0933B028091E90B9091EA0BA091EB0B5C
:10727000B091EC0B8093340290933502A0933602C8
:10728000B09337028091ED0B9091EE0BA091EF0B34
:10729000B091F00B80932E0290932F02A0933002B6
:1072A000B093310261E07CE0CE0101960E948990AA
:1072B000BE016F5F7F4F8EE09EE00E941091CE0175
:1072C00001960E941E908091F10B9091F20BA0917B
:1072D000F30BB091F40B8093220290932302A093BE
:1072E0002402B09325028091F50B9091F60BA091AA
:1072F000F70BB091F80B80931E0290931F02A0939E
:107300002002B09321028091F90B9091FA0BA09189
:10731000FB0BB091FC0B80931A0290931B02A0937D
:107320001C02B0931D028091FD0B9091FE0BA09169
:10733000FF0BB091000C8093160290931702A0935C
:107340001802B09319028091090C90910A0CA09137
:107350000B0CB0910C0C8093450290934602A093C5
:107360004702B093480280910D0C90910E0CA091B1
:107370000F0CB091100C8093410290934202A093A5
:107380004302B09344028091110C9091120CA09191
:10739000130CB091140C8093490290934A02A0936D
:1073A0004B02B0934C028091150C9091160CA09159
:1073B000170CB091180C80933D0290933E02A0935D
:1073C0003F02B09340028091190C90911A0CA09149
:1073D0001B0CB0911C0C80934D0290934E02A09315
:1073E0004F02B0935002C0902F0CD090300CE09020
:1073F000310CF090320CA7019601C701B6010E9432
:107400005498811108C0C0921202D0921302E092E7
:107410001402F092150260915B0C70915C0C88274D
:1074200077FD8095982F0E94CC959B01AC010E941E
:107430005498882321F010925C0C10925B0C03E3AB
:10744000A02E0CE0B02E85E6882E8CE0982ED5017B
:10745000CD90DD90ED90FD905D01A7019601C701F3
:10746000B6010E945498811105C0F401C082D182F6
:10747000E282F382F4E08F0E911C8BE5A8168CE07B
:10748000B80629F781E090E00E94F32B0EE8010F87
:10749000023070F08091E50B9091E60BA091E70B24
:1074A000B091E80B85369105A105B1050CF045C1F9
:1074B0008091380290913902A0913A02B0913B023A
:1074C0008093E50B9093E60BA093E70BB093E80B4A
:1074D0008091340290913502A0913602B09137022A
:1074E0008093E90B9093EA0BA093EB0BB093EC0B1A
:1074F00080912E0290912F02A0913002B091310222
:107500008093ED0B9093EE0BA093EF0BB093F00BE9
:10751000123751F420E030E048E050E061E07CE0D8
:107520008EE09EE00E94EF928091220290912302D1
:10753000A0912402B09125028093F10B9093F20B5D
:10754000A093F30BB093F40B80911E0290911F0255
:10755000A0912002B09121028093F50B9093F60B3D
:10756000A093F70BB093F80B80911A0290911B0235
:10757000A0911C02B0911D028093F90B9093FA0B1D
:10758000A093FB0BB093FC0B809116029091170215
:10759000A0911802B09119028093FD0B9093FE0BFD
:1075A000A093FF0BB093000C80914502909146028E
:1075B000A0914702B09148028093090C90930A0C65
:1075C000A0930B0CB0930C0C80914102909142025D
:1075D000A0914302B091440280930D0C90930E0C45
:1075E000A0930F0CB093100C8091490290914A0225
:1075F000A0914B02B0914C028093110C9093120C0D
:10760000A093130CB093140C80913D0290913E0214
:10761000A0913F02B09140028093150C9093160CFC
:10762000A093170CB093180C80914D0290914E02CC
:10763000A0914F02B09150028093190C90931A0CB4
:10764000A0931B0CB0931C0C80911202909113021A
:10765000A0911402B091150280932F0C9093300CDE
:10766000A093310CB093320CE5E6FCE023E33CE060
:107670004191519161917191D9014D935D936D93B8
:107680007D939D01BCE0ED38FB0791F76EE17CE056
:10769000CE0101960E942792CE0101960E94C20956
:1076A000CE0101960E941E90A4E9CA2EA4E0DA2E13
:1076B000BDE1AB2EBCE0BB2EE12CF12C80919404FB
:1076C000909195048E159F0574F1F601808191814A
:1076D000D5018D939D935D018091FB0C8823E1F092
:1076E00064E077E086EC9FE00E94D48C4AE050E0B2
:1076F000B70186EC9FE00E94BE8D61E077E086ECEA
:107700009FE00E94D48CF601608171814AE050E0D4
:1077100086EC9FE00E94C58DFFEFEF1AFF0A82E022
:10772000C80ED11CCBCF023040F410928E0C1092B8
:107730008D0C80E090E00E94750980915B0C909127
:107740005C0C892B41F440E855E260E070E080E099
:1077500091E10E944B0980915B0C90915C0C019728
:1077600041F440E052EC61E070E080E091E10E9481
:107770004B0964E670E080E090E00E94F38664E6E6
:1077800070E080E090E00E94F38684EE9BE00E942F
:107790009E7C66E077E0CE0101960E9489904AE0E7
:1077A00050E06FEF7FEFCE0101960E94EE09CE010F
:1077B00001960E941E9080915B0C90915C0C892B2D
:1077C00009F56AE075E0CE0107960E9489906EE0A7
:1077D0007EE0CE0107960E948292BC01CE01019606
:1077E0000E9408914AE050E06FEF7FEFCE010196D2
:1077F0000E94620BCE0101960E941E90CE01079658
:107800000E941E9080915B0C90915C0C019709F591
:107810006EE075E0CE0107960E9489906EE07EE0F2
:10782000CE0107960E948292BC01CE0101960E9471
:1078300008914AE050E06FEF7FEFCE0101960E9481
:10784000620BCE0101960E941E90CE0107960E9407
:107850001E9064E077E0CE0107960E9489906EE06A
:107860007EE0CE0107960E94829266E177E00E9458
:107870009392BC01CE0101960E940891CE0101961F
:107880000E94DC0FCE0101960E941E90CE01079649
:107890000E941E9064E670E080E090E00E94F38613
:1078A0008CE29EE00E94E26B64E670E080E090E093
:1078B0000E94F38663E270E08CE29EE00E94F56B2A
:1078C00061E070E08CE29EE00E944E098CE29EE056
:1078D0000E94696C83E090E09093290E8093280EBB
:1078E00060E070E08DEF9DE00E9444746B017C01CC
:1078F00062E370E080E090E00E94F386A7019601C9
:10790000C701B6010E945498882309F475C060E04D
:1079100070E08DEF9DE00E9442746B017C0162E398
:1079200070E080E090E00E94F386A7019601C70115
:10793000B6010E945498882309F45EC081E090E06B
:107940009093290E8093280E40E052EC61E070E0A5
:1079500083E690E10E944B0964E670E080E090E0ED
:107960000E94F38682E090E039DB882379F065E0BD
:107970007CE0CE0101960E942792CE0101960E94E2
:10798000C209CE0101960E941E9036C01092290EA7
:107990001092280E83E690E10E94338A64E670E03C
:1079A00080E090E00E94F38640E855E260E070E0FD
:1079B00083E690E10E944B0983E690E10E94C4882F
:1079C000892BD1F06BEE7BE0CE0101960E942792CD
:1079D000CE0101960E94C209CE0101960E941E901E
:1079E00082E090E09093290E8093280E64E670E088
:1079F00080E090E00E94F3868091280E9091290EFD
:107A0000039771F466ED7BE0CE0101960E94279208
:107A1000CE0101960E94C209CE0101960E941E90DD
:107A200063E08EE29DE00E940862811111C060EB6C
:107A30007BE0CE0101960E942792CE0101960E9422
:107A4000DC0FCE0101960E941E9010923C02A3C052
:107A50006DE97BE08CE09DE00E94079240E050E001
:107A6000BA018EE29DE00E9429640E94CC9520E03C
:107A700030E048EC52E40E940095AB01BC0122E0EA
:107A8000CE0107960E94AB91BE01695F7F4FCE0188
:107A900001960E94089161E279E0CE0101960E9470
:107AA0009392BC018CE09DE00E945A92CE01019617
:107AB0000E941E90CE0107960E941E906CE07DE011
:107AC000CE0101960E940891CE0101960E94C20942
:107AD000CE0101960E941E9067E87BE08CE09DE05D
:107AE0000E940792609138027091390280913A02A7
:107AF00090913B020E94CC9520E030E048EC52E4AB
:107B00000E940095AB01BC0122E0CE0107960E94C5
:107B1000AB91BE01695F7F4FCE0101960E94089133
:107B200061E279E0CE0101960E949392BC018CE063
:107B30009DE00E945A92CE0101960E941E90CE01B5
:107B400007960E941E906CE07DE0CE0101960E9497
:107B50000891CE0101960E94C209CE0101960E94B1
:107B60001E90113629F481E00E94A11981E011C014
:107B700086EC9FE00E94DD88182F64E670E080E0CC
:107B800090E00E94F386113671F380E00E94A11903
:107B900080E00E94F20F64E670E080E090E00E94D6
:107BA000F3868091F804882331F068EE73E080E07A
:107BB00090E00E94F3866CEB77E088E19DE00E9404
:107BC000269182E090E09093FA0C8093F90C8091DA
:107BD000F80481110E94F3172C960FB6F894DEBFBB
:107BE0000FBECDBFDF91CF911F910F91FF90EF900E
:107BF000DF90CF90BF90AF909F908F9008952F927D
:107C00003F924F925F926F927F928F929F92AF922C
:107C1000BF92CF92DF92EF92FF920F931F93CF9379
:107C2000DF93CDB7DEB72B970FB6F894DEBF0FBE4C
:107C3000CDBF1C018BEB8F838AEA888781E089871F
:107C400084E6829D9001839D300D11243B872A8715
:107C5000E12CF12CC12CD12C812C912C5401C2147B
:107C6000D30494F1C501B4010E94CC9520E030E02A
:107C700040E251E40E9400956B017C01B10188272C
:107C800077FD8095982F0E94CC959B01AC01C70190
:107C9000B6010E9400952B960FB6F894DEBF0FBE7A
:107CA000CDBFDF91CF911F910F91FF90EF90DF90AB
:107CB000CF90BF90AF909F908F907F906F905F908C
:107CC0004F903F902F9008952A853B85E216F3064A
:107CD0004CF6C7016AE070E00E949098892B79F415
:107CE000E0916310F09164100280F381E02D43E095
:107CF00050E0BE01695F7F4F83E690E1199565E032
:107D000070E080E090E00E94F3863FEFE31AF30A10
:107D100000E010E0412C512C320183E690E10E94FA
:107D2000C488892B39F424E042165104610471049B
:107D30000CF095CF063011050CF091CF83E690E161
:107D40000E94C488892B69F083E690E10E94DD8857
:107D5000E1E0F0E0EC0FFD1FE00FF11F80830F5F0B
:107D60001F4F65E070E080E090E00E94F3860630EF
:107D7000110501F599818F8198131CC09A8188851E
:107D8000981318C09B818985981314C02C818D810C
:107D900090E0A0E0B0E0BA2FA92F982F8827820F9B
:107DA000911DA11DB11D880E991EAA1EBB1E8FEF2D
:107DB000C81AD80A9FEF491A590A690A790AADCF39
:107DC000CF92DF92EF92FF92CF93DF93CDB7DEB7E2
:107DD0002C970FB6F894DEBF0FBECDBF83E690E1BF
:107DE0000E94338A40E052EC61E070E083E690E16B
:107DF0000E944B094CED55E060E070E083E690E1B5
:107E00000E94368F64E670E080E090E00E94F38686
:107E100068E377E08CE09DE00E9426916CE07DE0D5
:107E2000CE0101960E940891CE0101960E94C209DE
:107E3000CE0101960E941E9062E370E080E090E027
:107E40000E94F3866CE07DE0CE0101960E940891CD
:107E500042E350E06FEF7FEFCE0101960E94EE0902
:107E6000CE0101960E941E9064E477E086E09DE0DA
:107E70000E94269166E07DE0CE0101960E94089165
:107E800044E150E06FEF7FEFCE0101960E94620B5C
:107E9000CE0101960E941E908091280E9091290E8D
:107EA000019731F484E090E0AADE6B017C0103C00D
:107EB000C12CD12C76018091280E9091290E892B0E
:107EC00029F481E090E09BDE6B017C0120E030E052
:107ED00040EA51E4C701B6010E94A196181664F564
:107EE00021E0B701A601CE0107960E94AB9164EB99
:107EF00079E0CE0101960E948990BE01695F7F4FB3
:107F0000CE0101960E94829266E376E00E949392EF
:107F1000BC018CE09DE00E94F390CE0101960E948E
:107F20001E90CE0107960E941E9081E090E09093F3
:107F3000290E8093280E10C060E577E08CE09DE06C
:107F40000E9426918091280E9091290E019721F48C
:107F50001092290E1092280E6CE07DE0CE01019661
:107F60000E9408914AE050E060E070E0CE01019686
:107F70000E94EE09CE0101960E941E906CE07DE009
:107F8000CE0101960E94089160E375E0CE01019652
:107F90000E94939266E07DE00E948292BC018CE098
:107FA0009DE00E94F390CE0101960E941E9083E610
:107FB00090E10E94338A8091FD0C882331F060E2C9
:107FC00073E080E090E00E94F3862C960FB6F89460
:107FD000DEBF0FBECDBFDF91CF91FF90EF90DF905E
:107FE000CF9008952F923F924F925F926F927F921F
:107FF0008F929F92AF92BF92CF92DF92EF92FF92B9
:108000000F931F93CF93DF93CDB7DEB766970FB66D
:10801000F894DEBF0FBECDBF6C0183E690E10E94F5
:10802000338A40E855E260E070E083E690E10E9428
:108030004B0964E670E080E090E00E94F3864CED2E
:1080400055E060E070E083E690E10E94368F64E6E0
:1080500070E080E090E00E94F3868FEF898381E0FA
:108060008A8386E88B831C821D821E821F8218866B
:1080700089E78987C601880F991F9E8B8D8B212CDC
:10808000312CE12CF12C812C912C5401EC14FD04A9
:108090004CF083E690E10E94338AE114F104B9F1D7
:1080A000670135C08D899E892816390694F783E6C5
:1080B00090E10E94558A08977CF0E0916310F0915E
:1080C00064100280F381E02D49E050E0BE016F5F53
:1080D0007F4F83E690E1199565E070E080E090E0E5
:1080E0000E94F38600E010E0412C512C320183E61F
:1080F00090E10E94C488892B31F4E4E04E165104CB
:108100006104710484F5023011056CF530C0C501BD
:10811000B4010E94CC954B015C01B601882777FD24
:108120008095982F0E94CC959B01AC01C501B401AC
:108130000E94009566960FB6F894DEBF0FBECDBFC5
:10814000DF91CF911F910F91FF90EF90DF90CF9033
:10815000BF90AF909F908F907F906F905F904F9067
:108160003F902F900895FFEF2F1A3F0A8FCF83E69D
:1081700090E10E94C488892B69F083E690E10E9417
:10818000DD88EAE0F0E0EC0FFD1FE00FF11F8083D7
:108190000F5F1F4F65E070E080E090E00E94F38683
:1081A0000230110569F59A858981981329C09B854C
:1081B0008B81981325C0FE013C96FC8BEB8B83E6EC
:1081C00090E10E94C488892B31F4F4E04F165104E9
:1081D00061047104DCF409301105E1F42D858C850E
:1081E00090E0982F8827820F911DAA2797FDA095D0
:1081F000BA2F880E991EAA1EBB1E8FEFE81AF80A26
:108200009FEF491A590A690A790A71CF043011059A
:10821000A4F3E4CF83E690E10E94DD88EB89FC893A
:108220008193FC8BEB8B0F5F1F4FC9CF8091F504BF
:10823000882349F08091F404882329F060E08CE1E0
:108240009EE00C94BA6608952F923F924F925F92EF
:108250006F927F928F929F92AF92BF92CF92DF9256
:10826000EF92FF920F931F93CF93DF93CDB7DEB7BB
:1082700063970FB6F894DEBF0FBECDBF8B8B60E067
:108280000E9402888091FD0C811105C08FE090E072
:10829000A0E0B0E004C082E090E0A0E0B0E08F8712
:1082A000988BA98BBA8B6CE577E08CE09DE00E94FF
:1082B00026916CE07DE0CE0101960E9408914AE093
:1082C00050E06FEF7FEFCE0101960E94EE09CE01E4
:1082D00001960E941E90C12CD12C7601312C1D8656
:1082E0001E86212C02E310E0412C512C32018B8997
:1082F0000E948987AA2797FDA095BA2F480E591E7C
:108300006A1E7B1E65E070E080E090E00E94F386CC
:108310000150110961F78090120290901302A09011
:108320001402B0901502C301B2010E94CC9520E066
:1083300030E040EA50E40E94609720E030E040E8FE
:108340005AE30E94609720E030E048E452E40E9443
:108350000095A50194010E94359420E030E040E7AB
:1083600051E40E9460972B013C01A50194016AE948
:1083700079E989E390E40E9435949B01AC01C30143
:10838000B2010E94009520E030E0A9010E943694DD
:1083900020E030E040E251E40E9460975B018C01F4
:1083A000232D3D854E85522D0E94A196181624F44A
:1083B0003A2CBD860E87212E20E030E0A901B501C0
:1083C000C8010E94FC9487FF04C0A12CB12C00E0DE
:1083D00010E022E0A501B801CE0107960E94AB9102
:1083E000BE01695F7F4FCE0101960E94089169E648
:1083F00077E0CE0101960E949392BC0186E09DE059
:108400000E94F390CE0101960E941E90CE01079625
:108410000E941E9066E07DE0CE0101960E940891C8
:108420004AE050E060E070E0CE0101960E94620BED
:10843000CE0101960E941E900E94C4868090E8049E
:108440009090E904A090EA04B090EB040091140E1F
:108450001091150E2091160E3091170E800E911E60
:10846000A21EB31E86169706A806B90608F4DDC03C
:108470000E94C4860E94CA954B015C016091E80489
:108480007091E9048091EA049091EB040E94CC95EC
:1084900020E030E040E85EE30E9460972B013C0161
:1084A0006091140E7091150E8091160E9091170E1A
:1084B0000E94CC959B01AC01C301B2010E9436948D
:1084C0009B01AC01C501B4010E94FC9487FDADC0C5
:1084D0006CE370E080E090E00E94F3869FEFC91AA1
:1084E000D90AE90AF90A8F859889A989BA898C1568
:1084F0009D05AE05BF050CF0F5CE64E670E080E0AA
:1085000090E00E94F3860E94290C64E670E080E00F
:1085100090E00E94F3866EE677E086E09DE00E94A0
:10852000269166E07DE0CE0101960E94089144E12B
:1085300050E060E070E0CE0101960E94EE09CE01AD
:1085400001960E941E9022E0432D5D856E85722D5E
:10855000CE0107960E94AB91BE01695F7F4FCE01AD
:1085600001960E94089169E677E0CE0101960E948B
:108570009392BC0186E09DE00E94F390CE010196AB
:108580000E941E90CE0107960E941E9066E07DE03C
:10859000CE0101960E94089142E350E06FEF7FEF19
:1085A000CE0101960E94620BCE0101960E941E90A0
:1085B0003DDE62E370E080E090E00E94F38666E7D3
:1085C00077E0CE0101960E94899066E07DE0CE01C1
:1085D00001960E9482926AE777E00E9493926CE093
:1085E0007DE00E948292BC018CE09DE00E94F390AD
:1085F000CE0101960E941E9063960FB6F894DEBFDE
:108600000FBECDBFDF91CF911F910F91FF90EF90E3
:10861000DF90CF90BF90AF909F908F907F906F90A2
:108620005F904F903F902F90089500DE51CFFF92C2
:108630000F931F93CF93DF93CDB7DEB72C970FB671
:10864000F894DEBF0FBECDBF1092FE0C64E97BE054
:1086500084E29DE00E94269111E086EC9FE00E945A
:10866000C4882091FE0C18161906C4F5211136C0D5
:1086700086EC9FE00E94DD888093FF0C8A3041F0F9
:108680008D3031F0682F84E29DE00E946F921FC010
:108690001093FE0C6EE777E0CE0107960E9489905A
:1086A00064E27DE0CE0107960E948292BC01CE0179
:1086B00001960E940891CE0101960E94C209CE0146
:1086C00001960E941E90CE0107960E941E906AE0BD
:1086D00070E080E090E00E94F386BFCF222361F03B
:1086E0002091FE0C8091280D9091290D211174C0CC
:1086F000009709F071C0B8C000E010E0FF24F394C7
:1087000080E091E10E94C48818161906A4F580E063
:1087100091E10E94DD888093FF0C8A3071F08D30EA
:1087200061F09091FE0C911108C0682F84E29DE0E9
:108730000E946F920F5F1F4F17C08091280D90917C
:10874000290D892B89F0F092FE0C80E091E10E94C6
:10875000C4881816190644F464E97BE084E29DE0BD
:108760000E9426911092FE0C6FE070E080E090E095
:108770000E94F386C5CF62E370E080E090E00E9443
:10878000F386012B09F4ACCF67E877E0CE010796BA
:108790000E94899064E27DE0CE0107960E94829259
:1087A000BC01CE0101960E940891CE0101960E9463
:1087B000C209CE0101960E941E90CE0107960E942A
:1087C0001E9080E091E10E944C8964E670E080E0B8
:1087D00090E00E94F38684CF019709F069C06DEBA9
:1087E00076E0CE0107960E948990BE01695F7F4FB7
:1087F00084E29DE00E94CF92811115C06DE877E080
:10880000CE0101960E948990BE016F5F7F4F84E286
:108810009DE00E94CF9211E0811110E0CE010196FF
:108820000E941E9001C010E0CE0107960E941E908B
:10883000112399F040E050E064E27DE0CE01019622
:108840000E943F09BE016F5F7F4F88E19DE00E945B
:108850001091CE0101960E941E9064E170E080E0CC
:1088600090E00E94F38624C064E670E080E090E02F
:108870000E94F3860E94C486CB0168EE73E00E94DA
:108880009098CB0164E670E00E9490988236910542
:108890007CF08091FD0C81110BC088E19DE00E946D
:1088A0000F94613071058105910511F40E94F31751
:1088B0002C960FB6F894DEBF0FBECDBFDF91CF91DF
:1088C0001F910F91FF900895BF92CF92DF92EF9288
:1088D000FF920F931F93CF93DF93CDB7DEB72B9704
:1088E0000FB6F894DEBF0FBECDBF6C0183E690E1FA
:1088F0000E94338A40E855E260E070E083E690E150
:108900000E944B0964E670E080E090E00E94F386EC
:108910004CED55E060E070E083E690E10E94368F18
:1089200064E670E080E090E00E94F3868FEF898338
:1089300081E08A8386E88B831C821D821E821F82CF
:10894000188689E7898783E690E10E944C8962E373
:1089500070E080E090E00E94F38683E690E10E9460
:10896000558A08977CF0E0916310F09164100280C2
:10897000F381E02D49E050E0BE016F5F7F4F83E659
:1089800090E1199562E370E080E090E00E94F38648
:10899000E12CF12CB12CEC14FD040CF05BC083E64F
:1089A00090E10E94C488892B21F183E690E10E9426
:1089B000558A08977CF0E0916310F0916410028072
:1089C000F381E02D49E050E0BE016F5F7F4F83E609
:1089D00090E1199565E070E080E090E00E94F386F8
:1089E00000E010E083E690E10E94C48802301105A7
:1089F00054F062E370E080E090E00E94F3868FEF35
:108A0000E81AF80AC8CF83E690E10E94C488892B4F
:108A100069F083E690E10E94DD88EAE0F0E0EC0F87
:108A2000FD1FE00FF11F80830F5F1F4F65E070E0B7
:108A300080E090E00E94F3860230110599F69A8555
:108A400089819813CFCF9B858B819813CBCFBB2483
:108A5000B394C8CF83E690E10E94338A8B2D2B9686
:108A60000FB6F894DEBF0FBECDBFDF91CF911F913F
:108A70000F91FF90EF90DF90CF90BF900895CF922D
:108A8000DF92EF92FF920F931F93CF93DF93CDB7B7
:108A9000DEB72C970FB6F894DEBF0FBECDBF0E9495
:108AA000290C61ED72E08CE09DE00E9407926CE081
:108AB0007DE0CE0101960E9408914AE050E060E01E
:108AC00070E0CE0101960E94EE09CE0101960E944F
:108AD0001E9068EC72E086E09DE00E94079266E0DE
:108AE0007DE0CE0101960E94089144E150E06FEFD5
:108AF0007FEFCE0101960E94620BCE0101960E948B
:108B00001E908091280E9091290E8430910551F489
:108B100081E090E0D9DE81111CC01092290E1092E4
:108B2000280E17C0892BA9F481E090E0CDDE8111D9
:108B30000AC081E090E0C8DE811105C081E090E0CC
:108B4000C3DE882331F084E090E09093290E809377
:108B5000280E8091280E9091290E049791F16CEBCC
:108B600072E08CE09DE00E9407926CE07DE0CE0117
:108B700001960E9408914AE050E060E070E0CE016A
:108B800001960E94EE09CE0101960E941E906CE0B3
:108B90007DE0CE0101960E94089160E375E0CE0170
:108BA00001960E94939266E07DE00E948292BC0151
:108BB0008CE09DE00E94F390CE0101960E941E90F1
:108BC00097C08AE090E00EDA6B017C0120E030E093
:108BD000A9010E94FC9418162CF08AE090E002DAB9
:108BE0006B017C010BE010E020E030E041EE53E44B
:108BF000C701B6010E94FC94181684F420E030E00E
:108C0000A901C701B6010E94FC941816B4F06EEADF
:108C100072E08CE09DE00E94079240C00150110973
:108C200069F368EC70E080E090E00E94F38683E0F6
:108C300090E0D8D96B017C01D7CF20E030E048EC40
:108C400052E4C701B6010E94FC9487FF02C021E0F4
:108C500001C020E0B701A601CE0107960E94AB91AA
:108C60006CE276E0CE0101960E948990BE01695FB8
:108C70007F4FCE0101960E94829261E376E00E94CE
:108C80009392BC018CE09DE00E94F390CE0101968E
:108C90000E941E90CE0107960E941E906CE07DE01F
:108CA000CE0101960E94089142E350E06FEF7FEF02
:108CB000CE0101960E94620BCE0101960E941E9089
:108CC00065EA72E086E09DE00E94079266E07DE042
:108CD000CE0101960E94089142E350E060E070E00E
:108CE000CE0101960E94EE09CE0101960E941E90CF
:108CF0008091FD0C882331F060E273E080E090E029
:108D00000E94F3862C960FB6F894DEBF0FBECDBF3F
:108D1000DF91CF911F910F91FF90EF90DF90CF9057
:108D200008954F925F926F927F928F929F92AF922F
:108D3000BF92CF92DF92EF92FF92CF93DF93CDB7A6
:108D4000DEB760970FB6F894DEBF0FBECDBF80913F
:108D5000FD0C811105C08EE190E0A0E0B0E004C000
:108D600082E090E0A0E0B0E08D879E87AF87B88B6F
:108D700064E173E08CE09DE00E9407926CE07DE08E
:108D8000CE0101960E9408914AE050E06FEF7FEF1C
:108D9000CE0101960E94620BCE0101960E941E90A8
:108DA000812C912C5401C12CD12C760163E270E00E
:108DB0008CE29EE00E94F56B67E070E08CE29EE042
:108DC0000E944E098CE29EE00E94696C66E970E0A8
:108DD00080E090E00E94F38663E270E08CE29EE027
:108DE0000E94F56B60E270E08CE29EE00E944E090A
:108DF0008CE29EE00E94696C66E970E080E090E0A1
:108E00000E94F38642E050E063E270E08CE29EE074
:108E10000E94676C412C512C32018CE29EE00E9432
:108E20004D6B181619066CF48CE29EE00E94556B8F
:108E3000762C652C542C4424480E511C611C711C4A
:108E4000ECCFC301B2010E94CC952AE939E949E986
:108E50005FE30E9400950E949995AB01BC01C41686
:108E6000D506E606F70614F46A017B012AE0CE0176
:108E700007960E947F91BE01695F7F4FCE010196E8
:108E80000E9408916FE877E0CE0101960E949392CC
:108E9000BC0186E09DE00E94F390CE0101960E9405
:108EA0001E90CE0107960E941E9066E07DE0CE01E6
:108EB00001960E9408914EE150E060E070E0CE0122
:108EC00001960E94970ACE0101960E941E909FEF84
:108ED000891A990AA90AB90A8D859E85AF85B8892C
:108EE00088159905AA05BB050CF060CF2AE0B701EB
:108EF000A601CE0107960E947F91BE01695F7F4F58
:108F0000CE0101960E9408916FE877E0CE010196AC
:108F10000E949392BC0186E09DE00E94F390CE01F6
:108F200001960E941E90CE0107960E941E9066E058
:108F30007DE0CE0101960E9408914AE050E060E099
:108F400070E0CE0101960E94EE09CE0101960E94CA
:108F50001E902AE0B701A601CE0107960E947F91DC
:108F600063E977E0CE0101960E948990BE01695FB6
:108F70007F4FCE0101960E94829266E977E00E94BF
:108F800093926CE07DE00E948292BC018CE09DE0B7
:108F90000E94F390CE0101960E941E90CE0107968A
:108FA0000E941E9062E370E080E090E00E94F386F1
:108FB00060960FB6F894DEBF0FBECDBFDF91CF91A4
:108FC000FF90EF90DF90CF90BF90AF909F908F90E9
:108FD0007F906F905F904F9008958F929F92AF9285
:108FE000BF92CF92DF92EF92FF920F931F93CF9396
:108FF000DF93CDB7DEB72C970FB6F894DEBF0FBE68
:10900000CDBF8C01E090F90CF090FA0C8091FB0C34
:10901000882369F067E478E086EC9FE00E94A38CE7
:109020004AE050E0B80186EC9FE00E94C58DC8017F
:109030000596059708F18091F90C9091FA0C80172C
:10904000910709F10E94290C1093FA0C0093F90C76
:109050000E942E2D4AE0B801CE0101960E94549143
:10906000BE016F5F7F4F88E19DE00E941091CE01AD
:1090700001960E941E9007C00E3F8FEF1807A9F4BB
:109080000E94412D4FC260E375E0CE0101960E941F
:1090900089904AE050E06FEF7FEFCE0101960E9489
:1090A000970ACE0101960E941E90F8017996E53349
:1090B000F10508F0D6C1EE58FF4F0C94E19880916D
:1090C000FD0C882319F00E942134F9C160910A0235
:1090D00070910B0280910C0290910D020E94163249
:1090E000EEC18091E2049091E3040E945C2DE7C1FF
:1090F0008091C8049091C904A7D8E1C18091BC04B3
:109100009091BD040E943F2BDAC18091BE049091E2
:10911000BF04B5DCD4C10E94C4860E940736CFC10B
:1091200060E070E08091C2049091C3040E94FC242E
:10913000C6C18091B8049091B9040E94F328BFC1C0
:109140008091FC0C91E089278093FC0C8091FD0CB0
:10915000882331F06CE07DE080E091E10E94EF8CAB
:1091600068EC70E080E090E00E94F386A8C1109265
:10917000FD0CA5C181E08093FD0C68E17DE08EE1EE
:109180009DE00E94F3908091F90C9091FA0C9093DD
:10919000F80C8093F70C93C10E944E0C90C10E9472
:1091A000E03E8DC10E94B1168AC180913C028823A5
:1091B00009F485C164E97BE0CE0101960E948990A3
:1091C0004AE050E061E070E0CE0101960E94EE09B5
:1091D000CE0101960E941E900E94800E70C1A1DDFA
:1091E0006EC18091C4049091C5040E94802A67C119
:1091F0008091BA049091BB040E948A2960C1809139
:109200003C02882309F45BC18091FD0C882329F07E
:1092100082E090E00E94C41052C183E090E00E947E
:10922000F3144DC10E942C2380E091E10E944C89EF
:1092300046C180918102909182020E9425273FC100
:1092400080913C02882309F43AC18091FD0C811180
:1092500027C0C0900A02D0900B02E0900C02F09060
:109260000D0220E030E04AE754E4C701B6010E9455
:1092700060970E9499954B015C0120E030E040EA44
:1092800050E4C701B6010E94609720E030E040EA58
:1092900050E40E9436940E949995A501940108C05B
:1092A00021E030E040E050E06AE070E080E090E0F3
:1092B0000E94FC1E04C180915B0C90915C0C892B78
:1092C000F1F581E090E090935C0C80935B0C6BE98E
:1092D00077E0CE0101960E948990CE0101960E940E
:1092E000C209CE0101960E941E906EE075E0CE018B
:1092F00007960E9489906EE07EE0CE0107960E945C
:109300008292BC01CE0101960E94089148EC50E087
:109310006FEF7FEFCE0101960E94EE09CE0101961C
:109320000E941E90CE0107960E941E9080E091E15F
:109330000E94338A40E052EC61E070E03BC0109242
:109340005C0C10925B0C64EA77E0CE0101960E94FF
:109350008990CE0101960E94C209CE0101960E9419
:109360001E906AE075E0CE0107960E9489906EE03B
:109370007EE0CE0107960E948292BC01CE0101964A
:109380000E94089148EC50E06FEF7FEFCE0101960C
:109390000E94EE09CE0101960E941E90CE01079612
:1093A0000E941E9080E091E10E94338A40E855E2DD
:1093B00060E070E080E091E10E944B0910928E0C19
:1093C00010928D0C80E090E00E94750964E175E0D8
:1093D000CE0107960E94899068E07EE0CE01079654
:1093E0000E948292BC01CE0101960E94089140ED3C
:1093F00057E06FEF7FEFCE0101960E94620BCE0126
:1094000001960E941E90CE0107960E941E9057C0A2
:1094100080912A0E90912B0E892BA1F481E090E08F
:1094200090932B0E80932A0E8EED93E090938E0CEA
:1094300080938D0C0E949E0968EC70E080E090E0C3
:109440000E94F386E091C20BF091C30B199537C0CF
:109450008CE19EE00E94BF660E94290C0E942E2D86
:109460002EC0F092FA0CE092F90C6AE378E08CE0FE
:109470009DE00E94079264E97BE0CE0101960E9484
:1094800089904AE050E060E070E0CE0101960E94D1
:10949000EE09CE0101960E941E906CE07DE0CE01A7
:1094A00001960E9408914AE050E06FEF7FEFCE01F5
:1094B00001960E94620BCE0101960E941E9080913F
:1094C000100D9091110D009799F0419718F402300A
:1094D0001105ACF46CE07DE0CE0101960E9408918C
:1094E000CE0101960E94DC0FCE0101960E941E90D3
:1094F00064E670E080E090E00E94F38613C06CE0C8
:109500007DE0CE0101960E9408914AE050E06FEFA5
:109510007FEFCE0101960E94620BCE0101960E9460
:109520001E90D8CF2C960FB6F894DEBF0FBECDBFDD
:10953000DF91CF911F910F91FF90EF90DF90CF902F
:10954000BF90AF909F908F900895FF920F931F93BD
:10955000CF93DF9300D000D0CDB7DEB7823409F4CB
:1095600041C0CCF4803309F45DC07CF4833209F44B
:1095700050C08A3209F075C06EEB77E084E29DE05E
:109580000E9426918FEF9FEF6AC0813309F459C082
:109590008134E9F066C08136D1F02CF4833469F16E
:1095A000843439F05EC0833641F1E4F0843609F04A
:1095B00058C080911C0D90911D0D892B09F4E7C0B6
:1095C00088E19DE00E940F9497FF68C0E0C062EBC5
:1095D00077E084E29DE00E9426918091F90C9091C1
:1095E000FA0C3DC065EB77E084E29DE00E94269195
:1095F0001092FD0C8CEF9FEF32C068EB77E084E2B5
:109600009DE00E94269181E08093FD0C8DEF9FEFFD
:1096100026C06BEB77E084E29DE00E9426918EEFFE
:109620009FEF1DC06CEC77E088E19DE00E942691E1
:109630006CEC77E084E29DE00E94269180E090E06F
:109640000EC06FEB77E088E19DE00E9426916FEB02
:1096500077E084E29DE00E94269181E090E0BDDC0D
:10966000A1C0682FCE0101960E943C91BE016F5FA0
:109670007F4F88E19DE00E941091CE0101960E94EB
:109680001E9088E19DE00E940F94CB01A6DC64E669
:1096900070E080E090E00E94F38684C08091FB0C33
:1096A000882361F063E378E086EC9FE00E94A38C5E
:1096B00068E17DE086EC9FE00E94EF8C88E19DE010
:1096C0000E940F94DC01CB014AEF5FEF6FEF7FEF59
:1096D000481B590B6A0B7B0B2AE0CE0101960E94B6
:1096E0007F91BE016F5F7F4F88E19DE00E941091E6
:1096F000CE0101960E941E9088E19DE044C00F5F5C
:109700001F4F093E83E0180709F449C06EE170E07D
:1097100080E090E00E94F3868EE89DE00E94F77A58
:10972000F82EFF2061F38FE28F15CCF56AE270E02E
:109730006F197109F7FC73954AE0CE0101960E94FA
:109740005491BE016F5F7F4F84E29DE00E941091B3
:10975000CE0101960E941E9064E27DE088E19DE0CA
:109760000E94F3908091FB0C882359F06CE278E022
:1097700086EC9FE00E94A38C6F2D86EC9FE00E94F8
:109780000F8D84E29DE00E940F94CB0168CF8EE89C
:109790009DE00E94F77AF82E00E010E0C2CF8CEE38
:1097A000F80EC4CF26960FB6F894DEBF0FBECDBF1D
:1097B000DF91CF911F910F91FF9008950F931F9309
:1097C000CF93DF9300D000D0CDB7DEB78091FB0CF4
:1097D0008823A1F064E077E086EC9FE00E94D48CBF
:1097E0004091D80B5091D90B6091DA0B7091DB0B43
:1097F00020E130E086EC9FE00E940C8E8091D80B37
:109800009091D90BA091DA0BB091DB0B883025E059
:109810009207A105B10509F4FCC108F08DC0893497
:1098200021E09207A105B10509F4F6C1E0F5843401
:1098300021E09207A105B10509F4DFC1E8F4813404
:1098400021E09207A105B10509F4C8C138F48034BC
:109850009140A105B10509F4B2C1E1C1823421E012
:109860009207A105B10509F4C2C183349140A10555
:10987000B10509F4BFC1D3C1863421E09207A10527
:10988000B10509F4C0C108F4BBC1873421E09207D7
:10989000A105B10509F4BAC188349140A105B1050B
:1098A00009F4B7C1BCC1823025E09207A105B1051A
:1098B00009F49DC1E8F4843721E09207A105B105C0
:1098C00009F448C138F482379140A105B10509F483
:1098D0004CC1A5C1811525E09207A105B10509F488
:1098E0006EC181309540A105B10509F477C197C1DA
:1098F000853025E09207A105B10509F481C170F416
:10990000833025E09207A105B10509F473C18430C5
:109910009540A105B10509F470C181C1863025E0EB
:109920009207A105B10509F46EC187309540A105E4
:10993000B10509F46BC173C18D3B22E492072FEF8F
:10994000A207B10509F42CC108F04BC08F3E20E1FD
:1099500092072FEFA207B10509F458C118F5823319
:1099600025E09207A105B10509F4FFC038F489305C
:109970009540A105B10509F44FC151C1843325E0DB
:109980009207A105B10509F4E5C08D3F9240AF4FA4
:10999000B10509F044C162EB77E084E29DE00E94EA
:1099A0002691E0C08D3D22E292072FEFA207B1057C
:1099B00009F4D0C038F4873E9841AF4FB10509F49F
:1099C0001FC12DC18F3C20E392072FEFA207B105E5
:1099D00009F413C1873C9843AF4FB10509F419C18D
:1099E0001EC1873928E692072FEFA207B10509F4B7
:1099F000F5C048F58D3A22E592072FEFA207B10591
:109A000009F4BFC038F4853B9A44AF4FB10509F45F
:109A1000D6C005C1853A2AE592072FEFA207B10506
:109A200009F4FAC08D399246AF4FB10509F0F7C07D
:109A300065EB77E084E29DE00E9426911092FD0C98
:109A40008CEF9FEF85C0873528EA92072FEFA2079A
:109A5000B105F9F078F485382AE792072FEFA207CD
:109A6000B10509F4D0C087369849AF4FB10509F464
:109A7000BEC0D5C08F3420EB92072FEFA207B105EF
:109A800009F4B8C08D33924CAF4FB10509F46DC0E5
:109A9000C6C084EE9BE00E94B57C00E010E064EC60
:109AA0007BE084EE9BE00E946A7D892B39F40F5F96
:109AB0001F4F093E83E0180709F09DC18091FB0C00
:109AC0008823A1F069E178E086EC9FE00E94A38CF6
:109AD0004091C80B5091C90B6091CA0B7091CB0B90
:109AE0002AE030E086EC9FE00E940C8E8091C80B4B
:109AF0009091C90BA091CA0BB091CB0B853025E09A
:109B00009207A105B10509F461C108F0E1C08734ED
:109B100021E09207A105B10509F464C108F0B8C0BD
:109B2000833421E09207A105B10509F43DC108F095
:109B3000A5C0813421E09207A105B10509F097C0C5
:109B400061EC77E088E19DE00E94269189EF9FEF2C
:109B500044DA7EC062EB77E084E29DE00E942691C9
:109B60001092FD0C8BEF9FEFF3CF68EB77E084E270
:109B70009DE00E94269181E08093FD0C8DEF9FEF88
:109B8000E7CF6BEB77E088E19DE00E9426916BEBDD
:109B900077E084E29DE00E9426918EEF9FEFD8CF80
:109BA0006EEB77E088E19DE00E9426916EEB77E016
:109BB00084E29DE00E9426918FEF9FEFC9CF6CEC6D
:109BC00077E088E19DE00E9426916CEC77E084E2EA
:109BD0009DE00E94269180E090E0BACF6FEB77E0A5
:109BE00088E19DE00E94269181E090E0B1CF82E083
:109BF00090E0AECF83E090E0ABCF84E090E0A8CFE0
:109C000085E090E0A5CF86E090E0A2CF87E090E0ED
:109C10009FCF88E090E09CCF89E090E099CF40E032
:109C200050E064E27DE0CE0101960E943F09BE0152
:109C30006F5F7F4F88E19DE00E941091CE010196F9
:109C40000E941E9064E670E080E090E00E94F3863F
:109C500084EE9BE00E94B57C26960FB6F894DEBF9A
:109C60000FBECDBFDF91CF911F910F910895823428
:109C70009140A105B10509F48EC0E4CF853421E0FF
:109C80009207A105B10509F4A1C008F496C0A7C0C8
:109C9000813025E09207A105B10509F451CF70F498
:109CA000883421E09207A105B10509F49EC08934EA
:109CB0009140A105B10509F49BC0C4CF833025E0D4
:109CC0009207A105B10509F46FC008F464C075C01E
:109CD0008F3C20E392072FEFA207B10509F46DC076
:109CE00068F5883025E09207A105B10509F47DC02B
:109CF00070F4863025E09207A105B10509F46FC024
:109D000087309540A105B10509F46CC09BCF8F3E0B
:109D100020E192072FEFA207B10509F463C0873E47
:109D200028E192072FEFA207B10509F44FC089304F
:109D30009540A105B10509F085CF5AC0873928E6BD
:109D400092072FEFA207B10509F4FACE78F4873C09
:109D500028E392072FEFA207B10509F446C0853A20
:109D60009A45AF4FB10509F443C06CCF873628E957
:109D700092072FEFA207B10571F08F3420EB920705
:109D80002FEFA207B10581F085389A47AF4FB10593
:109D900009F058CF24C064EC77E088E19DE00E9490
:109DA000269188EF9FEFD4CE67EC77E088E19DE0C5
:109DB0000E94269187EF9FEFCBCE6AEC77E088E197
:109DC0009DE00E94269186EF9FEFC2CE6EEC77E079
:109DD00088E19DE00E94269185EF9FEFB9CE84EF48
:109DE0009FEFB6CE83EF9FEFB3CE82EF9FEFB0CE63
:109DF00081EF9FEFADCE6EE170E080E090E00E94D9
:109E0000F3864DCE8F929F92AF92BF92CF92DF9208
:109E1000EF92FF920F931F93CF93DF93CDB7DEB7EF
:109E2000A6970FB6F894DEBF0FBECDBF64ED7BE002
:109E300084EE9BE00E946A7D892BC9F00E942E2D42
:109E40000E94290C60E375E0CE0101960E94899082
:109E50004AE050E060E070E0CE0101960E94EE0919
:109E6000CE0101960E941E90A9DC0C94C06064E9AA
:109E70007BE084E29DE00E9426910E9417436AE005
:109E800070E080E090E00E94F3868091280D909130
:109E9000290D009711F40C94A160019709F046C0B8
:109EA0006EE376E0CE010F960E948990BE01615F5D
:109EB0007F4F84E29DE00E94CF9281112AC067E328
:109EC00076E0CE0109960E948990BE01675F7F4FC0
:109ED00084E29DE00E94CF92811115C06BE975E08C
:109EE000CE0101960E948990BE016F5F7F4F84E290
:109EF0009DE00E94CF9211E0811110E0CE01019609
:109F00000E941E9001C010E0CE0109960E941E9092
:109F100001C010E0CE010F960E941E90112331F077
:109F200064E27DE088E19DE00E94F3908091280D3D
:109F30009091290D0497F0F562ED77E0CE0101963E
:109F40000E948990BE016F5F7F4F84E29DE00E9476
:109F5000CF92182FCE0101960E941E90112351F12D
:109F600041E050E064E27DE0CE0109960E943F09A5
:109F7000CE0109960E940F94DC01CB014AEF5FEFFE
:109F80006FEF7FEF481B590B6A0B7B0B2AE0CE016A
:109F900001960E947F91BE016F5F7F4F88E19DE037
:109FA0000E941091CE0101960E941E90CE0109964A
:109FB0000E941E9064ED77E0CE0109960E94899080
:109FC000BE01675F7F4F84E29DE00E94CF928111C6
:109FD00016C068ED77E0CE0101960E948990BE011F
:109FE0006F5F7F4F84E29DE00E94CF9211E081116C
:109FF00001C010E0CE0101960E941E9001C011E048
:10A00000CE0109960E941E90112309F417C36BE735
:10A010007BE0CE0101960E942792CE0101960E941C
:10A02000DC0FCE0101960E941E906CED77E0CE0110
:10A0300009960E9489906EE07EE0CE0109960E940A
:10A040008292BC01CE0101960E940891CE01019638
:10A050000E94DC0FCE0101960E941E90CE0109964F
:10A060000E941E90609138027091390280913A02EC
:10A0700090913B020E94CC9520E030E048EC52E405
:10A080000E940095AB01BC0122E0CE010F960E9418
:10A09000AB9162EF77E0CE0109960E948990BE01F4
:10A0A000615F7F4FCE0109960E94829261E279E062
:10A0B0000E949392BC01CE0101960E940891CE01AC
:10A0C00001960E94DC0FCE0101960E941E90CE01E7
:10A0D00009960E941E90CE010F960E941E904091FC
:10A0E000340250913502609136027091370224E0BB
:10A0F000CE010F960E94AB9167E078E0CE01099601
:10A100000E948990BE01615F7F4FCE0109960E9437
:10A110008292BC01CE0101960E940891CE01019667
:10A120000E94DC0FCE0101960E941E90CE0109967E
:10A130000E941E90CE010F960E941E9040911E021A
:10A1400050911F02609120027091210222E0CE0105
:10A1500009960E94AB9140911602509117026091AE
:10A1600018027091190223E0CE010F960E94AB9164
:10A1700040912202509123026091240270912502A5
:10A1800022E0CE0145960E94AB9140911A02509177
:10A190001B0260911C0270911D0223E0CE0181968A
:10A1A0000E94AB9164E278E0CE014B960E948990C8
:10A1B000BE016F5D7F4FCE014B960E94829269E394
:10A1C00078E00E949392BE016B5E7F4F0E94829264
:10A1D0006CE378E00E949392BE01615F7F4F0E9422
:10A1E000829269E378E00E949392BE01675F7F4F9D
:10A1F0000E94829262E478E00E949392BC01CE01B8
:10A2000001960E940891CE0101960E94DC0FCE01BA
:10A2100001960E941E90CE014B960E941E90CE0188
:10A2200081960E941E90CE0145960E941E90CE01FE
:10A230000F960E941E90CE0109960E941E9040919A
:10A24000450250914602609147027091480223E016
:10A25000CE0109960E94AB912091490230914A02A9
:10A2600040914B0250914C0260E070E080E291E43A
:10A270000E94C397AB01BC0121E0CE0145960E942C
:10A28000D99167E478E0CE010F960E948990BE01D3
:10A290006B5E7F4FCE010F960E9482926AE578E056
:10A2A0000E949392BE01675F7F4F0E94829260E49A
:10A2B00076E00E949392BC01CE0101960E94089123
:10A2C000CE0101960E94DC0FCE0101960E941E90E5
:10A2D000CE010F960E941E90CE0145960E941E90C0
:10A2E000CE0109960E941E90409141025091420277
:10A2F000609143027091440223E0CE0109960E94CE
:10A30000AB9120913D0230913E0240913F0250912D
:10A31000400260E070E080E291E40E94C397AB01EC
:10A32000BC0121E0CE0145960E94D99160E678E01B
:10A33000CE010F960E948990BE016B5E7F4FCE01C9
:10A340000F960E9482926AE578E00E949392BE0185
:10A35000675F7F4F0E94829260E476E00E94939252
:10A36000BC01CE0101960E940891CE0101960E9487
:10A37000DC0FCE0101960E941E90CE010F960E9426
:10A380001E90CE0145960E941E90CE0109960E9415
:10A390001E9040914D0250914E0260914F0270917B
:10A3A000500222E0CE010F960E94AB9163E778E065
:10A3B000CE0109960E948990BE01615F7F4FCE0158
:10A3C00009960E94829269E878E00E949392BC010B
:10A3D000CE0101960E940891CE0101960E94DC0FE9
:10A3E000CE0101960E941E90CE0109960E941E90F9
:10A3F000CE010F960E941E904091120250911302BE
:10A40000609114027091150222E0CE010F960E9415
:10A41000AB9160E978E0CE0109960E948990BE0177
:10A42000615F7F4FCE0109960E94829260E476E0E0
:10A430000E949392BC01CE0101960E940891CE0128
:10A4400001960E94DC0FCE0101960E941E90CE0163
:10A4500009960E941E90CE010F960E941E9016E94A
:10A46000C12E14E0D12E01E010E087E1E82E8091AA
:10A47000940490919504801791070CF44FC0D60175
:10A48000AD90BD906D014AE0B501CE0109960E94E4
:10A4900054914AE0B801CE0145960E94549163EA76
:10A4A00078E0CE010F960E948990BE016B5E7F4FCF
:10A4B000CE010F960E94829267E575E00E9493920A
:10A4C000BE01675F7F4F0E9482926BEA78E00E9434
:10A4D0009392EA9CB001EB9C700D11246D577D4F57
:10A4E0000E949392BC01CE0101960E940891CE0178
:10A4F00001960E94DC0FCE0101960E941E90CE01B3
:10A500000F960E941E90CE0145960E941E90CE018D
:10A5100009960E941E900F5F1F4FA9CF80915B0C80
:10A5200090915C0C892B71F461EB78E0CE0101967F
:10A530000E948990CE0101960E94DC0FCE01019607
:10A540000E941E9080915B0C90915C0C019771F4BD
:10A5500060EC78E0CE0101960E948990CE010196D0
:10A560000E94DC0FCE0101960E941E9040910E02C7
:10A5700050910F02609110027091110222E0CE0101
:10A580000F960E94AB916AEC78E0CE0109960E948A
:10A590008990BE01615F7F4FCE0109960E94829231
:10A5A0006DEB76E00E949392BC01CE0101960E9471
:10A5B0000891CE0101960E94DC0FCE0101960E9407
:10A5C0001E90CE0109960E941E90CE010F960E9409
:10A5D0001E9040910A0250910B0260910C02709102
:10A5E0000D0222E0CE010F960E94AB916AED78E059
:10A5F000CE0109960E948990BE01615F7F4FCE0116
:10A6000009960E9482926DEB76E00E949392BC01C3
:10A61000CE0101960E940891CE0101960E94DC0FA6
:10A62000CE0101960E941E90CE0109960E941E90B6
:10A63000CE010F960E941E9010E001C011E08091A3
:10A64000280D9091290D039708F08EC00E942E2DA1
:10A650000E94290C60E375E0CE0101960E9489906A
:10A660004AE050E060E070E0CE0101960E94970A57
:10A67000CE0101960E941E908091280D9091290D87
:10A68000019739F460E070E084E29DE00E94EE9270
:10A69000F82E8091280D9091290D029709F055C050
:10A6A00062ED77E0CE0101960E948990BE016F5F56
:10A6B0007F4F84E29DE00E94CF92182FCE01019639
:10A6C0000E941E90112309F440C061E070E084E212
:10A6D0009DE00E94EE92682FCE0101960E943C916F
:10A6E000BE016F5F7F4F88E19DE00E941B91CE010C
:10A6F00001960E941E9060E070E084E29DE00E945E
:10A70000EE92F82E8091FB0C8823F9F06AEE78E047
:10A71000CE0101960E94899064E27DE0CE0101960F
:10A720000E94829260E375E00E949392BC0186ECE5
:10A730009FE00E94C68CCE0101960E941E9068E1A7
:10A740007DE086EC9FE00E94EF8C8F2D0E94A54A51
:10A750000E94C48660932A0D70932B0D80932C0D5C
:10A7600090932D0D0C94C06021E030E040E050E06B
:10A7700064E27DE0CE0101960E947093BE016F5F9E
:10A780007F4F86E09DE00E941091CE0101960E94CD
:10A790001E906DE179E0CE0109960E948990BE017C
:10A7A000675F7F4F84E29DE00E94CF92811116C0C7
:10A7B0006DEF75E0CE0101960E948990BE016F5F3A
:10A7C0007F4F84E29DE00E94CF9201E0811101C0A1
:10A7D00000E0CE0101960E941E9001C001E0CE0172
:10A7E00009960E941E90002309F4B6C042E050E092
:10A7F00064E27DE0CE0101960E943F09BE016F5FD9
:10A800007F4F86E09DE00E941091CE0101960E944C
:10A810001E9066E07DE0CE0101960E940891CE0177
:10A8200001960E94C209CE0101960E941E9086E008
:10A830009DE00E94199420E030E048EC52E40E9430
:10A8400060970E949995AB01BC01409338025093E8
:10A85000390260933A0270933B022AE0CE010196DE
:10A860000E947F91CE0101960E94C209CE010196FD
:10A870000E941E90609138027091390280913A02D4
:10A8800090913B028B019C0100591F4521403109E9
:10A8900001341C492105310588F060EF78E0CE01D4
:10A8A00001960E94899066E07DE0CE0101960E94AB
:10A8B000829263E079E00E9493926AC119821A82BF
:10A8C0001B821C821D821E821F8218860E94CC95CC
:10A8D00020E030E048EC52E40E9400958E010F5FCA
:10A8E0001F4F22E047E00E944199BC018CE09DE0AF
:10A8F0000E94269163E179E0CE0109960E94899039
:10A900006CE07DE0CE0109960E94829260E279E0DF
:10A910000E949392BC018CE09DE00E94F390CE01D6
:10A9200009960E941E9010928E0C10928D0C8091B0
:10A93000380290913902A0913A02B0913B02809383
:10A94000E50B9093E60BA093E70BB093E80B80E048
:10A9500090E00E94750925C165E279E0CE01099673
:10A960000E948990BE01675F7F4F84E29DE00E9454
:10A97000CF92811116C06BE279E0CE0101960E9460
:10A980008990BE016F5F7F4F84E29DE00E94CF926D
:10A9900001E0811101C000E0CE0101960E941E90ED
:10A9A00001C001E0CE0109960E941E90002309F427
:10A9B0006DC026E030E045E050E064E27DE0CE018D
:10A9C00001960E947093BE016F5F7F4F86E09DE00D
:10A9D0000E941091CE0101960E941E9086E09DE09B
:10A9E0000E940F946B017C0167E878E0CE01099624
:10A9F0000E948990BE01675F7F4F84E29DE00E94C4
:10AA00006793AC014F5F5F4F64E27DE0CE0101963A
:10AA10000E943F09BE016F5F7F4F86E09DE00E946C
:10AA20001091CE0101960E941E90CE0109960E94BF
:10AA30001E9086E09DE00E940F94DB01E6E9F4E0C1
:10AA400021E030E04091940450919504421753075F
:10AA50005CF0408151814A175B0711F4118210822A
:10AA60002F5F3F4F3296EECFF601EE0FFF1FEC56F1
:10AA7000FB4F7183608382E090E00E94F32B64E2DD
:10AA80007DE086EC9FE00E94EF8CB3C261E379E049
:10AA9000CE0109960E948990BE01675F7F4F84E2D4
:10AAA0009DE00E94CF92811116C067E379E0CE014C
:10AAB00001960E948990BE016F5F7F4F84E29DE006
:10AAC0000E94CF9201E0811101C000E0CE01019609
:10AAD0000E941E9001C001E0CE0109960E941E90C6
:10AAE0000023F1F0E6E9F4E081E090E020919404A5
:10AAF000309195042817390774F0863091051CF4BD
:10AB00009183808305C09C012E5F3F4F318320835A
:10AB100001963296EBCF82E090E00E94F32B69C25F
:10AB20006DE379E0CE0109960E948990BE01675FCE
:10AB30007F4F84E29DE00E94CF92811116C065E4B0
:10AB400079E0CE0101960E948990BE016F5F7F4F30
:10AB500084E29DE00E94CF9201E0811101C000E0FB
:10AB6000CE0101960E941E9001C001E0CE0109961F
:10AB70000E941E900023A1F16DE479E0CE010196C0
:10AB80000E94899068E07EE0CE0101960E94829248
:10AB9000BC018CE09DE00E94F390CE0101960E94E2
:10ABA0001E9064E077E0CE0109960E9489906CE0E7
:10ABB0007DE0CE0109960E948292BC01CE010196F1
:10ABC0000E940891CE0101960E94DC0FCE010196F1
:10ABD0000E941E90CE0109960E941E900C94C060A7
:10ABE00067E579E0CE0109960E948990BE01675F12
:10ABF0007F4F84E29DE00E94CF92811116C06EE5E6
:10AC000079E0CE0101960E948990BE016F5F7F4F6F
:10AC100084E29DE00E94CF9201E0811101C000E03A
:10AC2000CE0101960E941E9001C001E0CE0109965E
:10AC30000E941E900023B9F065E679E0CE010196EE
:10AC40000E9489906EE07EE0CE0101960E94829281
:10AC5000BC018CE09DE00E94F390CE0101960E9421
:10AC60001E900C94856064E779E0CE0109960E94FD
:10AC70008990BE01675F7F4F84E29DE00E94CF9282
:10AC8000811116C069E779E0CE0101960E94899092
:10AC9000BE016F5F7F4F84E29DE00E94CF9201E092
:10ACA000811101C000E0CE0101960E941E9001C0FA
:10ACB00001E0CE0109960E941E90002309F444C0D1
:10ACC00067E878E0CE0109960E948990BE01675F2F
:10ACD0007F4F84E29DE00E946793AC014F5F5F4F1E
:10ACE00064E27DE0CE0101960E943F09BE016F5FE4
:10ACF0007F4F86E09DE00E941091CE0101960E9458
:10AD00001E90CE0109960E941E9086E09DE00E9452
:10AD10000F946115710521F481E08093F50410C052
:10AD20006130710519F41092F5040AC062307105A2
:10AD300011F00C94C06081E08093F5041092F4044B
:10AD40000E94412D0C94C0606EE779E0CE01099617
:10AD50000E948990BE01675F7F4F84E29DE00E9460
:10AD6000CF92811116C062E879E0CE0101960E946F
:10AD70008990BE016F5F7F4F84E29DE00E94CF9279
:10AD800001E0811101C000E0CE0101960E941E90F9
:10AD900001C001E0CE0109960E941E90002309F433
:10ADA0005CC043E050E064E27DE0CE0101960E9489
:10ADB0003F09BE016F5F7F4F86E09DE00E941091CA
:10ADC000CE0101960E941E9066E07DE086EC9FE039
:10ADD0000E94EF8C10928E0C10928D0C66E07DE03C
:10ADE0008EE09EE00E94F39020E030E048E050E0EA
:10ADF00061E07CE08EE09EE00E94EF9280918D0CFD
:10AE000090918E0C0E94750966E879E0CE0101965A
:10AE10000E9489906EE07EE0CE0101960E948292AF
:10AE2000BC01CE0109960E940891CE0101960E94B4
:10AE30001E90BE01675F7F4F80E091E10E94C68C4B
:10AE400068EB7BE080E090E00E94F38661E07CE0CC
:10AE5000CE0101960E94899069C06EE879E0CE012A
:10AE600009960E948990BE01675F7F4F84E29DE052
:10AE70000E94CF92811116C063E979E0CE0101965C
:10AE80000E948990BE016F5F7F4F84E29DE00E9427
:10AE9000CF9201E0811101C000E0CE0101960E9435
:10AEA0001E9001C001E0CE0109960E941E90002371
:10AEB00009F448C044E050E064E27DE0CE01019630
:10AEC0000E943F09BE016F5F7F4F86E09DE00E94B8
:10AED0001091CE0101960E941E9068E979E0CE01A2
:10AEE00001960E94899066E07DE0CE0101960E9465
:10AEF0008292BC01CE0109960E940891CE01019672
:10AF00000E941E90BE01675F7F4F80E091E10E942A
:10AF1000C68C68EB7BE080E090E00E94F386BE0187
:10AF2000675F7F4FCE0101960E940891CE01019686
:10AF30000E94C209CE0101960E941E90CE01099680
:10AF40000C949E606FE979E0CE0109960E94899089
:10AF5000BE01675F7F4F84E29DE00E94CF92811126
:10AF600016C064EA79E0CE0101960E948990BE0184
:10AF70006F5F7F4F84E29DE00E94CF9201E08111DC
:10AF800001C000E0CE0101960E941E9001C001E0C8
:10AF9000CE0109960E941E900023A9F125E030E021
:10AFA00044E050E064E27DE0CE0101960E9470939F
:10AFB000BE016F5F7F4F86E09DE00E941091CE0141
:10AFC00001960E941E9086E09DE00E940F9470936F
:10AFD0005C0C60935B0C64E27DE0CE0101960E9404
:10AFE0000891CE0101960E94C209CE0101960E94ED
:10AFF0001E9010928E0C10928D0C80E090E00E94BA
:10B0000075090C94C06069EA79E0CE0109960E9446
:10B010008990BE01675F7F4F84E29DE00E94CF92DE
:10B02000811116C060EB79E0CE0101960E948990F3
:10B03000BE016F5F7F4F84E29DE00E94CF9201E0EE
:10B04000811101C000E0CE0101960E941E9001C056
:10B0500001E0CE0109960E941E90002321F127E015
:10B0600030E046E050E064E27DE0CE0101960E94CF
:10B070007093BE016F5F7F4F86E09DE00E9410914C
:10B08000CE0101960E941E9086E09DE00E940F94E2
:10B09000672B21F41092FB0C0C94926081E080935A
:10B0A000FB0C0C94926067EB79E0CE010F960E9446
:10B0B0008990BE01615F7F4F84E29DE00E94CF9244
:10B0C00081112BC06AEB79E0CE0109960E9489902C
:10B0D000BE01675F7F4F84E29DE00E94CF928111A5
:10B0E00016C06DEB79E0CE0101960E948990BE01F9
:10B0F0006F5F7F4F84E29DE00E94CF9201E081115B
:10B1000001C000E0CE0101960E941E9001C001E046
:10B11000CE0109960E941E9001C001E0CE010F965B
:10B120000E941E90002309F42DC1FAE0AF2EB12C2D
:10B13000C12CD12C760188248A94A3E09A2E6EE14A
:10B1400070E080E090E00E94F386809181020E948E
:10B150008987B4010E949098882777FD8095982F61
:10B160000E94CC9520E030E040EA50E40E946097D5
:10B170009B01AC01C701B6010E9436946B017C01B2
:10B18000E1E0AE1AB108D9F620E030E040E251E447
:10B190000E9400956B017C0160EC79E0CE0109967C
:10B1A0000E948990BE01675F7F4F84E29DE00E940C
:10B1B000CF92811116C064EC79E0CE0101960E9415
:10B1C0008990BE016F5F7F4F84E29DE00E94CF9225
:10B1D00001E0811101C000E0CE0101960E941E90A5
:10B1E00001C001E0CE0109960E941E90002309F4DF
:10B1F0003FC020E030E040E650E4C701B6010E94C5
:10B2000060979B01AC0160E070E080E890E40E94F0
:10B210003594AB01BC0140932A0250932B026093FA
:10B220002C0270932D0222E0CE0101960E94AB9178
:10B23000BE016F5F7F4F8CE09DE00E941091CE01B8
:10B2400001960E941E9068EC79E0CE0101960E9462
:10B2500089906CE07DE0CE0101960E948292BC0153
:10B260008CE09DE00E94F390CE0101960E941E901A
:10B2700067ED79E0CE0109960E948990BE01675F73
:10B280007F4F84E29DE00E94CF92811116C06CED49
:10B2900079E0CE0101960E948990BE016F5F7F4FD9
:10B2A00084E29DE00E94CF9201E0811101C000E0A4
:10B2B000CE0101960E941E9001C001E0CE010996C8
:10B2C0000E941E90002309F43FC020E030E040E6D9
:10B2D00050E4C701B6010E9460979B01AC0160E099
:10B2E00070E080E291E40E943594AB01BC01409390
:10B2F000260250932702609328027093290222E0CD
:10B30000CE0101960E94AB91BE016F5F7F4F8CE032
:10B310009DE00E941091CE0101960E941E9061EE68
:10B3200079E0CE0101960E9489906CE07DE0CE012B
:10B3300001960E948292BC018CE09DE00E94F390F5
:10B34000CE0101960E941E9064E077E0CE0109963E
:10B350000E9489906CE07DE0CE0109960E94829265
:10B36000BC01CE0101960E940891CE0101960E9477
:10B37000DC0FCE0101960E941E90CE0109960E941C
:10B380001E90CEC661EF79E0CE0101960E948990B1
:10B39000BE016F5F7F4F84E29DE00E94CF92082F35
:10B3A000CE0101960E941E90002309F46EC0809188
:10B3B000280D9091290D079708F4B2C646E050E099
:10B3C00064E27DE0CE0101960E943F09BE016F5FFD
:10B3D0007F4F86E09DE00E941091CE0101960E9471
:10B3E0001E9086E09DE00E941994AB01BC01409341
:10B3F0000E0250930F02609310027093110221E02D
:10B40000CE0109960E94AB916AEC78E0CE010196DC
:10B410000E948990BE01675F7F4FCE0101960E9416
:10B4200082926DEB76E00E949392BC018CE09DE0ED
:10B430000E94F390CE0101960E941E90CE010996C3
:10B440000E941E906CE07DE0CE0101960E94089162
:10B45000CE0101960E94DC0FCE0101960E941E9043
:10B460000E94C48628EE33E040E050E00E94A3989A
:10B47000CA01B9010E94CA956093610C7093620C75
:10B480008093630C9093640C4BC668EF79E0CE0117
:10B4900001960E948990BE016F5F7F4F84E29DE01C
:10B4A0000E94CF92082FCE0101960E941E90002389
:10B4B000E9F18091280D9091290D079708F430C685
:10B4C00046E050E064E27DE0CE0101960E943F0933
:10B4D000BE016F5F7F4F86E09DE00E941091CE011C
:10B4E00001960E941E9086E09DE00E941994AB0197
:10B4F000BC0140930A0250930B0260930C027093BC
:10B500000D0221E0CE0109960E94AB916AED78E030
:10B51000CE0101960E948990BE01675F7F4FCE01E8
:10B5200001960E9482926DEB76E0F5C16FEF79E0B3
:10B53000CE0109960E948990BE01675F7F4F84E229
:10B540009DE00E94CF92811116C063E07AE0CE01A7
:10B5500001960E948990BE016F5F7F4F84E29DE05B
:10B560000E94CF9201E0811101C000E0CE0101965E
:10B570000E941E9001C001E0CE0109960E941E901B
:10B58000002309F45AC08091C2049091C3040E9420
:10B59000D12460931A0270931B0280931C02909333
:10B5A0001D026093F90B7093FA0B8093FB0B909341
:10B5B000FC0B80E090E0A0E8BFE380932202909330
:10B5C0002302A0932402B09325028093F10B909361
:10B5D000F20BA093F30BB093F40B8091FB0C882338
:10B5E000A1F06FE57BE086EC9FE00E94A38C409188
:10B5F0001A0250911B0260911C0270911D0222E000
:10B6000030E086EC9FE00E94F88E10928E0C109233
:10B610008D0C80E090E00E94750940911A025091D3
:10B620001B0260911C0270911D0222E0CE0109965E
:10B630000E94AB9167E07AE050C560E17AE0CE010C
:10B6400009960E948990BE01675F7F4F84E29DE06A
:10B650000E94CF92811116C066E17AE0CE01019678
:10B660000E948990BE016F5F7F4F84E29DE00E943F
:10B67000CF9201E0811101C000E0CE0101960E944D
:10B680001E9001C001E0CE0109960E941E90002389
:10B6900009F469C08091280D9091290D0797F8F061
:10B6A00046E050E064E27DE0CE0101960E943F0951
:10B6B000BE016F5F7F4F86E09DE00E941091CE013A
:10B6C00001960E941E9086E09DE00E94199460936E
:10B6D0004D0270934E0280934F02909350028091DE
:10B6E000BC040E94B62B80914D0290914E02A09115
:10B6F0004F02B09150028093190C90931A0CA093B2
:10B700001B0CB0931C0C8091FB0C8823A1F06DE402
:10B710007BE086EC9FE00E94A38C40914D0250910B
:10B720004E0260914F027091500222E030E086ECB0
:10B730009FE00E94F88E10928E0C10928D0C80E08B
:10B7400090E00E94750940914D0250914E02609127
:10B750004F027091500222E0CE0109960E94AB91F7
:10B760006CE17AE0BAC466E27AE0CE0109960E9402
:10B770008990BE01675F7F4F84E29DE00E94CF9277
:10B78000811116C06BE27AE0CE0101960E94899089
:10B79000BE016F5F7F4F84E29DE00E94CF9201E087
:10B7A000811101C000E0CE0101960E941E9001C0EF
:10B7B00001E0CE0109960E941E90002309F4AEC05C
:10B7C0008091280D9091290D069708F145E050E0F1
:10B7D00064E27DE0CE0101960E943F09BE016F5FE9
:10B7E0007F4F86E09DE00E941091CE0101960E945D
:10B7F0001E9086E09DE00E9419940E94E29660935C
:10B80000490270934A0280934B0290934C028091BC
:10B81000BE049091BF040E94642820E030E048E01C
:10B8200051E40E9400956093450270934602809314
:10B830004702909348026093090C70930A0C80931E
:10B840000B0C90930C0C8091490290914A02A091AC
:10B850004B02B0914C028093110C9093120CA09368
:10B86000130CB093140C8091FB0C882381F16CE3D2
:10B870007BE086EC9FE00E94A38C209149023091EE
:10B880004A0240914B0250914C0260E070E080E22D
:10B8900091E40E94C397AB01BC0121E030E086EC4B
:10B8A0009FE00E94F78E60E37AE086EC9FE00E94C2
:10B8B000D48C4091450250914602609147027091AC
:10B8C000480222E030E086EC9FE00E94F88E109261
:10B8D0008E0C10928D0C80E090E00E9475094091D2
:10B8E000450250914602609147027091480223E060
:10B8F000CE0109960E94AB9167E37AE0CE010196F2
:10B900000E948990BE01675F7F4FCE0101960E9421
:10B91000829267E176E00E949392EAC360E47AE063
:10B92000CE0109960E948990BE01675F7F4F84E235
:10B930009DE00E94CF92811116C065E47AE0CE01AD
:10B9400001960E948990BE016F5F7F4F84E29DE067
:10B950000E94CF9201E0811101C000E0CE0101966A
:10B960000E941E9001C001E0CE0109960E941E9027
:10B97000002309F491C08091280D9091290D06971C
:10B9800008F145E050E064E27DE0CE0101960E94BE
:10B990003F09BE016F5F7F4F86E09DE00E941091DE
:10B9A000CE0101960E941E9086E09DE00E941994AF
:10B9B0000E94E29660933D0270933E0280933F02A4
:10B9C000909340028091BE049091BF040E9464282D
:10B9D00020E030E048E051E40E940095609341028D
:10B9E00070934202809343029093440260930D0C43
:10B9F00070930E0C80930F0C9093100C20913D02CD
:10BA000030913E0240913F02509140022093150C2C
:10BA10003093160C4093170C5093180C8091FB0C2C
:10BA2000882311F160E070E080E291E40E94C39706
:10BA3000AB01BC0121E030E086EC9FE00E94F78E74
:10BA400060E37AE086EC9FE00E94D48C4091410252
:10BA500050914202609143027091440222E030E032
:10BA600086EC9FE00E94F88E10928E0C10928D0C46
:10BA700080E090E00E94750940914102509142029D
:10BA8000609143027091440223E0CE0109960E9426
:10BA9000AB916AE47AE032CF63E57AE0CE010996B1
:10BAA0000E948990BE01675F7F4F84E29DE00E9403
:10BAB000CF92811116C067E57AE0CE0101960E940F
:10BAC0008990BE016F5F7F4F84E29DE00E94CF921C
:10BAD00001E0811101C000E0CE0101960E941E909C
:10BAE00001C001E0CE0109960E941E90002309F4D6
:10BAF0006FC060E08091C8040E94028809E110E0F4
:10BB0000C12CD12C76018091C8040E948987BC0188
:10BB1000882777FD8095982F0E94CC959B01AC01DA
:10BB2000C701B6010E9436946B017C016AE070E0A7
:10BB300080E090E00E94F3860150110921F720E097
:10BB400030E040EA50E4C701B6010E94609720E06F
:10BB500030E040E85AE30E94609720E030E048EC93
:10BB600051E40E9400956093120270931302809337
:10BB700014029093150260932F0C7093300C8093F5
:10BB8000310C9093320C10928E0C10928D0C80E040
:10BB900090E00E9475094091120250911302609149
:10BBA00014027091150222E0CE0109960E94AB9119
:10BBB00060E978E0CE0101960E948990BE01675F3E
:10BBC0007F4FCE0101960E94829260E476E0A3CE80
:10BBD0006BE57AE0CE0109960E948990BE01675F0D
:10BBE0007F4F84E29DE00E94CF92811116C06FE5E5
:10BBF0007AE0CE0101960E948990BE016F5F7F4F6F
:10BC000084E29DE00E94CF9201E0811101C000E03A
:10BC1000CE0101960E941E9001C001E0CE0109965E
:10BC20000E941E90002309F473C026E030E044E037
:10BC300050E064E27DE0CE0101960E947093BE0167
:10BC40006F5F7F4F86E09DE00E941091CE010196CC
:10BC50000E941E9086E09DE00E940F946B017C0183
:10BC600067E878E0CE0109960E948990BE01675F7F
:10BC70007F4F84E29DE00E946793AC014F5F5F4F6E
:10BC800064E27DE0CE0101960E943F09BE016F5F34
:10BC90007F4F86E09DE00E941091CE0101960E94A8
:10BCA0001E90CE0109960E941E900091E204109110
:10BCB000E30486E09DE00E941994AB01BC01980169
:10BCC000C6010E94E72FE5E6FCE023E33CE041915A
:10BCD000519161917191D9014D935D936D937D93D4
:10BCE0009D01BCE0ED38FB0791F710928E0C10928D
:10BCF0008D0C80E090E00E94750944E050E064E221
:10BD00007DE0CE0109960E943F0963E67AE0E5C135
:10BD100064E87AE0CE0109960E948990BE01675FCF
:10BD20007F4F84E29DE00E94CF92811116C068E8A7
:10BD30007AE0CE0101960E948990BE016F5F7F4F2D
:10BD400084E29DE00E94CF9201E0811101C000E0F9
:10BD5000CE0101960E941E9001C001E0CE0109961D
:10BD60000E941E90002309F44EC08091C20490915D
:10BD7000C3040E94D124AB01BC014093160250932E
:10BD8000170260931802709319024093FD0B5093B1
:10BD9000FE0B6093FF0B7093000C80E090E5A3EC2A
:10BDA000B7E480931E0290931F02A0932002B093E9
:10BDB00021028093F50B9093F60BA093F70BB093B1
:10BDC000F80B8091FB0C882331F022E030E086EC08
:10BDD0009FE00E94F88E10928E0C10928D0C80E0E5
:10BDE00090E00E94750940911602509117026091EF
:10BDF00018027091190222E0CE0109960E94AB91BF
:10BE00006CE87AE06AC167E97AE0CE0109960E949F
:10BE10008990BE01675F7F4F84E29DE00E94CF92D0
:10BE2000811116C06BE97AE0CE0101960E948990DB
:10BE3000BE016F5F7F4F84E29DE00E94CF9201E0E0
:10BE4000811101C000E0CE0101960E941E9001C048
:10BE500001E0CE0109960E941E90002309F47EC0E5
:10BE60008091280D9091290D0497F8F044E050E05E
:10BE700064E27DE0CE0101960E943F09BE016F5F42
:10BE80007F4F86E09DE00E941091CE0101960E94B6
:10BE90001E9086E09DE00E941994609322027093A8
:10BEA0002302809324029093250240912202509114
:10BEB000230260912402709125024093F10B50936C
:10BEC000F20B6093F30B7093F40B8091FB0C8823BF
:10BED00031F022E030E086EC9FE00E94F78E809106
:10BEE000C2049091C3040E94D12460931A027093FB
:10BEF0001B0280931C0290931D026093F90B7093B8
:10BF0000FA0B8093FB0B9093FC0B8091FB0C882326
:10BF1000A1F062E37BE086EC9FE00E94A38C40915D
:10BF20001A0250911B0260911C0270911D0222E0C6
:10BF300030E086EC9FE00E94F88E10928E0C1092FA
:10BF40008D0C80E090E00E94750940911A0250919A
:10BF50001B0260911C0270911D02B8C067EA7AE072
:10BF6000CE0109960E948990BE01675F7F4F84E2EF
:10BF70009DE00E94CF92811116C06BEA7AE0CE015B
:10BF800001960E948990BE016F5F7F4F84E29DE021
:10BF90000E94CF9201E0811101C000E0CE01019624
:10BFA0000E941E9001C001E0CE0109960E941E90E1
:10BFB000002309F4B5C08091280D9091290D0497B4
:10BFC000F8F044E050E064E27DE0CE0101960E948A
:10BFD0003F09BE016F5F7F4F86E09DE00E94109198
:10BFE000CE0101960E941E9086E09DE00E94199469
:10BFF00060931E0270931F0280932002909321028F
:10C0000080911E0290911F02A0912002B091210206
:10C010008093F50B9093F60BA093F70BB093F80B6E
:10C020008091FB0C8823A1F069E17BE086EC9FE026
:10C030000E94A38C40911E0250911F026091200229
:10C040007091210222E030E086EC9FE00E94F78EA2
:10C050008091C2049091C3040E94D124609316027F
:10C060007093170280931802909319026093FD0B4E
:10C070007093FE0B8093FF0B9093000C8091FB0C50
:10C080008823A1F06FE07BE086EC9FE00E94A38C08
:10C090004091160250911702609118027091190296
:10C0A00022E030E086EC9FE00E94F88E10928E0C29
:10C0B00010928D0C80E090E00E947509409116026C
:10C0C00050911702609118027091190222E0CE017E
:10C0D00009960E94AB916FE97AE0CE0101960E9429
:10C0E0008990BE01675F7F4FCE0101960E948292C8
:10C0F000BC018CE09DE00E94F390CE0101960E946D
:10C100001E90CE0109960E941E906CE07DE0CE014B
:10C1100001960E940891CE0101960E94DC0F0CC08E
:10C12000112371F164E27DE0CE0101960E94089135
:10C13000CE0101960E94C209CE0101960E941E9076
:10C140001FC08EE89DE00E94F77A182F882319F10E
:10C1500064E97BE088E19DE00E9426918091FB0CE0
:10C16000882359F06FEA7AE086EC9FE00E94D48C35
:10C17000612F86EC9FE00E940F8D812F0E94A54ABF
:10C180000E94C48660932A0D70932B0D80932C0D12
:10C1900090932D0D49C08091FD0C882309F44FC068
:10C1A0000E94C486E8EECE2EE3E0DE2EE12CF12CD8
:10C1B000A70196010E94A398CA01B9010E94CA95DD
:10C1C0002091610C3091620C4091630C5091640C91
:10C1D0000E94359420910E0230910F02409110027E
:10C1E000509111020E94A19618164CF50E94C48627
:10C1F000A70196010E94A398CA01B9010E94CA959D
:10C200006093610C7093620C8093630C9093640C48
:10C210008091F70C9091F80C0E94ED4764E170E07A
:10C2200080E090E00E94F3868091FD0C8823E9F085
:10C2300064E670E080E090E00E94F38616C00E9401
:10C24000C486C0902A0DD0902B0DE0902C0DF0905C
:10C250002D0D6C197D098E099F0968347E4E81056C
:10C26000910510F30E943A2DDFCFA6960FB6F894F1
:10C27000DEBF0FBECDBFDF91CF911F910F91FF9019
:10C28000EF90DF90CF90BF90AF909F908F900895E8
:10C290000895CF92DF92EF92FF92FC0185899689F3
:10C2A000481B590B61097109A389B4899A01AB0133
:10C2B0000E94E7986B017C018FE0F594E794D79496
:10C2C000C7948A95D1F765857685882777FD80950F
:10C2D000982F2BE0660F771F881F991F2A95D1F79B
:10C2E00027853089442737FD4095542F2C0D3D1D5F
:10C2F0004E1D5F1D0E94C5982C0D3D1D4E1D5F1DDE
:10C30000CA01B901FF90EF90DF90CF9008951F937D
:10C31000CF93DF931F92CDB7DEB7162F67E770E09C
:10C320008CE29EE049830E94F56B612F8CE29EE0D7
:10C330000E94A46B4981642F8CE29EE00E94A46B52
:10C340008CE29EE00F90DF91CF911F910C94696C6D
:10C35000CF93C62F67E770E08CE29EE00E94F56BFA
:10C360006C2F8CE29EE00E94A46B8CE29EE00E9407
:10C37000696C67E770E08CE29EE00E94F56B41E03B
:10C3800050E067E770E08CE29EE00E94676C8CE210
:10C390009EE00E94556BC82F8CE29EE00E94696C63
:10C3A0008C2FCF910895CF93DF93C62F67E770E06E
:10C3B0008CE29EE00E94F56B6C2F8CE29EE00E9466
:10C3C000A46B8CE29EE00E94696C67E770E08CE2EF
:10C3D0009EE00E94F56B42E050E067E770E08CE27F
:10C3E0009EE00E94676C8CE29EE00E94556BD82F05
:10C3F00080E0C82F8CE29EE00E94556BC82BD92BA1
:10C400008CE29EE00E94696CCE01DF91CF9108958D
:10C41000CF93DF93EC01643008F063E068838CE233
:10C420009EE00E94E26B60EDCE0192DF853509F05F
:10C4300039C06AEACE01B7DF9A8389836CEACE01FC
:10C44000B2DF9C838B836EEACE01ADDF9E838D834A
:10C4500060EBCE01A8DF9A8B898B62EBCE01A3DF64
:10C460009C8B8B8B64EBCE019EDF9E8B8D8B66EB62
:10C47000CE0199DF98878F8368EBCE0194DF9A878E
:10C4800089876AEBCE018FDF9C878B876CEBCE01AF
:10C490008ADF9E878D876EEBCE0185DF988B8F8735
:10C4A00081E001C080E0DF91CF910895CF93DF93C9
:10C4B000EC014EE264EF2BDF65E070E080E090E09D
:10C4C0000E94F38666EFCE01DF91CF916CCFCF93C0
:10C4D000DF93EC01EBDFAC0160E070E0CE01D9DE70
:10C4E000685F7F4F8F4F9F4F34E095958795779585
:10C4F00067953A95D1F70E94CC9520E030E040E274
:10C5000051E40E940095DF91CF910895CF92DF9280
:10C51000EF92FF92CF93DF93EC0148814295440F55
:10C52000440F407C4C5C64EFF2DE8881811105C0D1
:10C5300065E070E080E090E012C0813029F468E0AE
:10C5400070E080E090E00BC0823029F46EE070E093
:10C5500080E090E004C06AE170E080E090E00E943A
:10C56000F38666EFCE011FDF6C01E12CF12CFE2C6F
:10C57000ED2CDC2CCC2468EFCE01EADEA70196017D
:10C58000282BCA01B901488128E030E0241B310979
:10C5900004C096958795779567952A95D2F7DF9190
:10C5A000CF91FF90EF90DF90CF9008952F923F9220
:10C5B0004F925F926F927F928F929F92AF92BF92B3
:10C5C000CF92DF92EF92FF920F931F93CF93DF935F
:10C5D000CDB7DEB72A970FB6F894DEBF0FBECDBF3A
:10C5E0009A87898763DF8C0189859A858FDF6D83C0
:10C5F0007E838F839887A80160E070E089859A85A3
:10C6000048DE4B015C0180EA881A8FE0980AA10895
:10C61000B108A5019401C501B4010E946D982B01D8
:10C620003C010CE075946794579447940A95D1F7B0
:10C63000A985BA8511962D903C9012971C9115965C
:10C640000D90BC91A02D0E94F1986B017C018DE0B2
:10C65000F594E794D794C7948A95D1F7E985FA853C
:10C66000A781B085A30192010E94F198BB2797FD95
:10C67000B095AB2FC80ED91EEA1EFB1EF2E0CF0EFE
:10C68000D11CE11CF11C32E0F594E794D794C794D7
:10C690003A95D1F780E8D80EE11CF11CE985FA85BE
:10C6A000A189B289A70196010E94E798DC01CB011C
:10C6B0004FE0B695A795979587954A95D1F78983C9
:10C6C0009A83AB83BC836101EE24D7FCE094FE2CFB
:10C6D00052E0CC0CDD1CEE1CFF1C5A95D1F7A18555
:10C6E000B285A30192010E94F1982B013C016BE0FD
:10C6F00075946794579447946A95D1F7A381B48150
:10C70000A50194010E94F198EBE0959587957795A6
:10C710006795EA95D1F7460E571E681E791EC40C20
:10C72000D51CE61CF71C012E04C0CC0CDD1CEE1C35
:10C73000FF1C0A94D2F792E0C90ED11CE11CF11C37
:10C74000C701B60124E030E040E050E00E94C59807
:10C750008D819E81AF81B885821B930BA40BB50B95
:10C760009C01AD0160E573EC80E090E004C096951B
:10C770008795779567951A95D2F70E946D9897FDE2
:10C780000DC0660F771F881F991F29813A814B8141
:10C790005C810E94A39849015A010CC029813A8109
:10C7A0004B815C810E94A39849015A01880C991C15
:10C7B000AA1CBB1C9927B7FC9A958B2D7A2D692D45
:10C7C0009B01AC010E946D989B01AC01AEEDBBE0FA
:10C7D0000E94E7986C01FF24D7FCF094EF2CA3E4AF
:10C7E000B3EEA50194010E94F398BB2797FDB09585
:10C7F000AB2FC80ED91EEA1EFB1E9FECC90E9EE091
:10C80000D91EE11CF11CA4E0F594E794D794C794D9
:10C81000AA95D1F7C80CD91CEA1CFB1CC701B601AC
:10C820002A960FB6F894DEBF0FBECDBFDF91CF9131
:10C830001F910F91FF90EF90DF90CF90BF90AF903E
:10C840009F908F907F906F905F904F903F902F9030
:10C8500008958F929F92AF92BF92CF92DF92EF9204
:10C86000FF92CF93DF9300D01F92CDB7DEB74A017E
:10C870005B019CDE6B017C0120E03AE24DE257E473
:10C88000C501B4010E9400959B01AC0160E070E01D
:10C8900080E89FE30E94359426EF38E248EA50E4AE
:10C8A0000E94C3979B01AC01C701B60129833A835B
:10C8B0004B835C830E94CC9529813A814B815C81BA
:10C8C0000E9400950E9499950F900F900F900F90E5
:10C8D000DF91CF91FF90EF90DF90CF90BF90AF901E
:10C8E0009F908F900895CF93DF9300D01F92CDB784
:10C8F000DEB79A01AB0129833A834B835C8356DE12
:10C900000E94CC9529813A814B815C810E940095DF
:10C9100021E03EED42E45EE30E94C3979B01AC013F
:10C9200060E070E080E89FE30E94359420E03AE206
:10C930004DE257E40E9460970F900F900F900F9078
:10C94000DF91CF9108953F924F925F926F927F92C5
:10C950008F929F92AF92BF92CF92DF92EF92FF920F
:10C960000F931F93CF93DF9300D01F921F92CDB7E9
:10C97000DEB75C01562E19821A821B821C821D8230
:10C9800061E0852D0E94028860E0852D0E943B8831
:10C9900062E170E080E090E00E94F38661E0852D26
:10C9A0000E943B8888E290E00E94198760E0852D14
:10C9B0000E94028801E117E2852D0E947088892B70
:10C9C00031F401501109C1F78EEF9FEF6EC001E104
:10C9D00017E2852D0E947088019721F401501109FA
:10C9E000C1F7F2CF08E210E0312C37E0432E882463
:10C9F0008394912C21E1E22E27E2F22E852D0E94D4
:10CA00007088892B29F481E0E81AF108B9F7DCCFA6
:10CA10000E94D0866B017C0191E1692E97E2792E0C
:10CA2000852D0E947088019729F4E1E06E1A710843
:10CA3000B9F7CACF0E94D0866C197D098E099F096B
:10CA4000693271058105910578F0E1E0F0E0EC0FC5
:10CA5000FD1FE30DF11D2081C401042C01C0880FCE
:10CA60000A94EAF7282B2083411004C0339487E00E
:10CA7000482E01C04A940150110909F0BBCF298109
:10CA8000822F90E0F501918380833B81832F90E09A
:10CA900093838283230F81E090E03D81321302C0B3
:10CAA00080E090E09195819591090F900F900F9003
:10CAB0000F900F90DF91CF911F910F91FF90EF900A
:10CAC000DF90CF90BF90AF909F908F907F906F90AE
:10CAD0005F904F903F900895FC011382128281E491
:10CAE0009BE091838083148260874187228788E05E
:10CAF00083870895FF920F931F93CF93DF938C0149
:10CB00008CE29EE05FD663EC7AE086EC9FE00E94C8
:10CB1000FF8CC0E0D0E087E2F82E6F2D8CE29EE023
:10CB20005AD68CE29EE0D5D681111EC06FEC7AE019
:10CB300086EC9FE00E94D48C40E150E06F2D86ECA3
:10CB40009FE00E94F78DF801F4826BEE7AE086ECAC
:10CB50009FE00E94D48C40E150E06F2D86EC9FE076
:10CB60000E94F78D21960FC0843069F465E07BE068
:10CB700086EC9FE00E94D48C40E150E06F2D86EC63
:10CB80009FE00E94F78DF394F0E4FF12C6CFCD2B07
:10CB900019F460E27BE002C066E37BE086EC9FE094
:10CBA000DF91CF911F910F91FF900C94FF8C1F93F9
:10CBB000CF93DF93EC01162F6C818CE29EE00BD6B5
:10CBC000E0912C0EF0912D0E6B85612B0190F08180
:10CBD000E02D8CE29EE019958CE29EE0DF91CF91F2
:10CBE0001F9177C6FC01138660E0E1CF28E0FC01CD
:10CBF000238760E0DCCF1F93CF93DF93EC01162FE8
:10CC00006460D5DF81E090E00E941987612F6B7F1F
:10CC1000CE01CDDF82E390E0DF91CF911F910C94A4
:10CC200019871F93CF93DF93EC01162FC0DF612F7D
:10CC3000CE01DF91CF911F91DECFEF92FF921F9334
:10CC4000CF93DF931F92CDB7DEB77C01162F607FA5
:10CC5000642B4983E6DF80E1189FB00111244981EC
:10CC6000642BC7010F90DF91CF911F91FF90EF9040
:10CC7000D8CF40E0E2CF61E0FCDF80ED97E00C949C
:10CC8000198762E0F6DF80ED97E00C941987CF9367
:10CC9000DF93CDB7DEB728970FB6F894DEBF0FBE8F
:10CCA000CDBF28E0E2E0F5E0DE01119601900D92A3
:10CCB0002A95E1F7FC012185241710F44FEF420F6C
:10CCC000FE013196E40FF11DE40FF11D2081260FC6
:10CCD0002068622F28960FB6F894DEBF0FBECDBF36
:10CCE000DF91CF91C6CFFC0166816B7F6683686060
:10CCF000C0CFFC016681262F246026836C60B9CFEB
:10CD0000CF92DF92EF92FF920F931F93CF93DF9317
:10CD10001F921F92CDB7DEB78C01677088E0689FC5
:10CD2000B00111246064C80149835A83A2DF49819C
:10CD3000C42E5A81D52EE12CF12CD6016D916D01B6
:10CD4000D801ED91FC910190F081E02DC801199579
:10CD5000BFEFEB1AFB0AE8E0EE16F10471F70F9053
:10CD60000F90DF91CF911F910F91FF90EF90DF9087
:10CD7000CF90089541E061DF81E090E00895CF9386
:10CD8000DF93EC018CE29EE01DD51D828985823007
:10CD900010F098E09D839A85992329F0813019F449
:10CDA0008D8184608D8362E370E080E090E00E947A
:10CDB000F3866B85CE01FBDE68EE73E080E090E0E9
:10CDC0000E94F38660E3CE012CDF84E991E10E94AA
:10CDD000198760E3CE0125DF84E991E10E9419877C
:10CDE00060E3CE011EDF86E990E00E94198760E2D1
:10CDF000CE0117DF6D816062CE013BDF84E08E8360
:10CE0000CE0177DFCE0137DF82E08F8366E0CE018F
:10CE100030DFCE01DF91CF9134CFFF920F931F937C
:10CE2000CF93DF93FC010081C181D281F894898185
:10CE3000F02EF0948F21898378941DE7115029F109
:10CE400082E090E00E94198788818023B9F3F894EA
:10CE50008A818F218A838981802B8983789480EECF
:10CE600091E00E941987F89489818F21898386E453
:10CE700090E00E9419878881802311E009F010E07A
:10CE800078948AE991E00E941987812FDF91CF91F0
:10CE90001F910F91FF9008951F93CF93DF93FC0193
:10CEA0001081C181D281912F909560FF12C0F894BA
:10CEB0008A8189238A838981812B89838AE090E012
:10CEC0000E9419878A81812B8A83789487E390E076
:10CED00011C0F8948A8189238A838981812B89836F
:10CEE00081E490E00E9419878A81812B8A8378945B
:10CEF00085E090E0DF91CF911F910C9419870F93FB
:10CF00001F93CF93DF93FC011081C181D281F894EC
:10CF10008981812B89838A81012F009580238A83CF
:10CF200083E090E00E9419878981802389838AE0C9
:10CF300090E00E941987C881789485E390E00E9470
:10CF400019871C2381E009F480E0DF91CF911F91C4
:10CF50000F910895CF92DF92EF92FF920F931F935C
:10CF6000CF93DF931F92CDB7DEB76C01E62E08E0BA
:10CF700010E0FF24F39461E09F2D9E2109F460E00E
:10CF8000C601498389DFFF0C015011094981011550
:10CF9000110589F7411115C0F894D6011196ED914C
:10CFA000FC91129791818C918095892381831196B0
:10CFB000ED91FC91129792818C91809589238283C7
:10CFC00078940F90DF91CF911F910F91FF90EF9088
:10CFD000DF90CF900895EF92FF920F931F93CF931E
:10CFE000DF938C01C8E0D0E0F12CEE24E394C8017B
:10CFF00086DF8111FE28EE0C2197C9F78F2DDF9176
:10D00000CF911F910F91FF90EF900895CF92DF92F3
:10D01000FF920F931F93CF93DF931F92CDB7DEB78D
:10D020008C01F62E40E065E5798394DFCF2C798181
:10D03000D72E88E0F82EF60161916F0140E0C8011B
:10D0400089DFFA94C1F70F90DF91CF911F910F9173
:10D05000FF90DF90CF90089540E06CEC7BCFFC0117
:10D0600013861586148627E030E0DF01A20FB31F78
:10D0700013961C922115310519F021503109F5CF75
:10D0800008951F93CF93DF93EC01162F60E0812F5B
:10D090000E940288612F70E0FB01E555F34FE49197
:10D0A000E883FB01EF50F34FE491F0E0EE0FFF1F38
:10D0B000E95CF24F859194919A838983CE01DF9147
:10D0C000CF911F91CCCFAF92BF92CF92DF92EF92D0
:10D0D000FF920F931F93CF93DF931F92CDB7DEB7CD
:10D0E0005C01D62EE72EFC01158511115EC0498327
:10D0F00094DE4981811105C0F501138615861486D9
:10D100006DC0442319F040E060EF02C040E06CEED7
:10D11000C50120DF01E0F12CC12C11E0C501EFDEDB
:10D12000682FC5016983EBDE6981613019F48130B4
:10D13000B9F432C02F2D30E068131BC0F501838590
:10D14000181730F4E20FF31F8381802349F402C0E3
:10D15000181731F060E0193058F4F501148708C051
:10D16000F501EF0DF11D8381802B838361E009C000
:10D17000C12EF501E20FF31F8381902F9095892333
:10D180008383C50189DE1F5F000F11F4F39401E072
:10D19000F7E0FF1508F0C2CF113438F0F501C3866F
:10D1A000C11009C081E0858706C0F5011386158688
:10D1B000148610E013C0F50183818823B1F3ED2DAF
:10D1C000FE2D80E090E0D501A80FB91F13962C9199
:10D1D0002193019688309105B1F711E0812F0F90CE
:10D1E000DF91CF911F910F91FF90EF90DF90CF9043
:10D1F000BF90AF900895DC0180E0615088F09D9170
:10D200009827E92FEF70F0E0EB5BF34F24919295B4
:10D210009F70E92FF0E0EB5AF34F84918227EDCF16
:10D22000089529EB3AE0FC0131832083089529EB2E
:10D230003AE0FC01318320830C9433940F931F93C5
:10D24000CF93DF938C01EB0188E2FB0111928A9569
:10D25000E9F74BE050E065E47BE0CE010E94CF9B14
:10D260001B8641E050E060E070E04C875D876E8790
:10D270007F87F801458956896789708D488B598B5E
:10D280006A8B7B8B42E050E060E070E04C8B5D8B02
:10D290006E8B7F8B1CA21DA21EA21FA240E050E03D
:10D2A00068E474E4488F598F6A8F7B8F40E050E0C8
:10D2B00068E474EC4C8F5D8F6E8F7F8F4DEC5CEC6F
:10D2C0006CE47EE348A359A36AA37BA3DF91CF91CB
:10D2D0001F910F91089521E53BE0FC0131832083EC
:10D2E000458B568B678B708F0895CF93DF931F927A
:10D2F0001F92CDB7DEB78CE29EE02A8349836BD2C2
:10D300004981642F8CE29EE01FD22A81622F8CE239
:10D310009EE01AD28CE29EE00F900F90DF91CF91A9
:10D32000D8C20F931F93CF93DF938C01EB01262F6D
:10D3300041E06EE1DADFF801D483C383C038D10560
:10D3400009F45BC0DCF4C034D105A9F1C036D105C5
:10D3500009F442C0A09709F08AC080E090E8A9E8EB
:10D36000B4E48093FD049093FE04A093FF04B09373
:10D37000000580E090E0A5E7B4E471C0C03CD105B1
:10D3800009F44CC0C03ED10509F459C0C03AD105DA
:10D3900009F06DC080E090E0A8ECB3E48093FD0458
:10D3A0009093FE04A093FF04B093000580E090E00A
:10D3B000AFE7B3E454C080E090ECA5E5B4E480931B
:10D3C000FD049093FE04A093FF04B093000580E059
:10D3D00090E0AEE3B4E443C080E090E8A7E2B4E4B8
:10D3E0008093FD049093FE04A093FF04B093000586
:10D3F00080E090E0A6E1B4E432C080E090E0A1EEED
:10D40000B3E48093FD049093FE04A093FF04B093D3
:10D41000000580E090E0A8ECB3E421C080E090E05B
:10D42000A5EAB3E48093FD049093FE04A093FF0467
:10D43000B093000580E090E8A3E9B3E410C080E079
:10D4400090E0A6E6B3E48093FD049093FE04A093DD
:10D45000FF04B093000580E090E0ADE4B3E4809376
:10D46000F9049093FA04A093FB04B093FC04DF91B9
:10D47000CF911F910F910895CF93DF93EC018CE230
:10D480009EE0A0D120E042E06EE1CE012EDF60E21E
:10D4900070E0CE0146DF81E0DF91CF9108956F9279
:10D4A0007F928F929F92AF92BF92CF92DF92EF9234
:10D4B000FF920F931F93CF93DF93EC016EE18CE209
:10D4C0009EE089D1E0912C0EF0912D0E0190F0811B
:10D4D000E02D63E08CE29EE019958CE29EE0F9D1AC
:10D4E00046E06EE18CE29EE0F0D18CE29EE0D5D089
:10D4F0000697DCF38CE29EE0D8D0682E8CE29EE0AA
:10D50000D4D0782E8CE29EE0D0D0C82E8CE29EE063
:10D51000CCD0D82E8CE29EE0C8D0882E8CE29EE043
:10D52000C4D0982EB62CA12CA728B501882777FD4A
:10D530008095982F0E94CC956D837E838F839887EA
:10D54000F82CE12CE928B701882777FD8095982FE2
:10D550000E94CC9569877A878B879C871C2D00E079
:10D560000D29B801882777FD8095982F0E94CC95CA
:10D570006D877E878F87988B198A1A8A1B8A1C8AE7
:10D58000DF91CF911F910F91FF90EF90DF90CF909F
:10D59000BF90AF909F908F907F906F900895CF92A3
:10D5A000DF92EF92FF920F931F93CF93DF938C0143
:10D5B000EB0184E2FB0111928A95E9F7C8016FDF64
:10D5C00084E290E0A0E0B0E088839983AA83BB83E3
:10D5D000F80185899689A789B08D8C839D83AE8358
:10D5E000BF8382E090E0A0E0B0E088879987AA87B7
:10D5F000BB87188A198A1A8A1B8AC090FD04D090AA
:10D60000FE04E090FF04F0900005A70196016581FB
:10D610007681878190850E94009520E030E048EC7B
:10D6200052E40E9460976C8B7D8B8E8B9F8BA70141
:10D630009601F80161857285838594850E94009525
:10D6400020E030E048EC52E40E946097688F798FC8
:10D650008A8F9B8F2091F9043091FA044091FB044A
:10D660005091FC04F80165857685878590890E9434
:10D67000009520E030E048EC52E40E9460976C8F07
:10D680007D8F8E8F9F8F81E0DF91CF911F910F91C2
:10D69000FF90EF90DF90CF90089580915C0E90E026
:10D6A00020915D0E821B9109089520915D0E80915D
:10D6B0005C0E281750F4E22FF0E0E25AF14F80811F
:10D6C00090E02F5F20935D0E08958FEF9FEF0895F8
:10D6D000E0915D0E80915C0EE81730F4F0E0E25AC4
:10D6E000F14F808190E008958FEF9FEF08950895A6
:10D6F000CF92DF92EF92FF920F931F93CF93DF931E
:10D700007C01CB018A012091380E222389F0EB01A4
:10D710006B01C40ED51ECC15DD0561F06991D701F2
:10D72000ED91FC910190F081E02DC7011995F3CFA7
:10D73000642F91D1C801DF91CF911F910F91FF907C
:10D74000EF90DF90CF900895CF93DF931F92CDB7E6
:10D75000DEB769832091380E2223D1F02091390E53
:10D76000203240F021E030E0FC013383228380E06E
:10D7700090E014C080913A0EE82FF0E0E55CF14FA4
:10D78000998190838F5F80933A0E8093390E04C005
:10D7900061E0CE0101965FD181E090E00F90DF91D2
:10D7A000CF910895FC011382128248EE53E060E0AD
:10D7B00070E044835583668377838FE59BE0918394
:10D7C0008083089510925D0E10925C0E10923A0EB6
:10D7D0001092390E83C081E08093380E60935B0E07
:10D7E00010923A0E1092390E0895F5CF0F93062F2E
:10D7F00021E04091390E6BE37EE080915B0ED4D046
:10D8000010923A0E1092390E1092380E0F91089520
:10D810008F929F92AF92BF92CF92DF92EF92FF9240
:10D820000F931F93CF93DF93EC01F62ED42E480174
:10D830005901EE2009F1CFDF1E2D143008F013E05E
:10D840001150B8F0E881F98128E0129FB00111244D
:10D85000A501940104C056954795379527956A957B
:10D86000D2F7CA01B9010190F081E02DCE011995DE
:10D87000E7CF60E0CE01BADF4D2D413208F040E243
:10D880002C2D6EE57EE08F2D47D010925D0E80939B
:10D890005C0EDF91CF911F910F91FF90EF90DF9081
:10D8A000CF90BF90AF909F908F900895CF92EF92BE
:10D8B0000F931F93C22EE12C00E010E09801A8DF27
:10D8C0001F910F91EF90CF90089521E0EFCF21E0CD
:10D8D000EDCF61E08BCF8CE29EE064CF1092EB0E37
:10D8E00081E08093E90E1092E80E61E084E10E94ED
:10D8F0003B8861E085E10E943B88E9EBF0E08081B4
:10D900008E7F808380818D7F808388E48093B800C0
:10D9100085E48093BC000895413208F043C09091A3
:10D92000EB0E9111FCCF91E09093EB0E2093E90E5A
:10D930002FEF20937E0E1092C30E240F2093C20E61
:10D940009093EA0E9091EA0E880F892B8093EA0E4D
:10D950008091E80E813061F41092E80E8091EA0E19
:10D960008093BB008091BC0083FDF8CF85EC01C0A3
:10D9700085EE8093BC008091EB0E8130E1F38091C5
:10D98000C30E841710F44091C30E24EC3EE0FB015B
:10D99000D9018A2F821B841718F48D918193F9CFB6
:10D9A000842F089580E008950F93413208F04AC013
:10D9B0009091EB0E9111FCCF92E09093EB0E0093BF
:10D9C000E90E9FEF90937E0E1092C30E4093C20E0D
:10D9D000FB0164EC7EE0DB019A2F961B941718F490
:10D9E00091919D93F9CF1092EA0E9091EA0E880FD3
:10D9F000892B8093EA0E8091E80E813061F41092B9
:10DA0000E80E8091EA0E8093BB008091BC0083FDFC
:10DA1000F8CF85EC01C085EE8093BC00222321F075
:10DA20008091EB0E8230E1F380917E0E8F3F61F0AA
:10DA300080917E0E803251F080917E0E803341F4D1
:10DA400083E007C081E005C080E003C082E001C040
:10DA500084E00F910895613298F42091EB0E243008
:10DA600089F46093A00EFC0182EA9EE0DC012A2F7B
:10DA7000281B261718F421912D93F9CF80E00895E3
:10DA800081E0089582E0089585ED8093BC00809147
:10DA9000BC0084FDFCCF1092EB0E089585EC8093C2
:10DAA000BC001092EB0E08951F920F920FB60F92CA
:10DAB00011240BB60F922F933F934F935F936F9365
:10DAC0007F938F939F93AF93BF93EF93FF93809137
:10DAD000B900887F803609F49DC070F5883209F45A
:10DAE0005CC090F4803109F455C038F4882309F4FF
:10DAF000F3C0883009F44EC0F2C0883109F44DC03B
:10DB0000803209F45EC0EBC0803409F469C050F47F
:10DB1000803309F456C0883309F0E1C080937E0E4B
:10DB2000BDDFDDC0803509F44FC0883509F45DC024
:10DB3000883409F0D4C0D2C0883909F4C3C0A8F42D
:10DB4000883709F467C038F4883609F463C0803731
:10DB500009F460C0C4C0883809F4B4C0803909F43D
:10DB60005FC0803809F0BBC05BC0803B09F482C055
:10DB700038F4803A09F466C0883A09F47BC0AFC033
:10DB8000803C09F4A3C0883C09F4A0C0883B09F498
:10DB900086C0A5C08091EA0E10C09091C30E8091FE
:10DBA000C20E981770F5E091C30E81E08E0F80933E
:10DBB000C30EF0E0EC53F14F80818093BB0085EC05
:10DBC00082C080937E0E8AC0E091C30E81E08E0FEA
:10DBD0008093C30E8091BB00F0E0EC53F14F808343
:10DBE0009091C30E8091C20E6AC0E091C30E81E095
:10DBF0008E0F8093C30E8091BB00F0E0EC53F14F89
:10DC000080838091E90E811169C081E08093E80EE4
:10DC100084EA5DC083E08093EB0E10927F0ECFCF3D
:10DC200080917F0E803208F04DC0E0917F0E81E040
:10DC30008E0F80937F0E8091BB00F0E0E058F14F93
:10DC40008083BDCF2BDF80917F0E803230F4E09156
:10DC50007F0EF0E0E058F14F108260917F0E70E08F
:10DC6000E091E40EF091E50E80E89EE019951092A7
:10DC70007F0E35C084E08093EB0E1092A10E1092BF
:10DC8000A00EE091E60EF091E70E19958091A00E9E
:10DC9000811105C081E08093A00E1092A20EE09148
:10DCA000A10E81E08E0F8093A10EF0E0EE55F14FB2
:10DCB00080818093BB009091A10E8091A00E981757
:10DCC00008F47DCF85E88093BC0009C085EC809383
:10DCD000BC001092EB0E03C010927E0ED5DEFF91B9
:10DCE000EF91BF91AF919F918F917F916F915F91D4
:10DCF0004F913F912F910F900BBE0F900FBE0F9041
:10DD00001F901895FC0181E08083118243EC5BEA4F
:10DD100066E77BE3428353836483758348ED5BE668
:10DD200066E77BE3468357836087718742EF54EE53
:10DD300064E67BE342875387648775870895FC0117
:10DD4000DB014D915D916D917C91139742835383DB
:10DD50006483758314964D915D916D917C911797B5
:10DD6000468357836087718718964D915D916D91B9
:10DD70007C911B9742875387648775870895CF935B
:10DD8000DF93FC01EB0142815381648175814883FB
:10DD900059836A837B8346815781608571854C8373
:10DDA0005D836E837F8382859385A485B58588870F
:10DDB0009987AA87BB87DF91CF9108950F931F930F
:10DDC000CF93DF93082F67E376E086EC9FE00E9415
:10DDD000D48CC7E0D0E010E0B8010C2E02C07595DD
:10DDE00067950A94E2F76170772742E050E086EC8D
:10DDF0009FE00E94BE8D219778F7DF91CF911F9110
:10DE00000F9108951F93CF93DF931F92CDB7DEB785
:10DE1000162F63E570E08CE29EE04983E6DC612F1B
:10DE20008CE29EE091DC4981642F8CE29EE08CDCE8
:10DE30008CE29EE00F90DF91CF911F914ACDCF935E
:10DE4000DF93EC018CE29EE0BDDC40E06DE2CE01B0
:10DE5000D9DF40E16DE2CE01D5DF48E06DE2CE01D1
:10DE6000DF91CF91CFCF6F3F710534F4AB0177FFD6
:10DE700005C040E050E002C04FEF50E06DE1C2CF7E
:10DE8000EF92FF921F93CF93DF931F92CDB7DEB730
:10DE90007C01142F462F6EE12983B4DF412F6FE1FF
:10DEA000C701B0DF2981422F60E2C7010F90DF91E7
:10DEB000CF911F91FF90EF90A5CF6F3F710534F484
:10DEC000AB0177FF05C040E050E002C04FEF50E0EB
:10DED00061E298CF462F62E295CF6F3F710534F42F
:10DEE000AB0177FF05C040E050E002C04FEF50E0CB
:10DEF00063E288CF6F3F710534F4AB0177FF05C053
:10DF000040E050E002C04FEF50E064E27BCF6F3F53
:10DF1000710534F4AB0177FF05C040E050E002C06A
:10DF20004FEF50E065E26ECF6F3F710534F4AB0107
:10DF300077FF05C040E050E002C04FEF50E066E2DE
:10DF400061CF6F3F710534F4AB0177FF05C040E04E
:10DF500050E002C04FEF50E068E254CF6F3F7105D0
:10DF600034F4AB0177FF05C040E050E002C04FEF52
:10DF700050E069E247CFAF92BF92CF92DF92EF922B
:10DF8000FF920F931F93CF93DF938C01C62F7A01DB
:10DF9000690163E570E08CE29EE027DC6C2F8CE287
:10DFA0009EE0D2DB8CE29EE094DC63E570E08CE2E4
:10DFB0009EE01BDCA70163E570E08CE29EE087DC5D
:10DFC000E6015E01AC18BD088CE29EE066DB892BA1
:10DFD00029F08CE29EE069DB8993F3CFAE14BF0495
:10DFE00021F0F801108281E081838CE29EE0DF91D4
:10DFF000CF911F910F91FF90EF90DF90CF90BF9046
:10E00000AF9067CCCF92DF92EF92FF920F931F9366
:10E01000CF93DF93EC016B017A0189019C01225FB0
:10E020003F4F46E050E062E3A6DF8F8590E0982FF7
:10E0300088272E85822BF60191838083898990E041
:10E04000982F88272889822BF701918380838B89D9
:10E0500090E0982F88272A89822BF801918380836A
:10E06000DF91CF911F910F91FF90EF90DF90CF90B4
:10E0700008959B012C5F3F4FAB014E5F5F4FC2CFB6
:10E08000AF92BF92CF92DF92EF92FF920F931F93C6
:10E09000CF93DF9300D000D0CDB7DEB77C015B011A
:10E0A000BE016F5F7F4FE5DFCE0101966C018701F6
:10E0B00075015E0197E0A90EB11CF60161917191A5
:10E0C0006F01882777FD8095982F0E94CC95F801E5
:10E0D00022813381448155810E946097F7016193C9
:10E0E0007193819391937F010C5F1F4FCA14DB04DE
:10E0F00021F726960FB6F894DEBF0FBECDBFDF9195
:10E10000CF911F910F91FF90EF90DF90CF90BF9034
:10E11000AF900895CF93DF931F92CDB7DEB79E01E6
:10E120002F5F3F4F41E050E06DE125DF898190E0B6
:10E130000F90DF91CF910895AF92BF92CF92DF926F
:10E14000EF92FF920F931F93CF93DF931F92CDB760
:10E15000DEB78C015B016A0179019E012F5F3F4FA1
:10E1600041E050E06EE107DF898190E0F5019183A5
:10E1700080839E012F5F3F4F41E050E06FE1C80177
:10E18000FADE898190E0F601918380839E012F5F02
:10E190003F4F41E050E060E2C801EDDE898190E050
:10E1A000F701918380830F90DF91CF911F910F91A1
:10E1B000FF90EF90DF90CF90BF90AF900895CF93F6
:10E1C000DF931F92CDB7DEB79E012F5F3F4F41E037
:10E1D00050E061E2D0DE898190E00F90DF91CF9135
:10E1E0000895CF93DF931F92CDB7DEB79E012F5FC7
:10E1F0003F4F41E050E062E2BEDE898190E00F9047
:10E20000DF91CF910895CF93DF931F92CDB7DEB703
:10E210009E012F5F3F4F41E050E063E2ACDE898119
:10E2200090E00F90DF91CF910895CF93DF931F92ED
:10E23000CDB7DEB79E012F5F3F4F41E050E064E273
:10E240009ADE898190E00F90DF91CF910895CF936E
:10E25000DF931F92CDB7DEB79E012F5F3F4F41E0A6
:10E2600050E065E288DE898190E00F90DF91CF91E8
:10E270000895CF93DF931F92CDB7DEB79E012F5F36
:10E280003F4F41E050E066E276DE898190E00F90FA
:10E29000DF91CF910895CF93DF931F92CDB7DEB773
:10E2A0009E012F5F3F4F41E050E068E264DE8981CC
:10E2B00090E00F90DF91CF910895CF93DF931F925D
:10E2C000CDB7DEB79E012F5F3F4F41E050E069E2DE
:10E2D00052DE898190E00F90DF91CF910895CF9326
:10E2E000DF931F92CDB7DEB79E012F5F3F4F41E016
:10E2F00050E06CE240DE69816F7070E06650710939
:10E30000882777FD8095982F0E94CC959B01AC01C2
:10E3100060E070E080E090E40E94C39720E030E08D
:10E3200048EC50E40E9460970F90DF91CF910895E0
:10E33000EF92FF920F931F93CF93DF931F92CDB76E
:10E34000DEB78C01CB01BA0120E030E048EC50E4AC
:10E350000E9400950E949995E12CF12C7595679586
:10E360006115710521F08FEFE81AF80AF7CF8AE0FE
:10E37000E816F10484F49E012F5F3F4F41E050E026
:10E380006CE2C801F8DD46E04E0D8981807F482BA4
:10E390006CE2C80137DD0F90DF91CF911F910F9193
:10E3A000FF90EF900895CF93DF931F92CDB7DEB724
:10E3B0009E012F5F3F4F41E050E060E3DCDD89814B
:10E3C0000F90DF91CF910895DF92EF92FF920F931C
:10E3D0001F93CF93DF931F92CDB7DEB78C01F62E3C
:10E3E000E42ED22E9E012F5F3F4F41E050E0C3DD6F
:10E3F000898121E030E00E2C01C0220F0A94EAF757
:10E40000DD2011F0282B02C0209528232983498183
:10E410006F2DC801F7DC0F90DF91CF911F910F9105
:10E42000FF90EF90DF900895262F47E050E061E3E2
:10E43000CBCF262F46E050E067E2C6CF262F45E03F
:10E4400050E067E2C1CF262F44E050E067E2BCCF46
:10E45000262F42E050E067E2B7CF262F41E050E0A0
:10E4600067E2B2CF262F40E050E067E2ADCF262F23
:10E4700047E050E067E2A8CF262F43E050E067E294
:10E48000A3CF262F43E050E06AE29ECF262F42E042
:10E4900050E06AE299CF262F41E050E06AE294CF43
:10E4A000262F40E050E06AE28FCF262F44E050E074
:10E4B0006CE28ACF242F462F50E06FE285CF242FC5
:10E4C000462F50E06EE280CF1F93CF93DF931F92D1
:10E4D000CDB7DEB7142F9E012F5F3F4F41E050E0D4
:10E4E0004ADD898190E002C0959587951A95E2F7FB
:10E4F00081700F90DF91CF911F91089547E050E018
:10E5000061E3E2CF46E050E067E2DECF45E050E075
:10E5100067E2DACF44E050E067E2D6CF42E050E075
:10E5200067E2D2CF41E050E067E2CECF40E050E07A
:10E5300067E2CACF43E050E067E2C6CF43E050E075
:10E540006AE2C2CF42E050E06AE2BECF41E050E072
:10E550006AE2BACF40E050E06AE2B6CF46E050E06F
:10E560006BE2B2CF45E050E06BE2AECF44E050E06A
:10E570006BE2AACF42E050E06BE2A6CF41E050E070
:10E580006BE2A2CF40E050E06BE29ECF43E050E070
:10E590006BE29ACF44E050E06CE296CF462F50E019
:10E5A00060E392CF462F50E06FE28ECF462F50E0CF
:10E5B0006EE28ACFEF92FF920F931F93CF93DF9378
:10E5C0001F92CDB7DEB77C016BE67BE086EC9FE067
:10E5D0000E94D48C9E012F5F3F4F41E050E060E0ED
:10E5E000C701C9DC8981EADB64E97BE086EC9FE056
:10E5F0000E94FF8C0DE110E068EE7AE086EC9FE06F
:10E600000E94D48C40E150E0B80186EC9FE00E946B
:10E61000BE8D64E37AE086EC9FE00E94D48C9E017C
:10E620002F5F3F4F41E050E0602FC701A4DC89819C
:10E63000C5DB64E97BE086EC9FE00E94FF8C0F5F06
:10E640001F4F0A331105C1F60F90DF91CF911F9133
:10E650000F91FF90EF900895FB016181828170E03E
:10E66000762F6627680F711D882777FD8095982F74
:10E670000E94CC9520E030E040E85DE30E94609786
:10E6800023E333E948E853E40C943594089521E0FA
:10E690006227FC0180810C943B88CF93DF93EC01CF
:10E6A000862F688349832A8361E00E94028861E0A3
:10E6B00088810E943B8860E089810E94028860E036
:10E6C0008A810E94028861E089810E943B8861E022
:10E6D0008A810E943B8860E0CE01DF91CF91D7CF45
:10E6E000FB0181819081890F9281890F9381981319
:10E6F00004C081E094819D3009F080E008952F925C
:10E700003F924F925F926F927F928F929F92AF92C1
:10E71000BF92CF92DF92EF92FF920F931F93CF930E
:10E72000DF9300D000D0CDB7DEB78C013B014E8324
:10E730000E94C4861B012C0180ED280E87E0381E44
:10E74000411C511C61E0C801A2DFFE0131966F013E
:10E750004E01F6E08F0E911CF60185E011928A952C
:10E76000E9F7760127E0A22EB12CF80181810E9401
:10E770007088019739F40E94C48662157305840578
:10E78000950598F3F80181810E947088892B39F4EE
:10E790000E94C486621573058405950598F3F801F7
:10E7A00082810E947088892B59F0F701208181E0D5
:10E7B00090E00A2C01C0880F0A94EAF7282B2083E6
:10E7C000F1E0AF1AB10888F69FEFE91AF90AE814E8
:10E7D000F90441F60E94C486621573058405950507
:10E7E00040F060E0C80153DF20E030E040EC5FE73C
:10E7F0002EC08981EE818E13AFCFB601C80170DFC4
:10E80000882309F4A9CF60E0C80141DFB601C8013F
:10E8100023DFFB01DC016A946728B9F420E030E0D3
:10E8200040E151E4BF01CD010E94609720E030E05B
:10E8300040EA50E40E94009520E030E040E052E4DD
:10E840000E9436949B01AC0102C09F01AD01B90149
:10E85000CA0126960FB6F894DEBF0FBECDBFDF917A
:10E86000CF911F910F91FF90EF90DF90CF90BF90CD
:10E87000AF909F908F907F906F905F904F903F9060
:10E880002F90089546E63BCF4CE439CFFB018081C1
:10E89000883251F028F4803139F0823239F404C0E2
:10E8A0008B3311F0823411F481E0089580E00895F3
:10E8B000FC017783668314821582108289E081834C
:10E8C00081E0828383830895CF93DF93EC01F0DFAF
:10E8D0001B8A1A8ADF91CF910895FC0185810895E2
:10E8E000CF93DF93EB0167E0CE010E94FB6891E0DC
:10E8F0002F81821390E0892FDF91CF910895EF92BD
:10E90000FF920F931F93CF93DF93EC018B01E42EC3
:10E910008E819F810E942F68F12C41E0B8018E8189
:10E920009F810E946368882351F0FE1005C0B801E2
:10E93000CE01D6DF811104C0F394EF1470F780E0AC
:10E94000DF91CF911F910F91FF90EF900895CF929B
:10E95000DF92EF92FF920F931F93CF93DF931F925B
:10E960001F92CDB7DEB76C01F42EE52EFC01868137
:10E97000978169837A830E940D6769817A818823F0
:10E9800011F1F601868197810E94066840E06EEBE6
:10E99000F601868197810E94AA670F2D1E2D89E0BE
:10E9A000F82EF601868197810E94EB67F80181932A
:10E9B0008F01FA94B1F7F601868197810E940D6765
:10E9C00091E0813009F090E0892F0F900F90DF9156
:10E9D000CF911F910F91FF90EF90DF90CF9008950E
:10E9E000CF93DF93EA01B3DF882351F068E0CE01D3
:10E9F0000E94FB6891E02885821390E0892F01C076
:10EA000080E0DF91CF910895EF92FF920F931F93D3
:10EA1000CF93DF93EC018B017A018E819F810E945D
:10EA20000D67B8018E819F810E94066840E06EE408
:10EA30008E819F810E94AA6740E0F70162818E81EA
:10EA40009F810E94AA6740E0F70163818E819F81C8
:10EA50000E94AA67F8018081803139F040E0F70117
:10EA600064818E819F810E94AA678E819F810E940E
:10EA70000D67B8018E819F810E940668488168E415
:10EA80008E819F810E94AA6764E170E080E090E03F
:10EA90000E94F3868881882331F06AE070E080E08C
:10EAA00090E00E94F3868E819F81DF91CF911F912C
:10EAB0000F91FF90EF900C940D67EF92FF921F93D0
:10EAC000CF93DF931F921F92CDB7DEB77C01FC017D
:10EAD0008681978169837A830E940D6769817A8133
:10EAE000F701868197810E94066840E064EBF70198
:10EAF000868197810E94AA67F701868197810E948B
:10EB00007F67182FF701868197810E940D6781E04A
:10EB1000111180E00F900F90DF91CF911F91FF9026
:10EB2000EF900895CF93DF93CDB7DEB729970FB657
:10EB3000F894DEBF0FBECDBFFB0120812031C9F0AC
:10EB4000AE014F5F5F4F4CDF882379F08D818F33AB
:10EB500051F020F48F3149F489E00CC08F3539F041
:10EB60008F3739F002C08AE005C080E003C08BE037
:10EB700001C08CE029960FB6F894DEBF0FBECDBF62
:10EB8000DF91CF910895FF920F931F93CF93DF935F
:10EB9000CDB7DEB728970FB6F894DEBF0FBECDBF56
:10EBA0008C01FC01868197810E942F68F8011482F4
:10EBB000158241E0BE016F5F7F4FF801868197812A
:10EBC0000E9463688823C1F1BE016F5F7F4FC80157
:10EBD00087DE882371F3F8018081811107C0BE01AF
:10EBE0006F5F7F4FC80169DF811122C0F801F1809A
:10EBF000BE016F5F7F4FC80195DF8F1518F4F801D4
:10EC0000818105C0BE016F5F7F4FC8018BDFF801B6
:10EC1000818384818F5F8483BE016F5F7F4FC801D2
:10EC200035DE882331F2F80185818F5F8583C1CF7E
:10EC300081E0F8018083DACF28960FB6F894DEBF22
:10EC40000FBECDBFDF91CF911F910F91FF9008951F
:10EC5000DF92EF92FF920F931F93CF93DF93CDB785
:10EC6000DEB762970FB6F894DEBF0FBECDBF8C0142
:10EC70007B01D22E493028F0342F4D3018F03CE083
:10EC800001C039E0B701C8013A8B4CDF3A898317DC
:10EC900009F458C0AE014F5F5F4FB701C8013A8B0E
:10ECA0009FDE3A89882309F44FC0F70180818031C3
:10ECB00009F448C03B3041F03C3021F03A3031F4A7
:10ECC0008FE305C08FE703C08FE501C08FE18D831F
:10ECD000AE014F5F5F4FB701C8013A8B95DEF80177
:10ECE00091813A89832F391708F4892FF80181839C
:10ECF000D11028C0381730F53183E12CF12CF80100
:10ED0000848190E0E816F906ECF44E2DBE01665FB2
:10ED10007F4FC801F4DDF801D180BE01665F7F4FEF
:10ED2000C80100DF8D1518F4F801818105C0BE010E
:10ED3000665F7F4FC801F6DEF8018183FFEFEF1AAF
:10ED4000FF0ADDCF81E001C080E062960FB6F89443
:10ED5000DEBF0FBECDBFDF91CF911F910F91FF900E
:10ED6000EF90DF900895EF92FF920F931F93CF9350
:10ED7000DF93CDB7DEB728970FB6F894DEBF0FBE8E
:10ED8000CDBF8C01693020F06D3018F06CE001C00F
:10ED900069E0F8016183E12CF12CF801848190E0B5
:10EDA000E816F90694F44E2DBE016F5F7F4FC8013F
:10EDB000A6DD21E0F8014181BE016F5F7F4FC801F0
:10EDC00047DFFFEFEF1AFF0AE8CF28960FB6F89457
:10EDD000DEBF0FBECDBFDF91CF911F910F91FF908E
:10EDE000EF900895FC01868197810E947F6791E0F2
:10EDF000813009F090E0892F08958F929F92AF9211
:10EE0000BF92CF92DF92EF92FF920F931F93CF9317
:10EE1000DF93EC016950633048F4E62FF0E0EE0F29
:10EE2000FF1FEE58F44F0081118102C00EEE12E078
:10EE30008B818823E1F08881811119C00E94C486EA
:10EE40006B017C014801AA2497FCA094BA2CCE0146
:10EE5000C9DF81111FC00E94C486681979098A0917
:10EE60009B096C157D058E059F05A0F4F0CFB801B8
:10EE7000882777FD8095982FDF91CF911F910F9173
:10EE8000FF90EF90DF90CF90BF90AF909F908F90CA
:10EE90000C94F386DF91CF911F910F91FF90EF902B
:10EEA000DF90CF90BF90AF909F908F900895CF93B9
:10EEB000DF93EC018E819F810E940D678E819F817F
:10EEC0000E942C68488164E48E819F810E94AA6719
:10EED0008A81882329F06981CE01DF91CF918DCF7E
:10EEE000DF91CF910895FA01208148E0249F90019D
:10EEF0001124818190E0982F8827990F990F990FFD
:10EF0000282B392BDB018C918031C1F4678170E0B3
:10EF10008681AB01481B5109CA019695982F882715
:10EF2000979587950E94909860517109207F53E0D2
:10EF3000220F331F5A95E1F7260F371FC901089595
:10EF4000EF92FF920F931F93CF93DF93CDB7DEB76E
:10EF500029970FB6F894DEBF0FBECDBF8C017B01A1
:10EF6000AE014F5F5F4F3CDD882339F0AE014F5F4C
:10EF70005F4FB701C801B7DF02C080E894EE299661
:10EF80000FB6F894DEBF0FBECDBFDF91CF911F91BA
:10EF90000F91FF90EF900895813824EE92076CF066
:10EFA000BC01882777FD8095982F0E94CC9520E0A2
:10EFB00030E040E05CE30C94609760E070E08EEF3E
:10EFC00092EC0895BDDFE8CF0F931F93CF93DF93AB
:10EFD000CDB7DEB728970FB6F894DEBF0FBECDBF12
:10EFE0008C01462FBE016F5F7F4F89DC882331F093
:10EFF000BE016F5F7F4FC801E5DF04C060E070E0D5
:10F000008EEF92EC28960FB6F894DEBF0FBECDBF00
:10F01000DF91CF911F910F910895FC01108214820E
:10F02000138215820895862F642F0C940288862FF0
:10F03000642F0C943B88862F0C9470884F925F92BB
:10F040006F927F928F929F92AF92BF92CF92DF92F8
:10F05000EF920F93CF93DF93EC014B013A015901EB
:10F060000296DBDF8CE79BE0998388836E018CE15D
:10F07000C80ED11C26018CE3480E511CC601CDDF01
:10F0800086E0C80ED11CC414D504C1F7FE01EE59A8
:10F09000FF4F718260823296B182A08232960083E5
:10F0A0003196E08237979182808238968AE090E0AC
:10F0B00091838083329684EF91E0918380833396AD
:10F0C0001182108271971082118212821382C459A8
:10F0D000DF4F1882DF91CF910F91EF90DF90CF90AB
:10F0E000BF90AF909F908F907F906F905F904F9068
:10F0F00008952F923F924F925F926F927F928F92DC
:10F100009F92AF92BF92CF92DF92EF92FF920F93B6
:10F110001F93CF93DF93CDB7DEB728970FB6F89440
:10F12000DEBF0FBECDBF98878F83F12C4C0186E6E2
:10F13000880E911C0F8118850E591F4FD4018C9198
:10F14000F816A0F4AF81B8858D919C91F801A0814B
:10F15000B181AF0DB11DFC012081318142E06C9184
:10F160008F819885F9011995F394E8CF512CEF819F
:10F17000F885E959FF4FFA83E9830F8118850C5907
:10F180001F4FC12CD12C7601C3948F8198858E5945
:10F190009F4F9C838B83A981BA818C91581608F06C
:10F1A00088C0A52CB12CAF81B8858D919C91F801B8
:10F1B000A081B181AA0DBB1DFC012081318141E0FC
:10F1C0006C918F819885F9011995AF81B8858D91E2
:10F1D0009C91F801A081B181AA0DBB1DFC01228187
:10F1E000338140E06C918F819885F9011995D701A1
:10F1F000C601052C04C0880F991FAA1FBB1F0A94C3
:10F20000D2F79C011C0120943094412CD4018C91A4
:10F21000EF81F88540815181481648F5642C712CA6
:10F22000EB81FC81A081B181A60DB71DFA0144815B
:10F2300055816C918F8198852D833E83FA011995B4
:10F24000660C771C2D813E81EF81F885E60DF71D58
:10F25000892B29F480859185822B932B04C080858E
:10F26000918582219321918780874394CFCFF801A4
:10F27000A081B181AA0DBB1DFA012281338141E039
:10F280006C918F819885F9011995AF81B8858D9121
:10F290009C91F801A081B181AA0DBB1DFC012081C8
:10F2A000318140E06C918F819885F90119955394D3
:10F2B00072CF28960FB6F894DEBF0FBECDBFDF9198
:10F2C000CF911F910F91FF90EF90DF90CF90BF9063
:10F2D000AF909F908F907F906F905F904F903F90F6
:10F2E0002F900895FC0180E090E0258D368D261743
:10F2F000370739F0019636968A309105B1F78FEFCE
:10F300009FEF0895DC0126E0629FA00DB11D11243E
:10F3100090965C934E935F9721E091962C939197F2
:10F32000FC01E459FF4F208131960190F081E02DDE
:10F33000222331F0309749F0611107C0DC0102C08F
:10F34000309719F05C968C9119940895CF92DF92C2
:10F35000FF920F931F93CF93DF931F92CDB7DEB72A
:10F360006C01F62EFC0186E0689FE00DF11D112472
:10F3700011A2878D90A181309105E9F01CF4892BB1
:10F3800051F044C08230910591F1039709F03EC0DD
:10F3900040E050E030C04423C9F141E050E0C601F4
:10F3A000B1DF0E94C486F601E85AFF4F6083718383
:10F3B000828393832BC049830E94C486F601E85A56
:10F3C000FF4F0081118122813381601B710B820B01
:10F3D000930B72960081118120E030E0498106177D
:10F3E00017072807390718F442E050E004C041111C
:10F3F0000DC043E050E06F2DC6010F90DF91CF911B
:10F400001F910F91FF90DF90CF907CCF0F90DF91F5
:10F41000CF911F910F91FF90DF90CF9008952F9281
:10F420003F924F925F926F927F928F929F92AF9294
:10F43000BF92CF92DF92EF92FF920F931F93CF93E1
:10F44000DF931F92CDB7DEB71C01FC014AE08FEFBE
:10F450009FEF278D30A1232B21F4148E968F858F5B
:10F4600011A2415036964111F4CF712C610126E66C
:10F47000C20ED11C510187E6A80EB11C4101A0E6C5
:10F480008A0E911C46E0442ED6018C91781608F025
:10F4900053C0612C8101070D111D070D111D085F5F
:10F4A0001F4FF501E0806E1408F044C0F801408160
:10F4B0005181062C02C0569547950A94E2F7417097
:10F4C0007E9C70011124E60CF11CD401ED91FC919D
:10F4D000EE0DFF1D5080B701C101498303DF498153
:10F4E00097FD02C0682F1BC0019611F5442301F15E
:10F4F00080E090E060E070E0F101E80FF91F248DFA
:10F50000211110C0469EF001479EF00D1124E20D1E
:10F51000F31D548EF68EE58E10A2178E41E0C101C8
:10F5200015DF06C06F5F7F4F06966A30710521F7C1
:10F530006394B7CF7394A8CF20E030E080E0F1016E
:10F54000E20FF31F91A1911181E02A5F3F4F2C330D
:10F550003105A9F70F90DF91CF911F910F91FF9087
:10F56000EF90DF90CF90BF90AF909F908F907F9063
:10F570006F905F904F903F902F900895CF92DF92C1
:10F58000EF92FF920F931F93CF93DF938C010E9412
:10F59000C486E801C45ADF4FC880D980EA80FB8066
:10F5A0006C197D098E099F09F801E859FF4FC08049
:10F5B000D180E12CF12CC616D706E806F90660F4D6
:10F5C000C80197DDC8012BDF182F0E94C48668830D
:10F5D00079838A839B8301C010E0812FDF91CF91D3
:10F5E0001F910F91FF90EF90DF90CF9008950F93B0
:10F5F0001F93CF93DF93EC018C0104591F4F81E0DF
:10F60000F8018083CE01BADF882349F089A18823DD
:10F6100031F08F8D98A1019711F48C8D03C0F80102
:10F62000108280E0DF91CF911F910F910895CF92CA
:10F63000DF92EF92FF92CF93DF93EC01882777FD63
:10F640008095982F0E94CC956B017C0120E030E0E2
:10F6500040E45FE30E94609720E030E048E452E439
:10F660000E9400950E949995C617D707ECF020E0FC
:10F6700030E040EA5FE3C701B6010E94609720E0F6
:10F6800030E048E452E40E94009520E030E040E899
:10F690005FE30E9436940E94999521E06C177D07E4
:10F6A0000CF420E0822F01C080E090E0DF91CF9148
:10F6B000FF90EF90DF90CF900895CF92DF92EF927E
:10F6C000FF92CF93DF93EC016C597F4F882777FD32
:10F6D0008095982F0E94CC956B017C0120E030E052
:10F6E00040E45FE30E94609720E030E048E452E4A9
:10F6F0000E9400950E949995C617D707ECF020E06C
:10F7000030E040EA5FE3C701B6010E94609720E065
:10F7100030E048E452E40E94009520E030E040E808
:10F720005FE30E9436940E94999521E06C177D0753
:10F730000CF420E0822F01C080E090E0DF91CF91B7
:10F74000FF90EF90DF90CF900895CF92DF92EF92ED
:10F75000FF92CF93DF93EC0164567109882777FD00
:10F760008095982F0E94CC956B017C0120E030E0C1
:10F7700040E45FE30E94609720E030E048E452E418
:10F780000E9400950E949995C617D707ECF020E0DB
:10F7900030E040EA5FE3C701B6010E94609720E0D5
:10F7A00030E048E452E40E94009520E030E040E878
:10F7B0005FE30E9436940E94999521E06C177D07C3
:10F7C0000CF420E0822F01C080E090E0DF91CF9127
:10F7D000FF90EF90DF90CF9008951F920F920FB699
:10F7E0000F9211240BB60F922F933F934F935F9379
:10F7F0006F937F938F939F93AF93BF93EF93FF93F9
:10F800008091ED0E0E9470882091F00E3091F10EE3
:10F810002F5F3F4F3093F10E2093F00E9091EF0E3B
:10F82000953618F096E09093EC0E9091EC0E943093
:10F83000C9F128F4923069F09330D1F05EC0953070
:10F8400009F451C0963009F058C091E09093BC0F74
:10F8500051C0811152C02091F00E3091F10E24362A
:10F86000310508F442C01092BC0F1092EF0E1CC07C
:10F87000813009F042C0E091EF0E91E09E0F90932D
:10F88000EF0EF0E02091F00E3091F10EEE0FFF1F21
:10F89000EE50F14F318320831092F10E1092F00E52
:10F8A00094E029C0811117C0E091EF0E91E09E0F06
:10F8B0009093EF0EF0E02091F00E3091F10EEE0FEC
:10F8C000FF1FEE50F14F318320831092F10E109202
:10F8D000F00E93E010C02091F00E3091F10E25361D
:10F8E000310558F007C0811108C01092F10E109236
:10F8F000F00E03C095E09093EC0E9091EE0E9923DC
:10F9000029F0811102C02F9A01C02F98FF91EF9129
:10F91000BF91AF919F918F917F916F915F914F9127
:10F920003F912F910F900BBE0F900FBE0F901F9025
:10F9300018956093ED0E1092EE0E0895F89482E003
:10F940008093B0008093B10094E69093B30010923E
:10F95000B2008093700078948093EC0E1092EF0EBA
:10F960008091ED0E60E00C94028882E08093EC0EB2
:10F970001092EF0E08958F929F92AF92BF92CF9206
:10F98000DF92EF92FF927B01BA0180E090E00E944B
:10F99000CA954B015C01B70180E090E00E94CA95D6
:10F9A0006B017C012DEC3CEC4CE45FE30E94609722
:10F9B0009B01AC01C501B4010E94FC9487FD17C0F6
:10F9C0002DEC3CEC4CE45FE3C501B4010E94609770
:10F9D0009B01AC01C701B6010E94FC94992787FDE9
:10F9E00090958827990F881F9927019602C080E07B
:10F9F00090E0FF90EF90DF90CF90BF90AF909F90FE
:10FA00008F9008958F929F92AF92BF92CF92DF9284
:10FA1000EF92FF920F931F93CF93DF936C01EB0153
:10FA2000EC84FD8486E0E816F1040CF443C0EE0C8F
:10FA3000FF1C06E010E045EC842E4DE9942E4CE1CD
:10FA4000A42E41E8B42E8A859B85FC01E00FF11FAE
:10FA500040815181F8013497E80FF91F608171816D
:10FA6000C60189DFFC01A501940163E971E080E032
:10FA700091E00E946D984F01AA2497FCA094BA2CA3
:10FA800086269726A826B9260E5F1F4F0E151F053E
:10FA9000D1F68C829D82AE82BF8280E290E099870F
:10FAA00088878FEF9FEF9983888361E070E080E023
:10FAB00090E003C060E070E0CB01DF91CF911F9137
:10FAC0000F91FF90EF90DF90CF90BF90AF909F90FD
:10FAD0008F9008950F931F93CF93DF938C01EB01C9
:10FAE00082EF9EE09B878A878091EF0E90E09D8752
:10FAF0008C878091BC0F90E09F878E878091EC0E61
:10FB0000853009F051C0C8011BD3882319F081E06A
:10FB100090E04CC0BE01C801B0D78111F8CFBE0142
:10FB2000C80107D78111F3CFBE01C8017ED2811170
:10FB3000EECFBE01C801CCD48111E9CFBE01C8010E
:10FB400069D58111E4CFBE01C80192D38111DFCF05
:10FB5000BE01C801E3D18111DACFBE01C8012DD1A8
:10FB60008111D5CFBE01C80145D68111D0CFBE01CC
:10FB7000C8010E94D8858111CACFBE01C8011BD01F
:10FB80008111C5CFBE01C801A2D08111C0CFBE0175
:10FB9000C80138DF672B682B692B09F0B8CF82E0EA
:10FBA0008093EC0E1092EF0E80E090E0DF91CF9109
:10FBB0001F910F910895AF92BF92CF92DF92EF9273
:10FBC000FF920F931F93CF93DF93EB018091EF0E82
:10FBD000883510F480E070C0EA85FB8582819381CE
:10FBE00060E672E26ADD892BA9F3EA85FB858481F0
:10FBF000958164E971E1A9DD892B61F3BEE1CB2E2A
:10FC0000D12C1DE1E12EF12C00E010E08091EF0EEF
:10FC100090E00497E816F906ACF5EA85FB85C70184
:10FC2000880F991FE80FF91F8081918164EF71E0BF
:10FC300044DD892B79F25601AA0CBB1CEA85FB85B1
:10FC4000EA0DFB1D8081918168E572E07EDD892BE4
:10FC500021F0000F111F01600DC0EA85FB85EA0D40
:10FC6000FB1D8081918164EA76E06FDD892B49F08C
:10FC7000000F111F82E0E80EF11C82E0C80ED11CBB
:10FC8000C5CF760181E0E81AF108F594E794F9868A
:10FC9000E8868AE2E816F1040CF49CCFC801AA2792
:10FCA00097FDA095BA2F8C839D83AE83BF8389E097
:10FCB00090E09983888381E0DF91CF911F910F912C
:10FCC000FF90EF90DF90CF90BF90AF900895AF92EC
:10FCD000BF92CF92DF92EF92FF920F931F93CF9339
:10FCE000DF93EB018091EF0E803211F080E05AC07B
:10FCF000EA85FB85828193816CE271E0DEDC892BF1
:10FD0000A9F3EA85FB85848195816EEE72E01DDDA5
:10FD1000892B61F306E010E0C12CD12C7601EA8535
:10FD2000FB85E00FF11F808191816CE271E0C5DC01
:10FD3000892BE1F2580182E0A80EB11CEA85FB850F
:10FD4000EA0DFB1D8081918168E077E0FEDC892B64
:10FD500039F0CC0CDD1CEE1CFF1C6894C0F810C000
:10FD6000EA85FB85EA0DFB1D808191816EEE72E0D4
:10FD7000ECDC892B09F4BACFCC0CDD1CEE1CFF1C8B
:10FD80000C5F1F4F0E33110551F68EE090E09987FE
:10FD90008887CC82DD82EE82FF828FE090E09983BB
:10FDA000888381E0DF91CF911F910F91FF90EF90B9
:10FDB000DF90CF90BF90AF900895AF92BF92CF9257
:10FDC000DF92EF92FF920F931F93CF93DF93EB019C
:10FDD0008091EF0E823251F5EA85FB858281938115
:10FDE00068E572E06ADC892B09F18091EF0E90E002
:10FDF00081509048880F991FEA85FB85E80FF91F0D
:10FE00008081918168E572E058DC892B79F0198650
:10FE100018868FEF9FEFDC018C839D83AE83BF83B9
:10FE200086E090E09983888381E06DC0EA85FB8558
:10FE30008281938160E47FE140DC892B21F0809115
:10FE4000EF0E813210F480E05EC0EA85FB8584818C
:10FE5000958160EA7FE079DC892BA9F358E0A52E33
:10FE6000B12C03E010E0C12CD12C7601EA85FB8592
:10FE7000C801880F991FE80FF91F8081918168E5FB
:10FE800072E01BDC892BF9F2EA85FB85EA0DFB1D8C
:10FE90008081918160E476E058DC892B39F0CC0CCC
:10FEA000DD1CEE1CFF1C6894C0F810C0EA85FB85C1
:10FEB000EA0DFB1D8081918166E272E046DC892BB0
:10FEC00009F4C1CFCC0CDD1CEE1CFF1C0E5F1F4FD4
:10FED00084E0A80EB11C0332110541F6EA85FB85CA
:10FEE000EA5BFF4F8081918168E572E0E6DB892B58
:10FEF00009F4A9CF80E190E099878887CC82DD82E0
:10FF0000EE82FF828DCFDF91CF911F910F91FF90F5
:10FF1000EF90DF90CF90BF90AF900895AF92BF92D7
:10FF2000CF92DF92EF92FF920F931F93CF93DF93C5
:10FF3000EB018091EF0E893310F480E06BC0EA850D
:10FF4000FB858281938160E47FE1B7DB892BA9F394
:10FF5000EA85FB858481958160EA7FE0F6DB892B69
:10FF600061F338E0A32EB12C03E010E0C12CD12CBA
:10FF70007601EA85FB85C801880F991FE80FF91FF4
:10FF80008081918168E572E098DB892BB1F2EA8586
:10FF9000FB85EA0DFB1D8081918160E476E0D5DB75
:10FFA000892B39F0CC0CDD1CEE1CFF1C6894C0F8CA
:10FFB00010C0EA85FB85EA0DFB1D8081918166E218
:10FFC00072E0C3DB892B09F4B8CFCC0CDD1CEE1C2E
:10FFD000FF1C0E5F1F4F84E0A80EB11C0B331105F0
:10FFE00041F6EA85FB85EA58FF4F8081918168E5FB
:10FFF00072E063DB892B09F4A0CF8CE190E0998754
:020000021000EC
:100000008887CC82DD82EE82FF828AE090E099834D
:10001000888381E0DF91CF911F910F91FF90EF9046
:10002000DF90CF90BF90AF9008956F927F928F92A4
:100030009F92AF92BF92CF92DF92EF92FF920F9377
:100040001F93CF93DF93EB018091EF0E823208F480
:100050005DC0EA85FB85828193816EE571E02DDBD1
:10006000892B09F453C063E0A62EB12C02E010E006
:10007000C12CD12C760135018091EF0E90E0A816AD
:10008000B906CCF54801880C991CEA85FB85E80D7A
:10009000F91D808191816EE977E00FDB892B39F0C2
:1000A000CC0CDD1CEE1CFF1C6894C0F80FC0EA8568
:1000B000FB85E80DF91D808191816EEE72E0FDDA1D
:1000C000892B21F1CC0CDD1CEE1CFF1CC501880F17
:1000D000991FEA85FB85E80FF91F808191816EE504
:1000E00071E033DB22E0A20EB11C892B19F00E5F08
:1000F0001F4FC1CF8301015011091595079519872D
:1001000008870031110524F41986188680E009C09B
:10011000CC82DD82EE82FF828CE090E0998388833E
:1001200081E0DF91CF911F910F91FF90EF90DF90D1
:10013000CF90BF90AF909F908F907F906F900895D9
:10014000AF92BF92CF92DF92EF92FF920F931F93E5
:10015000CF93DF93EB01EA85FB858281938168E28F
:1001600073E2ABDA892B11F480E077C08091EF0E57
:10017000843009F5EA85FB85848195816AEC78E015
:10018000E4DA892BC1F0EA85FB858681978160E3FB
:1001900072E093DA892B79F0198618868FEF9FEF3A
:1001A000DC018C839D83AE83BF8383E090E09983E1
:1001B000888381E052C08091EF0E8434A8F2EA85F2
:1001C000FB858481958164E971E1BFDA892B61F255
:1001D00006E010E0C12CD12C7601EA85FB85E00F0A
:1001E000F11F8081918160E372E067DA892B09F465
:1001F000BBCF580182E0A80EB11CEA85FB85EA0D51
:10020000FB1D808191816AE976E09FDA892B39F0C4
:10021000CC0CDD1CEE1CFF1C6894C0F810C0EA85F5
:10022000FB85EA0DFB1D8081918160E372E08DDA30
:10023000892B09F499CFCC0CDD1CEE1CFF1C0C5F44
:100240001F4F0638110549F680E290E099878887AC
:10025000CC82DD82EE82FF82A8CFDF91CF911F9109
:100260000F91FF90EF90DF90CF90BF90AF900895E7
:100270008F929F92AF92BF92CF92DF92EF92FF92B6
:100280000F931F93CF93DF9300D01F92CDB7DEB7AC
:100290004B01DB011A96ED91FC911B9782819381B2
:1002A0006EEA7DE00ADA892B11F480E08FC0D40178
:1002B0001A96ED91FC911B978481958166ED76E00D
:1002C000FCD9892B91F3E6E0EE2EF12C20E030E012
:1002D00040E050E0A12CB12CC12CD12CD4011A96B5
:1002E000ED91FC911B97EE0DFF1D8081918166EFD2
:1002F00071E029833A834B835C83DFD9892BA9F290
:1003000087010E5F1F4FD4011A96ED91FC911B9748
:10031000E00FF11F808191816CED74E016DA298184
:100320003A814B815C81892B39F0B501C60101E02E
:100330000E94FB9821601CC0D4011A96ED91FC919B
:100340001B97E00FF11F8081918160E971E02983A3
:100350003A834B835C83F9D929813A814B815C8153
:10036000892B09F4A2CFB501C60101E00E94FB98D8
:100370005B016C01B4E0EB0EF11CE6ECEE16F1044F
:1003800009F0ACCFD40114962C93149715963C9396
:10039000159716964C93169717965C931797B50179
:1003A000C60100E20E94169912962C93129713969A
:1003B0003C93139785E090E011969C938E9380E395
:1003C00090E019969C938E93189781E00F900F9070
:1003D0000F900F90DF91CF911F910F91FF90EF90B1
:1003E000DF90CF90BF90AF909F908F9008958F92A5
:1003F0009F92AF92BF92CF92DF92EF92FF920F93B4
:100400001F93CF93DF937A016901DA01CD91DC91DB
:10041000FB0184859585C817D9070CF047C0CE012C
:10042000880F991F0284F385E02DE80FF91FA08043
:10043000B180C170DD27F1E0CF27209719F484E661
:1004400090E002C08CE99FEF4801880E991EB4012C
:10045000C501EDD8892B89F4800E911EB401C50128
:10046000E6D8892B69F4B401600F711FC501DFD88C
:10047000892BF9F023E030E005C021E030E002C034
:1004800022E030E0D6018D919C9111970196821760
:10049000930744F0F60111821082D7018D919C914F
:1004A000119701968D939C93CE0105C081E090E059
:1004B00002C08FEF9FEFDF91CF911F910F91FF90BF
:1004C000EF90DF90CF90BF90AF909F908F90089566
:1004D0004F925F926F927F928F929F92AF92BF9254
:1004E000CF92DF92EF92FF920F931F93CF93DF9300
:1004F00000D01F92CDB7DEB76C017B011C821B823E
:1005000081E090E09A8389838091EF0E8D3010F422
:1005100080E06BC009E713E09E012D5F3F4FAE0105
:100520004F5F5F4FC60163DF892B91F79E012D5FFF
:100530003F4FAE014F5F5F4FB701C60158DF0197D4
:1005400039F79E012D5F3F4FAE014F5F5F4FB701FF
:10055000C6014DDF892BE1F6412C512C3201A12C33
:10056000B12C8091EF0E90E029813A81281739074C
:100570008CF509E713E09E012D5F3F4FAE014F5F01
:100580005F4FB701C60133DF4C019E012D5F3F4F26
:10059000AE014F5F5F4FB701C60129DF21E0821630
:1005A000910451F4892B09F0B3CF440C551C661CFF
:1005B000771C689440F80AC0892809F0A9CF0197F0
:1005C00009F0A6CF440C551C661C771C8FEFA81AA7
:1005D000B80AC7CFF701B186A086448255826682E9
:1005E000778281E090E0918380830F900F900F904D
:1005F0000F90DF91CF911F910F91FF90EF90DF90BF
:10060000CF90BF90AF909F908F907F906F905F90B2
:100610004F9008952F923F924F925F926F927F92E8
:100620008F929F92AF92BF92CF92DF92EF92FF9202
:100630000F931F93CF93DF9300D01F92CDB7DEB7F8
:100640006C017B011C821B82DB011C968D919C91AD
:100650001D971816190614F080E0B5C0DB011A9634
:10066000ED91FC911B9782E090E09A8389838281CF
:1006700093816AE67AE021D8892B71F3D7011A9623
:10068000ED91FC911B9789819A819C012F5F3F4FCF
:100690003A832983880F991FE80FF91F8081918180
:1006A00069E773E052D8892BB9F20CEB11E09E0197
:1006B0002D5F3F4FAE014F5F5F4FB701C60197DE21
:1006C000892B51F69E012D5F3F4FAE014F5F5F4F6B
:1006D000B701C6018CDE019709F0BECF212C312C69
:1006E0002101A12CB12C29813A81F70184859585BE
:1006F000281739070CF05CC00CEB11E09E012D5F50
:100700003F4FAE014F5F5F4FB701C60170DE3C0146
:10071000B3E0AB16B10489F00CEB11E09E012D5F44
:100720003F4FAE014F5F5F4FB701C60160DE4C0126
:10073000E3E0AE16B104F9F40FC00CEB11E09E013A
:100740002D5F3F4FAE014F5F5F4FB701C6014FDED8
:100750006816790609F380CF0CEB11E09E012D5F3E
:100760003F4FAE014F5F5F4FB701C60140DE8816B5
:10077000990609F071CF6114710459F48A9489289B
:1007800009F06ACF220C331C441C551C689420F8D5
:100790000BC06A94672809F05FCF892809F05CCF05
:1007A000220C331C441C551CAFEFAA1ABA0A9BCF6B
:1007B000B186A086248235824682578282E090E00C
:1007C0009183808381E00F900F900F900F90DF91C5
:1007D000CF911F910F91FF90EF90DF90CF90BF903E
:1007E000AF909F908F907F906F905F904F903F90D1
:1007F0002F900895AF92BF92CF92DF92EF92FF9227
:100800000F931F93CF93DF93EB01EA85FB858281E2
:10081000938168E873E10E945D7B892B11F480E08D
:100820007DC08091EF0E843019F5EA85FB858481C7
:1008300095816AEC78E00E94A57B892BC9F0EA8556
:10084000FB858681978160E372E00E945D7B892B46
:1008500079F0198618868FEF9FEFDC018C839D83DA
:10086000AE83BF8387E090E09983888381E056C0A0
:100870008091EF0E843498F2EA85FB85848195811E
:1008800068E873E10E94A57B892B49F206E010E03D
:10089000C12CD12C7601EA85FB85E00FF11F808108
:1008A000918160E372E00E945D7B892B09F4B7CFF0
:1008B000580182E0A80EB11CEA85FB85EA0DFB1DFC
:1008C0008081918160E476E00E94A57B892B39F0DC
:1008D000CC0CDD1CEE1CFF1C6894C0F811C0EA852E
:1008E000FB85EA0DFB1D8081918160E372E00E942F
:1008F000A57B892B09F493CFCC0CDD1CEE1CFF1CCF
:100900000C5F1F4F0638110531F680E290E09987A1
:100910008887CC82DD82EE82FF82A4CFDF91CF91E7
:100920001F910F91FF90EF90DF90CF90BF90AF900D
:1009300008958F929F92AF92BF92CF92DF92EF92E3
:10094000FF920F931F93CF93DF93EB018091EF0EF4
:100950008A3108F47AC0EA85FB85808191818032F2
:10096000934050F4198618868FEF9FEFDC018C833B
:100970009D83AE83BF836FC0828193816CEA7DE0EB
:100980000E945D7B892B09F460C0EA85FB85848128
:1009900095816CEA7DE00E945D7B892B09F455C04E
:1009A00054E0A52EB12C03E010E0C12CD12C76012F
:1009B0008091EF0E90E0A816B906E4F5EA85FB8574
:1009C000C801880F991FE80FF91F8081918166EB9C
:1009D00073E00E94A57B892B61F14501880C991C6D
:1009E000EA85FB85E80DF91D8081918160E679E05B
:1009F0000E945D7B892B39F0CC0CDD1CEE1CFF1CAA
:100A00006894C0F810C0EA85FB85E80DF91D808167
:100A100091816CEB72E00E945D7B892BB1F0CC0C74
:100A2000DD1CEE1CFF1C0E5F1F4F82E0A80EB11CE8
:100A3000BFCF8501015011091595079519870887C2
:100A40000C30110524F41986188680E009C0CC8288
:100A5000DD82EE82FF828BE090E09983888381E0E3
:100A6000DF91CF911F910F91FF90EF90DF90CF908A
:100A7000BF90AF909F908F9008958F929F92AF926A
:100A8000BF92CF92DF92EF92FF920F931F93CF937B
:100A9000DF93EB018091EF0E8A3108F471C0EA8593
:100AA000FB8580819181843F914060F4198618868E
:100AB0008FEF9FEFDC018C839D83AE83BF838BE040
:100AC00090E066C08281938160E679E00E945D7B60
:100AD000892B09F455C073E0A72EB12C02E010E079
:100AE000C12CD12C76018091EF0E90E0A816B906AA
:100AF000E4F5EA85FB85C801880F991FE80FF91F07
:100B00008081918168E572E00E94A57B892B61F16B
:100B10004501880C991CEA85FB85E80DF91D80814B
:100B2000918160EB74E00E945D7B892B39F0CC0CE5
:100B3000DD1CEE1CFF1C6894C0F810C0EA85FB8524
:100B4000E80DF91D8081918168E572E00E945D7B6E
:100B5000892BB1F0CC0CDD1CEE1CFF1C0E5F1F4F6F
:100B600082E0A80EB11CBFCF850101501109159577
:100B70000795198708870C30110524F41986188603
:100B800080E009C0CC82DD82EE82FF8284E090E0CA
:100B90009983888381E0DF91CF911F910F91FF901E
:100BA000EF90DF90CF90BF90AF909F908F9008957F
:100BB000AF92BF92CF92DF92EF92FF920F931F936B
:100BC000CF93DF93EB018091EF0E863410F480E039
:100BD00086C0EA85FB85828193816EEE72E00E9479
:100BE0005D7B892BA1F3EA85FB85848195816EEE7F
:100BF00072E00E94A57B892B51F3EA85FB858681F3
:100C0000978162E27BE00E945D7B892B01F3EA859C
:100C1000FB858085918562E27BE00E94A57B892B24
:100C2000B1F25CE0A52EB12C05E010E0C12CD12C76
:100C30007601EA85FB85C801880F991FE80FF91F27
:100C4000808191816EEE72E00E945D7B892B09F4B8
:100C5000BECFEA85FB85EA0DFB1D8081918166E6AA
:100C600078E00E94A57B892B39F0CC0CDD1CEE1CB2
:100C7000FF1C6894C0F811C0EA85FB85EA0DFB1DD6
:100C8000808191816EEE72E00E94A57B892B09F430
:100C90009ECFCC0CDD1CEE1CFF1C0E5F1F4F84E0B2
:100CA000A80EB11C0534110521F6EA85FB85E6572F
:100CB000FF4F808191816EEE72E00E945D7B892BF7
:100CC00009F485CF80E290E099878887CC82DD8225
:100CD000EE82FF8288E090E09983888381E0DF9153
:100CE000CF911F910F91FF90EF90DF90CF90BF9029
:100CF000AF9008951F920F920FB60F9211242F9369
:100D00003F938F939F93AF93BF938091BE0F90912A
:100D1000BF0FA091C00FB091C10F3091BD0F23E064
:100D2000230F2D3720F40196A11DB11D05C026E823
:100D3000230F0296A11DB11D2093BD0F8093BE0FFE
:100D40009093BF0FA093C00FB093C10F8091C20FBB
:100D50009091C30FA091C40FB091C50F0196A11D32
:100D6000B11D8093C20F9093C30FA093C40FB09393
:100D7000C50FBF91AF919F918F913F912F910F9090
:100D80000FBE0F901F9018952FB7F8946091BE0F6B
:100D90007091BF0F8091C00F9091C10F2FBF089528
:100DA0003FB7F8948091C20F9091C30FA091C40FE8
:100DB000B091C50F26B5A89B05C02F3F19F001962D
:100DC000A11DB11D3FBF6627782F892F9A2F620F73
:100DD000711D811D911D42E0660F771F881F991FAD
:100DE0004A95D1F70895CF92DF92EF92FF92CF9379
:100DF000DF936B017C01D4DFEB01C114D104E1046A
:100E0000F10481F00E943494CBDF6C1B7D0B683EB3
:100E1000734098F381E0C81AD108E108F108C8517D
:100E2000DC4FEBCFDF91CF91FF90EF90DF90CF9031
:100E300008958230910538F0880F991F880F991F07
:100E400005970197F1F70895789484B5826084BD81
:100E500084B5816084BD85B5826085BD85B58160BE
:100E600085BDEEE6F0E0808181608083E1E8F0E01E
:100E70001082808182608083808181608083E0E84D
:100E8000F0E0808181608083E1EBF0E0808184602C
:100E90008083E0EBF0E0808181608083E1E9F0E035
:100EA000808182608083808181608083E0E9F0E0DE
:100EB000808181608083E1EAF0E0808182608083CC
:100EC000808181608083E0EAF0E0808181608083BE
:100ED000E1E2F1E0808182608083808181608083B3
:100EE000E0E2F1E0808181608083EAE7F0E08081E8
:100EF0008460808380818260808380818160808340
:100F00008081806880831092C100089580930105DC
:100F10000895863308F0865320917B00982F9870AF
:100F2000277F922B90937B0087702091010590E49E
:100F3000299F90011124822B80937C0080917A005C
:100F4000806480937A0080917A0086FDFCCF809146
:100F500078002091790090E0922B089590E0FC01B8
:100F60003197E231F10508F04CC0E955FF4F0C9480
:100F7000E198809180008F7703C0809180008F7D01
:100F800080938000089580918000877FF9CF84B599
:100F90008F7702C084B58F7D84BD08958091B000A5
:100FA0008F7703C08091B0008F7D8093B00008954B
:100FB000809190008F7707C0809190008F7D03C053
:100FC00080919000877F8093900008958091A00089
:100FD0008F7707C08091A0008F7D03C08091A00013
:100FE000877F8093A0000895809120018F7707C0AC
:100FF000809120018F7D03C080912001877F8093A5
:1010000020010895CF93DF9390E0FC01E555F34F65
:101010002491FC01EF50F34F8491882349F190E033
:10102000880F991FFC01E559F24FA591B4918F5A91
:10103000924FFC01C591D4919FB7611108C0F894FB
:101040008C91209582238C93888182230AC0623000
:1010500051F4F8948C91322F309583238C938881AE
:10106000822B888304C0F8948C91822B8C939FBF31
:10107000DF91CF9108950F931F93CF93DF931F922A
:10108000CDB7DEB7282F30E0F901EB59F34F84914B
:10109000F901E555F34F1491F901EF50F34F049125
:1010A0000023C1F0882319F0698358DF6981E02F9C
:1010B000F0E0EE0FFF1FEF5AF24FA591B4919FB7EA
:1010C000F8948C91611103C01095812301C0812B8C
:1010D0008C939FBF0F90DF91CF911F910F91089537
:1010E000CF93DF93282F30E0F901EB59F34F849130
:1010F000F901E555F34FD491F901EF50F34FC49145
:10110000CC2389F081112ADFEC2FF0E0EE0FFF1FD6
:10111000E95CF24FA591B4912C912D2381E090E0F0
:1011200021F480E002C080E090E0DF91CF9108954B
:101130000F931F93762F90E0FC01E555F34F6491D8
:10114000FC01EF50F34FE4917111762FF0E0EE0FB8
:10115000FF1FE95CF24F8591949189019A013F70DC
:10116000472F0E949507611571058105910531F0A2
:101170006F5F7F4F8F4F9F4F9F7003C060E070E0A5
:10118000CB011F910F910895FC01818D228D90E07C
:10119000805C9F4F821B91098F7399270895FC01F2
:1011A000918D828D981731F0828DE80FF11D858D1C
:1011B00090E008958FEF9FEF0895FC01918D828D4F
:1011C000981761F0828DDF01A80FB11D5D968C919B
:1011D000928D9F5F9F73928F90E008958FEF9FEFA6
:1011E000089583EC9AE8892B39F080E090E0892B10
:1011F00019F0C9D1811123C080E090E0892B41F022
:1012000080E090E0892B21F00E94000081111AC03B
:101210008EE69BE8892B39F080E090E0892B19F06D
:101220005DD2811112C089E19CE8892B99F080E0A0
:1012300090E0892B79F0FDD281110AC008950E94B7
:101240000000DACF0E940000E3CF0E940000EBCF45
:101250000C9400000895FC01848DDF01A80FB11DDE
:10126000A35ABF4F2C91848D90E001968F739927DC
:10127000848FA689B7892C93A089B1898C918064C9
:101280008C93938D848D981306C00288F389E02D8A
:1012900080818F7D80830895CF93DF93EC01888DCB
:1012A0008823C1F0EA89FB89808185FD05C0A88972
:1012B000B9898C9186FD0EC00FB607FCF5CF8081F1
:1012C00085FFF2CFA889B9898C9185FFEDCFCE013A
:1012D000C2DFE8CFDF91CF910895CF92DF92FF92E6
:1012E0000F931F93CF93DF931F92CDB7DEB76C019F
:1012F00081E0D60158968C9358975B969C915B97AA
:101300005C968C915C97981307C05096ED91FC9178
:101310005197808185FD2DC0F601038D10E00F5F90
:101320001F4F0F731127F02EF601848DF81210C095
:101330000FB607FCF9CFD6015096ED91FC9151976D
:10134000808185FFF1CFC601698385DF6981ECCF9C
:10135000838DE80FF11DE35AFF4F6083D6015B9642
:101360000C935B975296ED91FC915397808180622C
:101370000CC0D6015696ED91FC915797608350961C
:10138000ED91FC91519780818064808381E090E0B1
:101390000F90DF91CF911F910F91FF90DF90CF9031
:1013A0000895BF92CF92DF92EF92FF92CF93DF9397
:1013B000EC016A017B01B22EE889F98982E0808321
:1013C000411581EE580761057105A1F060E079E0F3
:1013D0008DE390E0A70196010E94A3982150310966
:1013E000410951095695479537952795211580E173
:1013F000380798F0E889F989108260E874E88EE18E
:1014000090E0A70196010E94A3982150310941095B
:1014100051095695479537952795EC85FD8530837D
:10142000EE85FF852083188EEC89FD89B082EA89DC
:10143000FB89808180618083EA89FB898081886063
:101440008083EA89FB89808180688083EA89FB89BF
:1014500080818F7D8083DF91CF91FF90EF90DF902F
:10146000CF90BF900895CF93DF93EC01E881F9818D
:101470000284F385E02D1995EA89FB8980818F7EAE
:101480008083EA89FB898081877F8083EA89FB8961
:1014900080818F778083EA89FB8980818F7D80833B
:1014A0008A8D898FDF91CF910895FC01538D448DF2
:1014B000252F30E0842F90E0821B930B541710F0FF
:1014C000CF960895019708951F920F920FB60F922D
:1014D00011240BB60F922F938F939F93EF93FF934B
:1014E000E091D60FF091D70F8081E091DC0FF09161
:1014F000DD0F82FD12C090818091DF0F8F5F8F73AF
:101500002091E00F821751F0E091DF0FF0E0EA53F5
:10151000F04F958F8093DF0F01C08081FF91EF9195
:101520009F918F912F910F900BBE0F900FBE0F9038
:101530001F9018951F920F920FB60F9211240BB6A1
:101540000F922F933F934F935F936F937F938F935C
:101550009F93AF93BF93EF93FF9386EC9FE07BDE67
:10156000FF91EF91BF91AF919F918F917F916F917B
:101570005F914F913F912F910F900BBE0F900FBE37
:101580000F901F90189586EC9FE0FEDD21E0892BDF
:1015900009F420E0822F08951092C90F1092C80F0D
:1015A00088EE93E0A0E0B0E08093CA0F9093CB0F59
:1015B000A093CC0FB093CD0F86E89BE09093C70F1C
:1015C0008093C60F85EC90E09093D30F8093D20F59
:1015D00084EC90E09093D50F8093D40F80EC90E052
:1015E0009093D70F8093D60F81EC90E09093D90F12
:1015F0008093D80F82EC90E09093DB0F8093DA0F0A
:1016000086EC90E09093DD0F8093DC0F1092DF0F5B
:101610001092E00F1092E10F1092E20F08951F92C6
:101620000F920FB60F9211240BB60F922F938F9338
:101630009F93EF93FF93E0917310F091741080816A
:10164000E0917910F0917A1082FD12C09081809122
:101650007C108F5F8F7320917D10821751F0E09185
:101660007C10F0E0ED59FF4E958F80937C1001C007
:101670008081FF91EF919F918F912F910F900BBEE1
:101680000F900FBE0F901F9018951F920F920FB6DC
:101690000F9211240BB60F922F933F934F935F93AA
:1016A0006F937F938F939F93AF93BF93EF93FF932A
:1016B00083E690E1D0DDFF91EF91BF91AF919F91D3
:1016C0008F917F916F915F914F913F912F910F90EB
:1016D0000BBE0F900FBE0F901F90189583E690E100
:1016E00053DD21E0892B09F420E0822F0895109228
:1016F00066101092651088EE93E0A0E0B0E0809351
:10170000671090936810A0936910B0936A1086E8F0
:101710009BE0909364108093631085ED90E090932C
:10172000701080936F1084ED90E09093721080930E
:10173000711080ED90E0909374108093731081EDA0
:1017400090E0909376108093751082ED90E09093E6
:1017500078108093771086ED90E090937A108093C4
:10176000791010927C1010927D1010927E101092C1
:101770007F1008951F920F920FB60F9211240BB68F
:101780000F922F938F939F93EF93FF93E0911011FC
:10179000F09111118081E0911611F091171182FDE5
:1017A00012C09081809119118F5F8F7320911A114F
:1017B000821751F0E0911911F0E0E050FF4E958F43
:1017C0008093191101C08081FF91EF919F918F91BA
:1017D0002F910F900BBE0F900FBE0F901F9018957A
:1017E0001F920F920FB60F9211240BB60F922F93E8
:1017F0003F934F935F936F937F938F939F93AF9399
:10180000BF93EF93FF9380E091E125DDFF91EF918E
:10181000BF91AF919F918F917F916F915F914F9108
:101820003F912F910F900BBE0F900FBE0F901F9006
:10183000189580E091E1A8DC21E0892B09F420E0F3
:10184000822F0895109203111092021188EE93E0F6
:10185000A0E0B0E08093041190930511A0930611CD
:10186000B093071186E89BE09093011180930011DB
:1018700085E391E090930D1180930C1184E391E046
:1018800090930F1180930E1180E391E090931111CA
:101890008093101181E391E09093131180931211C2
:1018A00082E391E0909315118093141186E391E007
:1018B00090931711809316111092191110921A110A
:1018C00010921B1110921C110895CF92DF92EF928B
:1018D000FF920F931F93CF93DF937C016A01EB017B
:1018E00000E010E00C151D0571F06991D701ED9134
:1018F000FC910190F081E02DC7011995892B19F019
:101900000F5F1F4FEFCFC801DF91CF911F910F9154
:10191000FF90EF90DF90CF9008956115710581F0F1
:10192000DB010D900020E9F7AD0141505109461B44
:10193000570BDC01ED91FC910280F381E02D1994AD
:1019400080E090E00895EF92FF920F931F93CF9362
:10195000DF938C017B01C0E0D0E0F701EC0FFD1FAD
:101960006491662359F0F801A081B181ED91FC9159
:10197000C8011995892B11F02196EFCFCE01DF9187
:10198000CF911F910F91FF90EF900895DC01ED91A1
:10199000FC91DB0114964D915C9115976D917C91B2
:1019A0000280F381E02D1994B8CFDC01ED91FC9118
:1019B0000190F081E02D199462E97BE0AECF0F93A6
:1019C0001F93CF93DF93EC01BEDF8C01CE01F4DFD8
:1019D000800F911FDF91CF911F910F9108950F9369
:1019E0001F93CF93DF93EC01D1DF8C01CE01E4DFB5
:1019F000800F911FDF91CF911F910F9108950F9349
:101A00001F93CF93DF93EC0188DF8C01CE01D4DFED
:101A1000800F911FDF91CF911F910F9108950F9328
:101A20001F93CF93DF93EC01C0DF8C01CE01C4DFA5
:101A3000800F911FDF91CF911F910F9108958F9289
:101A40009F92AF92BF92CF92DF92EF92FF920F934D
:101A50001F93CF93DF93CDB7DEB7A1970FB6F8945E
:101A6000DEBF0FBECDBF7C01C42EE52FCB01D22E31
:101A700019A221E02D1510F02AE0D22E8E010F5D63
:101A80001F4F8D2C912CA12CB12C6C2D7E2FA501DC
:101A900094010E94A3988C2DD29E8019112401508C
:101AA00011098A3014F4805D01C0895CF8018083DB
:101AB000211531054105510521F0C22EE32FCA0140
:101AC000E4CFB801C70129DFA1960FB6F894DEBFB5
:101AD0000FBECDBFDF91CF911F910F91FF90EF907F
:101AE000DF90CF90BF90AF909F908F900895CF924E
:101AF000DF92EF92FF920F931F93CF93DF93EC014E
:101B00006A017B012115310579F4E881F9810190A1
:101B1000F081E02D642FDF91CF911F910F91FF9005
:101B2000EF90DF90CF9019942A303105D9F477FFE8
:101B300018C06DE23ADF8C0144275527BA014C19D1
:101B40005D096E097F092AE0CE0179DF800F911FC0
:101B5000DF91CF911F910F91FF90EF90DF90CF9089
:101B600008952AE0B701A601CE01DF91CF911F9120
:101B70000F91FF90EF90DF90CF9061CF9A01AB0172
:101B8000662757FD6095762FB2CF0F931F93CF93A3
:101B9000DF93EC019A01AB01662757FD6095762F24
:101BA000A6DF8C01CE0108DF800F911FDF91CF915E
:101BB0001F910F9108950F931F93CF93DF93EC0123
:101BC00096DF8C01CE01F8DE800F911FDF91CF915F
:101BD0001F910F9108952115310541F4DC01ED911C
:101BE000FC910190F081E02D642F199428CF0F9380
:101BF0001F93CF93DF93EC019A01462F50E060E0F2
:101C000070E0E9DF8C01CE01D7DE800F911FDF91FC
